:100000000C94910A0C94B20A0C94B20A0C94091044
:100010000C9443100C94B20A0C94B20A0C94B20AD9
:100020000C94B20A0C94B20A0C94B20A0C94B20A60
:100030000C94B20A0C94B20A0C94B20A0C945E139B
:100040000C94B20A0C94B20A0C94B20A0C94B20A40
:100050000C94B20A0C94D1650C94B20A0C94B20AB6
:100060000C94B20A0C944C660C94B20A0C94B20A2A
:100070000C94B20A0C94B20A0C94B20A0C94B20A10
:100080000C94D2790C94B20A0C94B20A0C94B20A71
:100090000C947B660C94B20A0C94B20A0C94B20ACB
:1000A0000C94B20A0C94B20A0C94B20A0C94B20AE0
:1000B0000C94B20A0C94B20A0C94B20A0C94B20AD0
:1000C0000C94B20A0C94B20A0C94B20A0C94B20AC0
:1000D0000C94B20A0C94B20A0C94B20A0C94B20AB0
:1000E0000C94B20A0C940C6D0C94166D0C94026D69
:1000F0000C94C26C0C94426D0C94386D0C942C6D65
:100100000C94206D0C94B20A0C94B20A0C94B20AAE
:100110000C94B20A0C94B20A0C94B20A0C94B20A6F
:100120000C94B20A0C94B20A0C94B20A0C94B20A5F
:100130000C94B20A00801F8098808A81AA81CA81AB
:10014000D2817F81084AD73B3BCE016E84BCBFFD84
:10015000C12F3D6C74319ABD56833DDA3D00C77F97
:1001600011BED9E4BB4C3E916BAAAABE0000008030
:100170003F07634236B79BD8A71A39685618AEBAFC
:10018000AB558C1D3CB7CC5763BD6DEDFD753EF690
:10019000177231BF000000803F08000000BE9224AB
:1001A00049123EABAAAA2ABECDCCCC4C3E000000E0
:1001B00080BEABAAAAAA3E00000000BF00000080DB
:1001C0003F0000000000084178D3BB4387D1133DB6
:1001D000190E3CC3BD4282AD2B3E68EC8276BED97F
:1001E0008FE1A93E4C80EFFFBE01C4FF7F3F0000BE
:1001F000000000000C94C05B0C941F6B0C94A4795D
:100200000C9498800C9495830C945D6D0C940E1155
:100210000C94AD790C9452830C9487740C945474A0
:100220000C94CC6A0C94EE680C947D780C94DC668B
:100230000C941D160C94DC370C94970E0C94E589E5
:100240000C94C4740C94451D0C9421790C940B836C
:100250000C94F7680C947D0E0C94D3740C94CA81A2
:100260000C94C9740C94A94C0C949A760C94496C17
:100270000C942F680C942A150C949D730C9424688C
:100280000C942B740C943C790C9412880C94A969EE
:100290000C94DB740C94AC4D0C94E6820C948A8123
:1002A0000C94AA810C94E3860C947F6E0C941F80AE
:1002B0000C9400800C94BB820C9460670C94428672
:1002C0000C94D2810C94CE740C944E4D0C947F817E
:1002D0000C94646A0C94D8740C9491730C94827886
:1002E0000C9434670C9485786E616E00696E6600BC
:1002F000256300496E76616C6964206932632073FE
:100300007065656420696E20454550524F4D2E2022
:1003100053657474696E67203130206B6269742F85
:10032000730025730A00776474206E6F7420656E05
:1003300061626C65640A005854414C5F5452494DE7
:100340003D25640025730A0025730A005465737403
:1003500020362025730A00546573742035202573D8
:100360000A005465737420342025730A00546573A1
:100370007420332025730A005465737420322025BD
:10038000730A005465737420312025730A00636872
:10039000616E3D25640A0074787077723D25640AA9
:1003A000003530306B0A003235306B0A00313135A0
:1003B0006B0A0035366B0A0033386B0A0025730A66
:1003C00000765F6C6F773D252D332E32660A00254F
:1003D000730A0073656E743D252D75206475703D3C
:1003E000252D752069676E6F7265643D252D75201A
:1003F00074746C5F7A65726F3D252D750A00253720
:100400002E33662025372E33660025352E326620A2
:10041000004572726F72203020566F6C74004E6F00
:100420007420737570706F727465640A004572721F
:100430006F72203020566F6C74004572726F72209C
:100440003020566F6C740062756C6B5F64656C6114
:10045000793D252D750062756C6B3D252D75005617
:10046000616C7565206E6F7420616C6C6F7765646C
:100470000062756C6B3A206D61783D257520737450
:100480006172743D25752C20656E643D25752C20A8
:10049000696E5F7573653D25750A007062323D2592
:1004A000730A007062313D25730A00256C750041A6
:1004B0006C6C6F77656420737065656420312F31D3
:1004C000302F3130302F343030206B6269742F730D
:1004D0000025630074746C3D252D64200074746CD9
:1004E0003D252D6420004E65772074746C3D252DCC
:1004F0006420002563004D533536313120503D25B1
:100500002D372E326620252D372E32666D0A004299
:100510004D5030383520256C642050612020252D29
:10052000372E32666D00256300545F484541545FA5
:100530004944583D252D352E32662000545F4445F0
:10054000573D252D352E3266200041483D252D355D
:100550002E32662000545F53485432583D252D35C5
:100560002E3266200052485F53485432583D252DA4
:10057000352E32662000545F52483D252D342E31F1
:1005800066200052483D252D342E3166200025631B
:1005900000256300256300256300256300726570F4
:1005A0006F72745F616C6C3D007265706F72743D48
:1005B00000256300256300256300256300204F5359
:1005C0004343414C3D2564200020467573653A2025
:1005D00065653D253032782068663D2530327820CB
:1005E0006C663D25303278206C623D2530327800D3
:1005F0004D43553D2530366C780025630074785F97
:100600006C656E3D252D6C752C765F6C6F773D2586
:100610002D6C752C73687432783D252D6C752C62A9
:10062000756C6B3D252D6C75002563004F4B0A00E2
:1006300025630025630025630025630025630025ED
:10064000630025630025630064656275675F616C04
:100650006C3D0064656275673D0064656275673D69
:100660000025730A00646565700A006E6F6E650A86
:1006700000707772733D007764743D25730A0070D3
:1006800062323D25730A007062313D25730A0069AC
:100690006E74725F7365635F70313D252D372E3345
:1006A000660A00696E74725F70313D252D6C640AB4
:1006B00000696E74725F7365635F70303D252D371E
:1006C0002E33660A00696E74725F70303D252D6CA2
:1006D000640A00765F6D63753D252D352E32660AFE
:1006E00000745F6D63753D252D352E32660A0070EE
:1006F0007077723D25730A0064656275673D00720C
:10070000636D643D25730A0025730A006175746F7B
:100710000A006C6F675F6D6F64653D007573625FA3
:100720007077723D25730A0072656C61793D25739F
:100730000A0074746C3D252D640A0052494D455FD2
:10074000616464723D252D642E252D640A006E655A
:10075000696768626F725F7461626C655F73697A02
:10076000653D25640A00765F6C6F773D252D332E3D
:1007700032660A00747870773D25640A0063686108
:100780006E3D25640A0069643D006932635F6275ED
:10079000733D006932635F73706565643D252D6C40
:1007A000750A007478743D25730A00537973746573
:1007B0006D2053756D6D6172790A002530366C7845
:1007C0000041744D65676132353652465232004100
:1007D000744D656761313238524652320041744D72
:1007E0006567613634524652320041744D65676127
:1007F00031323852464131004D43553D006D6173F1
:100800006B3D002C00696E74657276616C3D252D20
:10081000750023252D642C00706232007062310057
:10082000745F686561745F69647800745F6465779C
:1008300000616800705F6D73353631310072685F3A
:10084000736874327800745F736874327800706112
:1008500000700061643400616433006164320061DF
:10086000643100613300613200613100765F696E8E
:100870000072680065727200757074696D65007051
:10088000315F6C73740070315F74007031007030D0
:100890005F6C73740070305F7400703000765F6D51
:1008A000637500745F6D6375007431007400696472
:1008B0000065363400747874002D002B0061757467
:1008C0006F006E6F6E650062756C6B00706F7765A0
:1008D000725F736176655F6C656472790072656CD6
:1008E00061795F6C65647900636F6D70617373002B
:1008F000616363656C007072657300705F7077721E
:10090000006165730070315F6C6564790070305F01
:100910006C656472006576656E74006C6564006F6A
:100920007700706B740074785F6C6564790072781E
:100930005F6C656472006F706572006E6F6E65004B
:100940002530327800765F6164343D252D382E36AF
:1009500066002000765F6164333D252D382E3666B3
:10096000002000765F6164323D252D382E3666000A
:100970002000765F6164313D252D382E36660020DB
:1009800000765F6C696768743D252D382E366600E9
:100990002000765F61323D252D372E336600200022
:1009A000765F61313D252D372E3366002000765F5E
:1009B000696E3D252D352E326600204E65766572B6
:1009C0002D7573656420737461636B203E2025640C
:1009D0002062797465730A00757074696D653D25D0
:1009E0002D642D646179732D253032643A253032BF
:1009F000643A253032642D686F7572730A0074652D
:100A00007374205B6F66667C317C327C337C347C13
:100A1000355D20202020202020202D207465737437
:100A2000206D6F6465730A0D007478205B706B74C1
:100A3000207061796C6F61645D202020202020206F
:100A400020202020202D2073656E6420726164694F
:100A50006F20706B74206B6579626F6172640A0D30
:100A600000776474205B6F6E7C6F66667C74657360
:100A7000745D20202020202020202020202D207781
:100A800061746368646F670A0D00765F6C6F77202E
:100A90005B765F6C6F775D20202020202020202057
:100AA0002020202020202D206C6F77657374207209
:100AB00065706F727420766F6C746167650A0D00E3
:100AC00075706772202020202020202020202020E8
:100AD0002020202020202020202020202D20726572
:100AE000626F6F742076696120626F6F746C6F61E2
:100AF0006465720A0D0075617274205B33386B7C1B
:100B000035366B7C3131356B7C3235306B7C353032
:100B1000306B5D202D20736574207465726D2F75A8
:100B20006172742073706565640A0D00626F6F7482
:100B300020202020202020202020202020202020B5
:100B400020202020202020202D207265626F6F74CD
:100B50000A0D0070777273205B646565707C6E6F40
:100B60006E655D2020202020202020202020202DA8
:100B7000206D637520736C656570206D6F64650A08
:100B80000D007265737420656570726F6D20202092
:100B900020202020202020202020202020202D2048
:100BA000726573746F726520656570726F6D0A0D82
:100BB0000070707772205B6F6E7C6F66665D2020C0
:100BC000202020202020202020202020202D2070C8
:100BD000726F6772616D6D61626C65207077720A09
:100BE0000D0070623220205B6F6E7C6F66665D2048
:100BF00020202020202020202020202020202D20E8
:100C000070726F6772616D6D61626C652070696E84
:100C10002062320A0D0070623120205B6F6E7C6FA3
:100C200066665D20202020202020202020202020FB
:100C300020202D2062756C6B204750494F20706931
:100C40006E0A0D00747874205B737472696E675D50
:100C50002020202020202020202020202020202094
:100C60002D20536574207265706F727420746578DE
:100C70007420737472696E670A0D0074787077203F
:100C80005B31352D305D20202020202020202020A9
:100C9000202020202020202D205458205077722EF4
:100CA0002048696768657374203020283364426D7A
:100CB000290A0D0074746C205B302D31355D2020C5
:100CC0002020202020202020202020202020202024
:100CD0002D2074696D652D746F2D6C6976652066A5
:100CE0006F72207061636B6574730A0D00737320FB
:100CF00020202020202020202020202020202020F4
:100D00002020202020202020202D2073797374653E
:100D10006D2073756D6D6172790A0D0072732020FC
:100D200020202020202020202020202020202020C3
:100D300020202020202020202D20726164696F2037
:100D400073746174730A0D007269205B236E5D20F9
:100D50005B696E745D202020202020202020202030
:100D6000202020202D207265706F727420696E74AF
:100D7000657276616C0A0D0072636D64205B6F6E44
:100D80007C6F66665D2020202020202020202020EF
:100D9000202020202D20616C6C6F7720636D6420F3
:100DA00066726F6D206E65746F726B0A0D007265EE
:100DB000205B236E5D205B2B7C2D5D205B6D617362
:100DC0006B7C6175746F2C6D61736B5D202D206D74
:100DD0006F7465207265706F7274207365742F6D07
:100DE0006F646966790A0D006F772020202020202B
:100DF00020202020202020202020202020202020F3
:100E0000202020202D206F6E652D7769726520735C
:100E1000656E736F72730A0D006C6F67205B61758E
:100E2000746F7C6F6E7C6F66665D202020202020B2
:100E300020202020202D206D6F7465732064617444
:100E400061206F6E205553420A0D006E65205B666F
:100E50006C7573685D202020202020202020202019
:100E6000202020202020202D206E65696768626F79
:100E700072207461626C650A0D0065727220202018
:100E80002020202020202020202020202020202062
:100E90002020202020202D206572726F7220737414
:100EA0006174730A0D006D637520202020202020BE
:100EB0002020202020202020202020202020202032
:100EC00020202D206D637520696E666F0A0D006904
:100ED0003263205B70726F62657C7370656564203D
:100EE000236E5D20202020202020202D20693263C9
:100EF0002070726F6265206275737C736574206206
:100F000075732073706565640A0D006964205B72F7
:100F1000657365745D202020202020202020202063
:100F2000202020202020202D2069642068616E640C
:100F30006C696E670A0D0068756D202020202020E6
:100F400020202020202020202020202020202020A1
:100F50002020202D2068756D69646974792073657F
:100F60006E736F720A0D0072656C6179205B6F6E33
:100F70007C6F66667C73746174735D202020202012
:100F80002020202D2072656C6179206E6574776F4A
:100F9000726B207265706F7274730A0D0064652045
:100FA0005B6D61736B5D202020202020202020209D
:100FB0002020202020202020202D206465627567BD
:100FC0000A0D006368616E205B31312D32365D2081
:100FD0002020202020202020202020202020202D04
:100FE000206368616E2031312D32362028322E3454
:100FF00030352D32343830204D687A290A0D00639F
:10100000616C69205B5B765F696E7C61317C61320B
:101010005D20766F6C747C72657365747C6E6F6E28
:10102000655D202D2063616C6962726174650A0DD3
:101030000062756C6B205B5B73686F777C666C75A8
:1010400073685D205B7365742074687273682064D4
:10105000656C61795D5D20202D2062756C6B696E19
:1010600067207061636B657473200A0D00616463AF
:101070002020202020202020202020202020202070
:101080002020202020202020202D2073686F772012
:10109000765F696E2C2061312C20613220766F6C76
:1010A00074616765730A0D007520202020202020C0
:1010B0002020202020202020202020202020202030
:1010C000202020202D20757074696D650A0D007632
:1010D0002020202020202020202020202020202010
:1010E00020202020202020202020202D2076657206
:1010F00073696F6E0A0D00682020202020202020B8
:1011000020202020202020202020202020202020DF
:101110002020202D2068656C700A0D002563007565
:101120006E6B6E6F776E20636D640A00484D4335B9
:1011300038383300257300257300202573002025DF
:10114000362E32662000253032780074656D705F6F
:1011500065787465726E3D252D362E326600202529
:1011600073002025362E3266204F6E2D426F61723D
:101170006400253032780074656D705F626F617253
:10118000643D252D362E3266000A0042756C6B20B8
:1011900072656D3A2073746172743D25752C2065FB
:1011A0006E643D25752C20696E5F7573653D2575F0
:1011B0000A0042756C6B206164643A20737461723A
:1011C000743D25752C20656E643D25752C20696E57
:1011D0005F7573653D25750A0042756C6B207468F8
:1011E000726573683A2074696D65723D25750A00F1
:1011F000503A20256C642050612020252D372E3256
:1012000066206D0A004932433A20004A5441472083
:10121000726573657474210A005761746368646F42
:1012200067207265736574210A0042726F776E6F72
:101230007574207265736574210A0045787465724F
:101240006E616C207265736574210A00506F77655A
:10125000722D6F6E207265736574212E0A004F6EB9
:101260006C696E650A00526F7574696E6720456E11
:1012700061626C65640A0052504C20456E61626C7C
:1012800065640A0025732025732C206368616E6EE7
:10129000656C202575202C20636865636B20726166
:1012A000746520257520487A20747820706F7765E2
:1012B000722025750A000A2A2A2A2A2A2A2A426F17
:1012C0006F74696E672025732A2A2A2A2A2A2A0A15
:1012D000004A544147207265736574210A005761C2
:1012E000746368646F67207265736574210A0042D5
:1012F000726F776E6F7574207265736574210A0062
:1013000045787465726E616C207265736574210A2C
:1013100000506F7765722D6F6E2072657365742E45
:101320000A00726E67206973737565732025640AFD
:1013300000454550524F4D20697320636F7272759E
:1013400070742C20726577726974696E6720776992
:1013500074682064656661756C74732E0A006C6F26
:1013600063616C686F73740041544D454741323579
:10137000367266723200020000FFFE000001452056
:1013800025642E256420636C6F636B20256C7520AB
:1013900063707520256C75206C706D20256C752030
:1013A00069727120256C7520676C656420256C75E9
:1013B00020796C656420256C7520726C656420252D
:1013C0006C7520747820256C75206C697374656E5B
:1013D00020256C752073656E736F727320256C7594
:1013E0002073657269616C20256C750A0000407A73
:1013F00010F35A00A0724E18090010A5D4E800009E
:10140000E87648170000E40B54020000CA9A3B003B
:101410000000E1F505000080969800000040420FB2
:10142000000000A08601000000102700000000E876
:1014300003000000006400000000000A000000003B
:10144000000100000000002C76D888DC674F0823DC
:10145000DFC1DFAE59E1B1B796E5E3E453C63AE642
:1014600051997696E8E6C28426EB898C9B62ED4022
:101470007C6FFCEFBC9C9F40F2BAA56FA5F4900571
:101480005A2AF75C936B6CF9676DC11BFCE0E40DA5
:1014900047FEF520E6B500D0ED902E030094357799
:1014A000050080841E080000204E0A000000C80CC1
:1014B000333333330F986E12831141EF8D2114892A
:1014C0003BE65516CFFEE6DB18D1844B381BF77C84
:1014D0001D901DA4BBE424203284725E228100C9C9
:1014E000F124ECA1E53D274E414E494E495459495E
:1014F0004E46CDCCCC3D0AD7233C17B7D13877CC5C
:101500002B329595E6241FB14F0A000020410000C0
:10151000C84200401C4620BCBE4CCA1B0E5AAEC579
:101520009D7411241FBECFEFD1E8DEBFCDBF00E018
:101530000CBF1AE0A0E0B2E0E8E2FEE201E00BBF7F
:1015400002C007900D92A634B107D9F729E3A6E4AB
:10155000BAE001C01D92AD3FB207E1F70E94AB6453
:101560000C9412970C9400002F923F924F925F922E
:101570006F927F928F929F92AF92BF92CF92DF92A3
:10158000EF92FF920F931F93CF93DF93CDB7DEB708
:1015900063970FB6F894DEBF0FBECDBF6C014B0151
:1015A0002A01FC0117821682838181FF43C3AE01A9
:1015B0004F5F5F4F3A01F6019381F40193FD8591EE
:1015C00093FF81914F01882309F430C3853239F4A8
:1015D00093FD859193FF81914F01853239F4B601D6
:1015E00090E00E94DE9352012501E5CF10E0F12C3E
:1015F00020E02032A0F48B3269F030F4803259F0D0
:10160000833269F420612CC08D3239F0803339F493
:10161000216026C02260246023C0286021C027FDED
:1016200027C030ED380F3A3078F426FF06C0FAE0D4
:101630001F9F300D1124132F13C04AE0F49E300D6C
:101640001124F32E20620CC08E3221F426FDEEC24E
:10165000206406C08C3611F4206802C0883641F43C
:10166000F40193FD859193FF81914F018111C1CFC9
:101670009BEB980F933018F42061805E06C09BE9C5
:10168000980F933008F071C12F7E26FF16E02F735C
:10169000322E853619F42064322E08C0863621F4A5
:1016A000F22FF0683F2E02C01111115037FE07C013
:1016B0001C3350F4EE24E394E10E27E00BC0183005
:1016C00038F027E017E005C027E04CE3E42E02C025
:1016D000212FE12C520144E0A40EB11CF2016081E3
:1016E0007181828193810E2DA3010E9455922C015C
:1016F000098100FF02C003FF07C031FC08C032FEB1
:1017000009C030E2232E07C02DE2222E04C09BE246
:10171000292E01C0212C802F8C7019F0211068C255
:10172000A8C237FE0FC0E40C04FF04C08A818133D5
:1017300009F4EA941E1474F5F8E0FE1578F588E0D3
:10174000E82E2CC036FC2AC0812F90E08415950528
:101750009CF02CEF42162FEF520674F0432D406898
:10176000342E0AC0E2E0F0E0EC0FFD1FE10FF11DA6
:101770008081803319F411501111F4CF37FE0EC05F
:10178000EE24E394E10E812F90E0481659062CF4E4
:10179000141904C0EE24E39401C010E037FE06C023
:1017A0001414150434F4C201019605C085E090E0DC
:1017B00002C081E090E021100196112331F0212F29
:1017C00030E02F5F3F4F820F931F2F2D30E08217A5
:1017D000930714F4F81A01C0F12C832D897049F491
:1017E000FF2039F0B60180E290E00E94DE93FA9487
:1017F000F7CF222029F0B601822D90E00E94DE93DF
:1018000033FC09C0FF2039F0B60180E390E00E946C
:10181000DE93FA94F7CF37FE5AC0942D852D57FEEC
:1018200002C090E080E0292E382E20E030E0A201B6
:101830004E1951095D874C87A201421953095F87F0
:101840004E87612F70E044275527461B570B598B55
:10185000488B5FEF2516350649F4B6018EE290E01D
:101860002A8B3B8B0E94DE933B892A8942145304C6
:101870006CF04C855D854215530544F4EE85FF857B
:10188000E20FF31FE60DF71D818101C080E351E0F7
:10189000251A31082F5F3F4F48895989241635068C
:1018A0004CF0B60190E02A8B3B8B0E94DE932A8994
:1018B0003B89CFCF2414350439F49A81963318F438
:1018C000953311F404FF81E3B60190E04BC08A81A7
:1018D000813309F00F7EB60190E00E94DE93111172
:1018E00005C034FC18C085E690E017C0B6018EE252
:1018F00090E00E94DE9382E0EE24E394E80EF30190
:10190000E80FF11D8081B60190E00E94DE93115036
:101910008E2D91F7E6CF85E490E0B6010E94DE932C
:1019200057FC05C04114510439F404FF05C051941B
:10193000419451088DE201C08BE2B60190E00E9413
:10194000DE9380E39AE0491651042CF08F5F5AE051
:10195000451A5108F7CFB60190E00E94DE93B60118
:10196000C201C0960E94DE9357C1833631F083379F
:1019700079F0833509F058C021C05201E2E0AE0E83
:10198000B11CF2018081898301E010E0230114C0C1
:101990005201F2E0AF0EB11CF2014080518026FFEF
:1019A00003C0612F70E002C06FEF7FEFC2012A8B8E
:1019B0000E948A938C012A892F7715C05201F2E088
:1019C000AF0EB11CF2014080518026FF03C0612F91
:1019D00070E002C06FEF7FEFC2012A8B0E943F933D
:1019E0008C012A892068322E23FD1AC08F2D90E0A9
:1019F00008171907A8F4B60180E290E00E94DE9370
:101A0000FA94F4CFF20137FC859137FE81912F01D2
:101A1000B60190E00E94DE93F110FA940150110992
:101A20000115110579F7F8C0843611F0893659F59A
:101A3000520127FF09C0F4E0AF0EB11CF201608132
:101A40007181828193810AC0F2E0AF0EB11CF20174
:101A500060817181072E000C880B990B2F76322E36
:101A600097FF09C090958095709561957F4F8F4F36
:101A70009F4F2068322E2AE030E0A3010E94EF94AD
:101A8000E82EE6183FC0022F853721F40F7E2AE0AA
:101A900030E01DC0097F8F3691F018F4883559F079
:101AA000C5C0803719F0883711F0C0C0006104FF4D
:101AB00009C0046007C024FF08C0066006C028E013
:101AC00030E005C020E130E002C020E132E0520108
:101AD00007FF09C0F4E0AF0EB11CF2016081718113
:101AE0008281938108C0F2E0AF0EB11CF2016081E7
:101AF000718180E090E0A3010E94EF94E82EE61847
:101B00000F77302E36FE0BC0332D3E7FE11650F49A
:101B100034FE0AC032FC08C0332D3E7E05C00E2DB7
:101B2000332D03C00E2D01C0012F34FF0CC0FE0168
:101B3000EE0DF11D8081803311F4397E08C032FF33
:101B400005C00E5F04C0832F867809F00F5F33FD58
:101B500013C030FF06C01E2D0F1518F41F0D101BEB
:101B60000F2D0F1568F4B60180E290E03B8B0E94C8
:101B7000DE930F5F3B89F5CF0F1510F4F01A01C00B
:101B8000F12C34FF12C0B60180E390E03B8B0E9441
:101B9000DE933B8932FF17C031FD03C088E790E038
:101BA00002C088E590E0B6010CC0832F867859F01A
:101BB00031FF02C08BE201C080E237FD8DE2B60149
:101BC00090E00E94DE93E11638F4B60180E390E0E5
:101BD0000E94DE931150F7CFEA94F301EE0DF11D50
:101BE0008081B60190E00E94DE93E110F5CF14C031
:101BF000F4E0FF1558F584E0F81A33FE1EC02110FA
:101C000026C003FF2AC008EE12E0F32DF0713F2E2C
:101C1000F8018491811124C0FF2009F4E5CCB601BC
:101C200080E290E00E94DE93FA94F6CFF60186817E
:101C3000978126C08FEF9FEF23C0B60180E290E02E
:101C40000E94DE93FA94F110F8CFD9CFF12CB601AF
:101C5000822D90E00E94DE93D4CF0CEE12E0D5CF1F
:101C600031108052B60190E00E94DE930F5F1F4F4B
:101C7000CFCF23E02F1510F483E0BECFF12CC1CFDE
:101C800063960FB6F894DEBF0FBECDBFDF91CF9144
:101C90001F910F91FF90EF90DF90CF90BF90AF908A
:101CA0009F908F907F906F905F904F903F902F907C
:101CB00008958115910511F00197F1F7089581E7D5
:101CC00096E09F938F930E942A9480916602909150
:101CD0006702A0916802B09169020F900F9093FF84
:101CE00003C08BE696E002C085E696E09F938F9353
:101CF0000E942A940F900F900895E091F81CEF73C2
:101D0000F0E0E75BF24E80838091F81C8F5F809358
:101D1000F81C809199358860809399354CE452E0A5
:101D200061E1CA010E94C17080E090E00895CF9304
:101D3000DF93EC0180919F139091A013A091A113C8
:101D4000B091A21386FF1DC08E811F928F938D814B
:101D50001F928F938C811F928F938B811F928F93F1
:101D60008A811F928F9389EE92E09F938F930E94B6
:101D700016948DB79EB70C960FB6F8949EBF0FBE03
:101D80008DBFBE0181E99AE00E94BA71BE0188E070
:101D900092E0DF91CF910C944B7252985A981DBAF1
:101DA000E9E6F0E0808180628083EA9A53985B984C
:101DB000EB9A808180688083E8E6F0E08081816032
:101DC00080830895EEEAFDE1118212821082089567
:101DD000CF92DF92EF92FF920F931F93CF93DF93F7
:101DE000EC019B018091AE1D843108F0BBC0809155
:101DF000B01D64E10E94A5889093B01DC090CB30C7
:101E0000D090CC30E090CD30F090CE30092F10E063
:101E10008DE8989FD0011124A255B24E1396CD9211
:101E2000DD92ED92FC9216974115510559F0FA0199
:101E30008081FD01EA57FF4F8083FA018181A95714
:101E4000BF4F8C932097A9F089819DE8909FF00166
:101E5000919FF00D1124E255F24EDF01A657BF4FBE
:101E60008C93E557FF4F88818F70808388818F70B6
:101E7000808321153105E1F1D90116964C91169711
:101E80005DE8509FC001519F900D11248255924EE4
:101E9000FC01E757FF4F408315964C9115973197FA
:101EA000408334961B964D915D916D917C911E9768
:101EB000452F562F672F7727518340837C01BEE83B
:101EC000EB0EF11CF9012385348545855685A4E682
:101ED000B0E00E944089672F782F892F992724E648
:101EE00030E040E050E00E94D988D7016D937C93A8
:101EF0008DE8809FD001819FB00D1124AB54B24E6C
:101F0000FE0132968FE701900D928A95E1F780915C
:101F1000B01D8F5F8093B01D9091AE1D9F5F909319
:101F2000AE1D40919F135091A0136091A113709129
:101F3000A21360FF2DC01F929F931F928F938091D9
:101F4000AF1D1F928F9382EB91E19F938F930E941D
:101F50002A94EDB7FEB738960FB6F894FEBF0FBEC1
:101F6000EDBF16C08091DB309091DC30A091DD3068
:101F7000B091DE300196A11DB11D8093DB309093AE
:101F8000DC30A093DD30B093DE3080E090E002C022
:101F900081E090E0DF91CF911F910F91FF90EF9042
:101FA000DF90CF9008952091AE1D222361F18091A2
:101FB000AF1D8F5F21502093AE1D64E10E94A58864
:101FC0009093AF1D40919F135091A0136091A11366
:101FD0007091A21360FF1AC01F922F938091B01DC1
:101FE0001F928F931F929F938BE891E19F938F9302
:101FF0000E942A948DB79EB708960FB6F8949EBF9C
:102000000FBE8DBF03C080E090E0089581E090E0B6
:1020100008951F920F920FB60F9211248F939F93E2
:10202000AF93BF938091680080FF24C08091743586
:1020300090917535A0917635B09177350196A11DB7
:10204000B11D8093743590937535A0937635B09318
:10205000773580919F139091A013A091A113B09117
:10206000A21387FF07C0749882E090E090939202D9
:1020700080939102BF91AF919F918F910F900FBE6E
:102080000F901F9018951F920F920FB60F92112468
:102090008F939F93AF93BF938091680080FF24C07C
:1020A0008091783590917935A0917A35B0917B35D2
:1020B0000196A11DB11D8093783590937935A09339
:1020C0007A35B0937B3580919F139091A013A091A6
:1020D000A113B091A21390FF07C0739882E090E023
:1020E0009093920280939102BF91AF919F918F91B3
:1020F0000F900FBE0F901F90189580937C008091D9
:102100007B00877F80937B0080917C00806C809334
:102110007C0085E080937A0080917A0080688093CB
:102120007A0080917B0087FFFCCF80917B0085FF48
:10213000FCCF80917A00806480937A0080917A004D
:1021400086FDFCCF109279001092780084E090E038
:1021500060E070E020917A00206420937A00209162
:102160007A0026FDFCCF2091780030917900620F33
:10217000731F019779F710927C0080917A008F7716
:1021800080937A00769567957695679580E090E0E4
:102190000E94AE8C089580E00E947D1020918902FB
:1021A00030918A0240918B0250918C020E94A88E3D
:1021B00021EE3AE744E95EE30E94198B08950F93FC
:1021C0001F93CF93DF930FE110E0CBE5DEE00093A8
:1021D000510182E991E00E94590E8091510185FDE3
:1021E0000DC00031110521F02CF0CB54D10903C0F2
:1021F000C4ECD9E0E29701501109E9CFBE0180E0BB
:1022000090E00E94AE8C20E030E04AE754E40E9467
:10221000FC8BDF91CF911F910F910895CF93DF93A6
:10222000EC0188819981009799F08331924121F0E6
:102230001982188283E011C0623171F40E94DF10AC
:102240006093C7307093C8308093C9309093CA3080
:1022500083E192E19983888381E0DF91CF910895B2
:1022600080917B00886080937B0089EC80937C0068
:1022700085E080937A0080917A00806880937A006C
:1022800080917B0087FFFCCF80917B0085FFFCCF96
:1022900080917A00806480937A0080917A0086FD34
:1022A000FCCF80917A00806480937A0080917A00DC
:1022B00086FDFCCF609178007091790080917A0062
:1022C0008F7780937A0080E090E00E94AE8C27EDBB
:1022D00033EA40E95FE30E94A88E26E636E648E846
:1022E00053E40E94188B0895CF92DF92EF92FF92F1
:1022F0001F93CF93DF93CDB7DEB729970FB6F8942E
:10230000DEBF0FBECDBF6C01109299138FEF89878E
:1023100081E0E82E8DE1F82E10E089858823E9F12F
:102320001830D9F1BE016F5F7F4FCE0109960E9430
:10233000825F99859F3F11F09E3F19F49093991306
:102340002CC0CE010196C114D10481F40E949C5F7F
:1023500080939635AEE8B5E3FE01319688E08E0FA6
:1023600091919D938E13FCCF81E018C00E949C5FD9
:10237000F7018087FE01319620E030E08191D7019E
:10238000A20FB31F8C932F5F3F4F28303105B1F759
:102390001F5FF9E0EF0EF11CC0CF812F29960FB619
:1023A000F894DEBF0FBECDBFDF91CF911F91FF909C
:1023B000EF90DF90CF90089589E891E19F938F93FC
:1023C0000E942A940F900F9008952F923F924F925F
:1023D0005F926F927F928F929F92AF92BF92CF92B5
:1023E000DF92EF92FF920F931F93CF93DF93EC0155
:1023F0005B01009711F427E003C0019749F426E040
:102400004AE250E06BE270E089E290E00E945C5E9C
:10241000CE010E9474119E0126563C4E6901D901DD
:102420008C93CD2B69F0C1E0DDE1E12CF12C8EE342
:10243000282E81E1382E9AE3892E91E1992E9EC0B3
:102440008EE895E30E942D60BC01990F880B990BD3
:102450000E94B08C6B017C01AB2869F020E030E079
:1024600048EC52E40E94FC8B9F938F937F936F9371
:1024700087E791E1A4C0CEE8D5E302E711E18991B5
:102480001F928F931F930F930E942A940F900F9087
:102490000F900F90B5E3C639DB0789F720E030E0F5
:1024A00048EC52E4C701B6010E94FC8B9F938F93C6
:1024B0007F936F9382E691E19F938F930E942A947A
:1024C0000F900F900F900F900F900F908091963576
:1024D000811103C08CE893E002C088E193E09F93F0
:1024E0008F938EE591E19F938F930E942A940F9092
:1024F0000F900F900F906DC000E010E0FE01E00F14
:10250000F11F80811F928F93A6E4B1E1BF93AF9337
:102510000E942A940F5F1F4F0F900F900F900F9003
:102520000830110559F720E030E048EC52E4C301CF
:10253000B2010E94FC8B9F938F937F936F933F9286
:102540002F920E942A940F900F900F900F900F904F
:102550000F908885811151C08CE893E09F938F93F1
:102560009F928F920E942A940E94DC11FFEFEF1A33
:10257000FF0A29960F900F900F900F90D6018C9123
:1025800090E0E816F906E4F5CE010E942D60BC014A
:10259000990F880B990B0E94B08C2B013C01A11460
:1025A000B10409F4A9CF20E030E048EC52E40E94E5
:1025B000FC8B9F938F937F936F938BE491E19F9319
:1025C0008F930E942A940F900F900F900F900F906E
:1025D0000F90DF91CF911F910F91FF90EF90DF90BF
:1025E000CF90BF90AF909F908F907F906F905F90B3
:1025F0004F903F902F900C94DC1188E193E0AECF88
:10260000DF91CF911F910F91FF90EF90DF90CF90CE
:10261000BF90AF909F908F907F906F905F904F9002
:102620003F902F900895CF93DF931F921F92CDB7C5
:10263000DEB7EEE8F5E38181898387818A83CE0165
:1026400001960E94EF740F900F90DF91CF91089543
:10265000CF93DF93EC0120918E3530918F354091EF
:10266000903550919135609192357091933580916C
:10267000943590919535AFEF0E940C8BE1F427E0F3
:102680004AE250E06BE270E089E290E00E945C5E1A
:1026900080E090E00E947411C656DC4E888349E0C9
:1026A00050E06EE070E08EE895E30E94F596DF91D1
:1026B000CF910C941313DF91CF9108951F920F9235
:1026C0000FB60F9211240BB60F92FF920F931F9328
:1026D0002F933F934F935F936F937F938F939F932A
:1026E000AF93BF93CF93DF93EF93FF93809199358F
:1026F0008260809399358091660286FD2B9A809145
:10270000660287FD2B9A8091910290919202181691
:10271000190614F4749A739A80919F139091A013E0
:10272000A091A113B091A21385FF02C07498739871
:10273000809106029091070201979093070280937F
:102740000602892B09F04CC18091540A9091550AD8
:1027500001969093550A8093540A8091CB309091C2
:10276000CC30A091CD30B091CE300196A11DB11DDD
:102770008093CB309093CC30A093CD30B093CE30BB
:1027800080E190E0909307028093060280916602B8
:1027900080FD02C01D9B05C010929E1310929D13D8
:1027A00006C081E090E090939E1380939D138091EA
:1027B0009F139091A013A091A113B091A21397FF22
:1027C00008C080919D1390919E13892B49F0749AB3
:1027D000739808EA1CE1C0EED0E3FF24F39421C013
:1027E000739A7498F6CF8091540A9091550A019685
:1027F0000E94B188892BE1F0F8016085718561152F
:102800007105A1F5F801608571856115710509F003
:102810003FC0065F1F4F2596F0E3C43FDF0709F472
:102820004CC0F801608571856115710529F3DBCF16
:102830004281417020E030E050E060E070E080E0F4
:1028400090E0A0E00E940C8BB9F2779880919F13E2
:102850009091A013A091A113B091A21392FFCCCF9D
:1028600074981092920210929102C6CF8091540AED
:102870009091550A01960E94B188892B19F61C8205
:102880001B82AE0162E184E292E00E94C170BACF85
:102890008091540A9091550A0E94B188892B09F0C1
:1028A000B8CFF8821A8309831C821B82AE0162E1D1
:1028B00082E492E00E94C170ACCF60916C02709192
:1028C0006D0261157105A1F18091540A9091550A2C
:1028D0000E94B188892B61F580917435909175358E
:1028E000A0917635B09177354091BD285091BE28A2
:1028F0006091BF287091C028841B950BA60BB70B65
:102900008093D01C9093D11CA093D21CB093D31C65
:102910008091743590917535A0917635B091773569
:102920008093BD289093BE28A093BF28B093C02861
:1029300060916A0270916B0261157105A1F180913D
:10294000540A9091550A0E94B188892B61F58091B3
:10295000783590917935A0917A35B0917B35409159
:10296000C1285091C2286091C3287091C428841B4B
:10297000950BA60BB70B8093D41C9093D51CA093FA
:10298000D61CB093D71C8091783590917935A09161
:102990007A35B0917B358093C1289093C228A0935B
:1029A000C328B093C4288091660286FD2B9880913D
:1029B000660290916702A0916802B091690291FF4E
:1029C0000FC00E94E7698A3119F0C1E0C80F01C049
:1029D000CBE00E9424688C2F0E94FF690E94EE6861
:1029E00040E050E060E085EB92E00E94C170FF9112
:1029F000EF91DF91CF91BF91AF919F918F917F9197
:102A00006F915F914F913F912F911F910F91FF9087
:102A10000F900BBE0F900FBE0F901F9018958091D6
:102A2000F81C9091DF30891B08950E940F158823B0
:102A300071F0E091DF30EF73F0E0E75BF24E808100
:102A400090E02091DF302F5F2093DF3008958FEFEB
:102A50009FEF0895CF93DF93EC011092850A1092B7
:102A6000840A888199810097C1F0863E934021F0C5
:102A70001982188283E0BDC0613109F0B9C00E949B
:102A8000151599279093800A80937F0A8D309105C0
:102A900009F444C08F3F910549F40E940F1581113C
:102AA000EECF86EE93E099838883A2C082319105B0
:102AB00009F45AC08F37910509F052C080917D0A00
:102AC00090917E0A181619060CF56091F7397091ED
:102AD000F83988E090E00E94DE936091F7397091B8
:102AE000F83980E290E00E94DE936091F7397091AE
:102AF000F83988E090E00E94DE9380917D0A909101
:102B00007E0A019790937E0A80937D0A80917D0AC8
:102B100090917E0A8F37910509F0BFCF1092DF3078
:102B20001092F81C80917D0A90917E0AFC01EC5075
:102B3000FF4C10829093850A8093840A10927E0A3B
:102B400010927D0A8091973590919835009709F4FD
:102B5000A4CF40E050E0609197130E94C1709DCFD8
:102B60008830910571F5AACF6091F7397091F839E5
:102B70008DE090E00E94DE9310927C0A10927B0A16
:102B800020917B0A30917C0A80917D0A90917E0A87
:102B9000281739070CF0BACFF901EC50FF4C8081AF
:102BA0006091F7397091F83990E00E94DE9380913E
:102BB0007B0A90917C0A019690937C0A80937B0A11
:102BC000DFCF6091F7397091F8390E94DE93209140
:102BD0007D0A30917E0A80917F0AF901EC50FF4C0A
:102BE00080832F5F3F4F30937E0A20937D0A8ECFE4
:102BF00081E0DF91CF91089580919D1390919E1374
:102C0000892BD1F08091660290916702A0916802B1
:102C1000B091690293FD10C00E94246883B7817F40
:102C2000866083BFF89483B7816083BF789488956A
:102C300083B78E7F83BF78940895CF93DF93FC0191
:102C4000208131812115310551F02634324129F09E
:102C5000FC011182108283E015C0653891F4EC010B
:102C60000E9422670E94FC1540E050E065E88091D8
:102C7000E1149091E2140E94C17086E492E199837C
:102C8000888381E0DF91CF910895CF93DF931F92E6
:102C90001F92CDB7DEB7892B81F05F934F9387E307
:102CA00091E19F938F9369837A830E942A940F9076
:102CB0000F900F900F907A8169817F936F9384E3D7
:102CC00091E19F938F930E942A940F900F900F9001
:102CD0000F900F900F90DF91CF910895EF92FF9298
:102CE0000F931F93CF93DF930E94226780EB0E9484
:102CF000B76081111CC00E9414618091C52C909115
:102D0000C62C81609093C62C8093C52C81E293E001
:102D10009F938F9384E391E19F938F930E942A94D2
:102D20000F900F900F900F90C1E0D0E002C0C0E074
:102D3000D0E01EB11470729A64E278E680E090E010
:102D40000E9494600E9422678EE40E94B760811105
:102D500017C00E9414618091C52C9091C62C82608E
:102D60009093C62C8093C52C7E018FEFE81AF80A49
:102D700048E259E069E273E0CE010E944516E7019E
:102D8000111101C0729864E278E680E090E00E9440
:102D900094600E9422678EEE0E94B760811116C077
:102DA0000E9414618091C52C9091C62C84609093F0
:102DB000C62C8093C52C8E010F5F1F4F48E259E04F
:102DC00061E373E0CE010E944516E80164E278E613
:102DD00080E090E00E9494600E94226786EA0E9450
:102DE000B760811116C00E9414618091C52C90912A
:102DF000C62C88609093C62C8093C52C8E010F5FE3
:102E00001F4F48E259E068E373E0CE010E94451687
:102E1000E80164E278E680E090E00E9494600E941D
:102E200022678CE30E94B76081111EC00E9414616A
:102E30008091C52C9091C62C80619093C62C809374
:102E4000C52C8E010F5F1F4F48E259E060E473E02C
:102E5000CE010E9445168CE291E19F938F930E94D0
:102E60002A940F900F90E80164E278E680E090E009
:102E70000E9494600E94226782ED0E94B7608111D7
:102E800016C00E9414618091C52C9091C62C80625E
:102E90009093C62C8093C52C8E010F5F1F4F48E284
:102EA00059E068E473E0CE010E944516E80164E24F
:102EB00078E680E090E00E9494600E94226780E8BB
:102EC0000E94B760811116C00E9414618091C52CC8
:102ED0009091C62C91609093C62C8093C52C8E0146
:102EE0000F5F1F4F48E259E061E573E0CE010E9499
:102EF0004516E80164E278E680E090E00E94946084
:102F00000E94226780ED0E94B760811116C00E9466
:102F100014618091C52C9091C62C80689093C62C2A
:102F20008093C52C8E010F5F1F4F48E259E067E583
:102F300073E0CE010E944516E80164E278E680E085
:102F400090E00E9494600E9422678CEE0E94B7601D
:102F5000811116C00E9414618091C52C9091C62CDD
:102F600092609093C62C8093C52C8E010F5F1F4FEB
:102F700048E259E06FE573E0CE010E944516E80192
:102F800007E010E064E278E680E090E00E94946060
:102F90000E9422678CE70E94B760811113C00E94D3
:102FA00014618091C52C9091C62C80649093C62C9E
:102FB0008093C52C48E259E066E673E0CE010E949A
:102FC000451603C001501109E9F60E941461DF9112
:102FD000CF911F910F91FF90EF900C94DC11CF9344
:102FE000DF931F921F92CDB7DEB74A8369830E9499
:102FF000EB606981862F0E941C614A81842F0E94A8
:103000001C610F900F90DF91CF910C941461AF92DF
:10301000BF92CF92DF92EF92FF920F931F93CF93C5
:10302000DF9300D0CDB7DEB7182F022F4A835B8322
:1030300069830E94EB606981862F0E941C61812F49
:1030400081600E9412614A81A42E5B81B52E10E03E
:10305000E12CF12C680181E0C81AD108E016F106D4
:1030600089F0EC14FD0419F40E94376102C00E943B
:103070002D61F5018083FFEFEF1AFF0A8FEFA81A89
:10308000B80AECCF0F900F900F90DF91CF911F9166
:103090000F91FF90EF90DF90CF90BF90AF900C9486
:1030A0001461BF92CF92DF92EF92FF920F931F9322
:1030B000CF93DF93CDB7DEB760970FB6F894DEBF3E
:1030C0000FBECDBFF82EE42E6623D9F18E010F5F1F
:1030D0001F4F80E1F80111928A95E9F728E0A801D5
:1030E00068E980EB0E940718FF2041F08FE693E02B
:1030F0009F938F930E9416940F900F9026E7C22EF5
:1031000023E0D22E37E0B32EB00EF80181918F016B
:103110001F928F93DF92CF920E9416940F900F9080
:103120000F900F90B012F1CF88851F928F938BEC88
:1031300093E09F938F930E9416940F900F900F909F
:103140000F90EE20D9F18E010F5F1F4F80E1F80143
:1031500011928A95E9F720E1A80160E880EB0E94CE
:103160000718FF2041F08BE793E09F938F930E9415
:1031700016940F900F9086E7E82E83E0F82E9FE0DC
:10318000D92ED00EF80181918F011F928F93FF925B
:10319000EF920E9416940F900F900F900F90D01204
:1031A000F1CF88891F928F938BEC93E09F938F933D
:1031B0000E9416940F900F900F900F9060960FB68C
:1031C000F894DEBF0FBECDBFDF91CF911F910F915D
:1031D000FF90EF90DF90CF90BF9008950F931F93D3
:1031E000CF93DF931F921F92CDB7DEB71A82198259
:1031F00022E0AE014F5F5F4F6AEA8EEE0E94071831
:1032000009E81DE1898190E0982F88272A81822B87
:10321000F8019183808322E0AE014F5F5F4F6CEA3B
:103220008EEE0E940718898190E0982F88272A81C6
:10323000822BF8019383828322E0AE014F5F5F4FC0
:103240006EEA8EEE0E940718898190E0982F8827F9
:103250002A81822BF8019583848322E0AE014F5F9F
:103260005F4F60EB8EEE0E940718898190E0982FE7
:1032700088272A81822BF801938B828B22E0AE0172
:103280004F5F5F4F62EB8EEE0E940718898190E0DE
:10329000982F88272A81822BF801958B848B22E036
:1032A000AE014F5F5F4F64EB8EEE0E94071889817D
:1032B00090E0982F88272A81822BF801978B868BA4
:1032C00022E0AE014F5F5F4F66EB8EEE0E94071863
:1032D000898190E0982F88272A81822BF801978393
:1032E000868322E0AE014F5F5F4F68EB8EEE0E9457
:1032F0000718898190E0982F88272A81822BF8016E
:103300009187808722E0AE014F5F5F4F6AEB8EEEC0
:103310000E940718898190E0982F88272A81822BA4
:10332000F8019587848722E0AE014F5F5F4F6CEB19
:103330008EEE0E940718898190E0982F88272A81B5
:10334000822BF8019787868722E0AE014F5F5F4F9F
:103350006EEB8EEE0E940718898190E0982F8827E7
:103360002A81822BF801918B808B0F900F90DF9137
:10337000CF911F910F9108952F923F924F925F929C
:103380006F927F928F929F92AF92BF92CF92DF9275
:10339000EF92FF920F931F93CF93DF93CDB7DEB7DA
:1033A0006C970FB6F894DEBF0FBECDBF182F042F59
:1033B0002D8B19821A821B828091AD1D811107C04D
:1033C0006C8F0E94EE1881E08093AD1D6C8D66239A
:1033D00009F472C04EE264EF8EEE0E94EF1762E1D4
:1033E00074E380E090E00E94946022E0AE014F5FC1
:1033F0005F4F66EF8EEE0E9407182981822F90E0C2
:10340000A0E0B0E04427582F692F7A2F8A81482BFB
:1034100080919F1D9091A01D9A01AB01281B390B33
:1034200041095109A0919D1DB0919E1D0E944089A6
:103430006B017C013FE0F594E794D794C7943A95EB
:10344000D1F76091971D7091981DCB01770FAA0B52
:10345000BB0BBC01CD014BE0660F771F881F991F86
:103460004A95D1F72091991D30919A1D4901330F4A
:10347000AA08BB08A7019601280D391D4A1D5B1D2E
:103480000E94FB88C20ED31ED092941DC092931D41
:1034900028E0C20ED11C54E0D594C7945A95E1F7A8
:1034A0000D2C000CEE08FF08C092A11DD092A21DA9
:1034B000E092A31DF092A41D812F8295880F880FA2
:1034C000807C8C5C8887212E312CA3E0B0E0012E1B
:1034D00002C0AA0FBB1F0A94E2F72AE63AE00E9454
:1034E00039899B01AC012E5F3F4F4F4F5F4F2987BA
:1034F0003A874B875C8780E593ECA0E0B0E09C01C5
:10350000AD0104C055954795379527951A95D2F783
:10351000298B3A8B4B8B5C8B10E0412C512C320168
:1035200088E090E0AC01421953095B8F4A8F101775
:1035300009F43EC1488564EF8EEE0E94EF1769855D
:103540007A858B859C850E94946023E0AE014F5F55
:103550005F4F66EF8EEE0E940718E091931DF09189
:10356000941DE05AFF409F01DF010E9422896C8375
:103570007D838E839F8380918B1D90918C1D9E8770
:103580008D872091891D30918A1D388B2F8720913E
:103590008D1D30918E1D0E9422896B017C01ADE052
:1035A000F594E794D794C794AA95D1F7A0918F1D6D
:1035B000B091901D2C813D814E815F818CE05595AD
:1035C0004795379527958A95D1F70E944B89BB2758
:1035D00097FDB095AB2F8C0D9D1DAE1DBF1D0296A6
:1035E000A11DB11D32E0B595A795979587953A95A0
:1035F000D1F79C01AD0130584F4F5F4FA0919B1DFB
:10360000B0919C1D0E9440894B015C014FE0B69433
:10361000A794979487944A95D1F739818A8190E04D
:10362000A0E0B0E0BA2FA92F982F8827A32B2B81D9
:10363000822B9C01AD010A8C04C0559547953795A6
:1036400027950A94D2F72E8B3F8B488F598F4F8541
:1036500058896A01550FEE08FF0862E0CC0CDD1CAA
:10366000EE1CFF1C6A95D1F7A091911DB091921D9F
:103670002C813D814E815F810E944B899B01AC0171
:1036800077E155954795379527957A95D1F72C830E
:103690003D834E835F832D853E85DF010E94228915
:1036A000DC01CB01EBE0B595A79597958795EA9559
:1036B000D1F72C813D814E815F81820F931FA41F22
:1036C000B51FC80ED91EEA1EFB1E022C04C0CC0C6E
:1036D000DD1CEE1CFF1C0A94D2F732E0C30ED11C95
:1036E000E11CF11CF2E0F594E794D794C794FA95A5
:1036F000D1F72E893F89488D598D2C193D094E09E6
:103700005F0969897A898B899C890E94958897FDD0
:103710000BC0660F771F881F991FA50194010E9497
:10372000D98869017A010AC0A50194010E94D9884B
:1037300069017A01CC0CDD1CEE1CFF1C9927F7FCFB
:103740009A958F2D7E2D6D2D9B01AC010E94958841
:103750009B01AC01AEEDBBE00E9440894C01BB2453
:1037600097FCB094AB2CA3E4B3EEA70196010E94A2
:103770004E89BB2797FDB095AB2F880E991EAA1EC8
:10378000BB1E4FEC840E4EE0941EA11CB11C44E005
:10379000B594A794979487944A95D1F7C80CD91CEF
:1037A000EA1CFB1C4C0C5D1C6E1C7F1C1F5FBFCEFB
:1037B000112381F0212F30E040E050E0C301B2013D
:1037C0000E94D9882093A51D3093A61D4093A71D64
:1037D0005093A81D5D89552389F16091A51D7091B5
:1037E000A61D8091A71D9091A81D611571058105E9
:1037F000910521F10E94B08C20E836EE45EC57E4AB
:103800000E94FC8B21E03EED42E45EE30E94158FB6
:103810009B01AC0160E070E080E89FE30E94188BA0
:103820002BE43AE34DEB57E30E94FC8B6093A91D18
:103830007093AA1D8093AB1D9093AC1D6C960FB630
:10384000F894DEBF0FBECDBFDF91CF911F910F91D6
:10385000FF90EF90DF90CF90BF90AF909F908F90B0
:103860007F906F905F904F903F902F9008950F93AF
:103870001F93CF93DF9300D000D0CDB7DEB78E017A
:103880000F5F1F4F86E0F80111928A95E9F780914A
:103890009F1C811113C040E061E386EA0E94EF178C
:1038A0004AE06CE286EA0E94EF1781E080939F1C59
:1038B00068EF7CE780E090E00E94946048E06DE271
:1038C00086EA0E94EF1768EF7CE780E090E00E94B4
:1038D000946026E0A80162E386EA0E94071847E0A8
:1038E0006DE286EA0E94EF178A8190E0982F882780
:1038F0002981822B90939A1C8093991C2C8130E013
:10390000322F22274B81242B30939C1C20939B1C0D
:103910004E8150E0542F44276D81462B50939E1CBE
:1039200040939D1C5F934F933F932F939F938F934F
:103930008FE793E09F938F930E9416940FB6F894AD
:10394000DEBF0FBECDBF26960FB6F894DEBF0FBE0A
:10395000CDBFDF91CF911F910F910895CF92DF924C
:10396000EF92FF920F931F93CF93DF93CDB7DEB704
:103970002A970FB6F894DEBF0FBECDBF8E010F5F42
:103980001F4F86E0F80111928A95E9F741E062E065
:103990008CE30E94EF1748E560E08CE30E94EF178C
:1039A00064E278E680E090E00E94946026E0A8015E
:1039B00063E08CE30E94071843E062E08CE30E941E
:1039C000EF17098110E0102F00278A81082BE9E703
:1039D000FCE111830083EB80F12CFE2CEE248C8122
:1039E000E82AF382E282CD80D12CDC2CCC248E819B
:1039F000C82AD582C482B801012E000C880B990B0D
:103A00000E94B08C9B01AC01B7010F2C000C880BFD
:103A1000990B2F83388749875A870E94B08C2F8152
:103A2000388549855A850E94988B20EE3EE245E60E
:103A300052E40E94A88E20E030E044E353E40E9468
:103A4000198B9F938F937F936F93DF92CF92FF9207
:103A5000EF921F930F938DE893E09F938F930E94B3
:103A600016940FB6F894DEBF0FBECDBF2A960FB6E0
:103A7000F894DEBF0FBECDBFDF91CF911F910F91A4
:103A8000FF90EF90DF90CF900895CF93DF93EC01FC
:103A900088819981009759F18F32924121F01982E2
:103AA000188283E071C082E69AE00E944F6F892BF2
:103AB00051F180919F139091A013A091A113B09107
:103AC000A21393FD22C080919F139091A013A09107
:103AD000A113B091A21394FD49C080919F139091BE
:103AE000A013A091A113B091A21395FD46C040E888
:103AF00050E060E070E082E69AE00E94316F8FE271
:103B000092E19983888381E03FC08091C52C82FF38
:103B1000DACF21E048E061E083E00E94BC198091A7
:103B2000AC1D8F938091AB1D8F938091AA1D8F93B5
:103B30008091A91D8F938091A81D8F938091A71DBF
:103B40008F938091A61D8F938091A51D8F9380EFF9
:103B500091E19F938F930E942A948DB79EB70A9606
:103B60000FB6F8949EBF0FBE8DBFADCF8091C52C10
:103B700083FFB3CF0E94371CB0CF8091C52C84FF48
:103B8000B6CF0E94AE1CB3CFDF91CF910895CF93F3
:103B9000DF93C82F8CEE0E9412618C2F0E941C6153
:103BA0006AE67AE080E090E00E9494608DEE0E94E8
:103BB00012610E942D61D82F0E943761C82F0E9488
:103BC00014618C2F90E09D2BDF91CF9108951F936E
:103BD000CF93DF93C82F8CEE0E9412618C2F0E942E
:103BE0001C6164E278E680E090E00E9494608CEED4
:103BF0000E94126180E00E941C616AE67AE080E027
:103C000090E00E9494608DEE0E9412610E942D61EE
:103C1000D82F0E942D61182F0E943761C82F0E9453
:103C20001461812F90E0A0E0B0E0BA2FA92F982F67
:103C30008827AD2BBC01CD016C2BDF91CF911F915B
:103C400008952F923F924F925F926F927F928F9240
:103C50009F92AF92BF92CF92DF92EF92FF920F931B
:103C60001F93CF93DF93CDB7DEB7CB54D1090FB6F7
:103C7000F894DEBF0FBECDBF809104029091050283
:103C8000892BE1F110920502109204028CEE0E9441
:103C900012618EE10E941C610E94146166E37CE95E
:103CA00080E090E00E94946082EA0E94C71D909399
:103CB000530A8093520A84EA0E94C71D9093510AC6
:103CC0008093500A86EA0E94C71D90934F0A809302
:103CD0004E0A88EA0E94C71D90934D0A80934C0AB1
:103CE0008AEA0E94C71D90934B0A80934A0A8CEA85
:103CF0000E94C71D9093490A8093480A88E40E9455
:103D0000E71D6DAB7EAB8FAB98AF88E50E94E71DDA
:103D10004B015C0180914A0A90914B0A8C0120E092
:103D200030E040E050E0BA0122968FAF2297239610
:103D30001FAF239724962FAF249725963FAF259743
:103D400026964FAF269727965FAF279728966FAF97
:103D5000289729967FAF29979C0140E050E060E0CA
:103D600070E080E090E008E00E94AE8A0E94678ADE
:103D70003901B42FA52FF62FE72F8C019401A5014F
:103D800060E070E080E090E05301CB2EDA2EEF2E61
:103D9000FE2E0E94E58A2CA33BA349835A831B0174
:103DA0002C01C201315041095F4F6F4F7F4F8F4F40
:103DB0009F4F88248394912C21153F4F4F4F5140A2
:103DC000610571058105910509F010F4812C912C94
:103DD00034010091480A1091490A5801C12CD12C94
:103DE000E12CF12C00E010E02CA13BA149815A818B
:103DF000B101C2010E945389F22E032F142FB52F57
:103E0000F62FE72FD82EE92EA0E00E940C8B84F429
:103E10002150310940485F4F6F4F7F4F8F4F9F4F69
:103E2000F22E032F142FB52FF62FE72FD82EE92EC1
:103E30002F2D302F412F5B2F6F2F7E2F8D2D9E2DFD
:103E400007E10E94C78A2B8F3C8F4D8F5E8F6F8F4B
:103E500078A389A39AA32053384F4F4F5F4F6F4FDA
:103E60007F4F8F4F9F4F2B8B3C8B4D8B5E8B6F8B80
:103E7000788F898F9A8F2056304F4F4F5F4F6F4FFB
:103E80007F4F8F4F9F4F243D3043410551056105C2
:103E900071058105910529F020F03401BFEF6B1AFF
:103EA0007B0A8090500A9090510A940140E050E0C3
:103EB00060E070E080E090E000E10E94AE8A2B8339
:103EC0003C834D835E836F8378874C0140914C0A1D
:103ED00050914D0AACA0BBA0C980DA80710182016B
:103EE0009A0140E050E060E070E080E090E00E94E5
:103EF0005389F22E032F142FB52FF62FE72FD82E2C
:103F0000E92EA0E00E940C8B5CF4AFE70E94EE8AE1
:103F1000F22E032F142FB52FF62FE72FD82EE92ED0
:103F20002F2D302F412F5B2F6F2F7E2F8D2D9E2D0C
:103F300007E00E94C78A59016A017B018C012B812D
:103F40003C814D815E816F817885C4010E94E58A44
:103F50002B833C834D835E836F8378878F87988B19
:103F60002E5F3F4F434051096E4F7F4F8F4F9F4F02
:103F700022303105494F5F4F64407105810591053D
:103F800021F018F0FFEF6F1A7F0A6091520A7091CA
:103F9000530A80E090E020E030E840E050E00E94EA
:103FA000AC8929873A874B875C876D877E874C0170
:103FB00040914E0A50914F0AACA0BBA0C980DA8054
:103FC000710182019A0140E050E060E070E080E021
:103FD00090E00E945389F22E032F142FB52FF62F55
:103FE000E72FD82EE92EA0E00E940C8B84F42150FC
:103FF0003F4F4F4F5F4F6F4F7F4F8F4F9F4FF22E6F
:10400000032F142FB52FF62FE72FD82EE92E2F2DA3
:10401000302F412F5B2F6F2F7E2F8D2D9E2D08E08F
:104020000E94C78A59016A017B018C0129853A8562
:104030004B855C856D857E85C4010E94E58A298754
:104040003A874B875C876D877E87898B9A8B2F5F3A
:104050003F4F41405109610971098109910921309E
:1040600030484C4F5F47614071058105910521F053
:1040700018F01FEF611A710A2B893C894D895E89FE
:104080006F89788D898D9A8D2F3C37404105510578
:10409000610571058105910511F00CF09CC1ACA082
:1040A000BBA0C980DA80710182019501A601B1012E
:1040B000C2010E945389A12CB12CC12CE0E8DE2E54
:1040C000E12CF12C00E010E00E94D98929AF3AAF31
:1040D0004BAF5CAF6DAF7EAF8FAF21969FAF219797
:1040E000AB8CBC8CCD8CDE8CEF8CF8A009A11AA116
:1040F0009501A601B701C8010E94538959016A01BF
:104100007B01E82F192F02E00E94AE8A0E2F0E9439
:10411000E58A7901142F452EF62FE72F6C01922E98
:10412000AF2CB42E052F362EB72F582E8D2CA0E095
:104130000E940C8B5CF4A1E00E94EE8A922EA32ECA
:10414000B42E052F362EB72F582E892E292D3A2D15
:104150004B2D502F632D7B2F852D982D01E00E9434
:10416000C78A29A73AA74A012C966FAF2C972B969E
:104170007FAF2B978BA79CA729833A834BA39CA245
:104180006DA37EA38FA398A7B42D9701412F542D23
:104190006F2F7E2FC601A0E00E940C8B4CF4A3E091
:1041A0000E94EE8A7901142FB52FF62FE72F6C01AC
:1041B0009701412F5B2F6F2F7E2FC60102E00E94D7
:1041C000C78A2DA73EA74FA758AB69AB7AAB8BAB7D
:1041D0009CAB2901B42FA52F22966FAF2297F72F02
:1041E0001C012B893C894D895E896F89788D898D69
:1041F0009A8D24323A4F4F4F5F4F6F4F7F4F8F4F03
:104200009F4F0CF08BC02B8D3C8D4D8D5E8D6F8D37
:1042100078A189A19AA12455324F4F4F5F4F6F4F1C
:104220007F4F8F4F9F4F59016A017B018C010E9484
:10423000538919012A01B62FA72FFC0103E00E9420
:10424000AE8A51016201EB2EFA2E8F010E94FA8A8A
:1042500059016A017B018C0129A53AA5A4012C967C
:104260006FAD2C972B967FAD2B978BA59CA50E94AD
:10427000E58A29833A834BA35CA36DA37EA38FA316
:1042800098A79101A2016B2F7A2FCF0102E00E9423
:10429000AE8A51016201EB2EFA2E8F010E94FA8A3A
:1042A00002E00E94AE8A0E2F0E94FA8A122FD32EAD
:1042B000E42EB52FF62FE72FF82E092FA0E00E944D
:1042C0000C8B5CF4A1E00E94EE8A122FD32EE42E18
:1042D000B52FF62FE72FF82E092F212F3D2D4E2D2C
:1042E0005B2F6F2F7E2F8F2D902F01E00E94C78AAA
:1042F00059016A017B018C012DA53EA54FA558A946
:1043000069A97AA98BA99CA90E94E58A2901B42FE1
:10431000A52F22966FAF2297F72F1C012B813C818E
:104320004D815E816F8178858F859889A980BA805B
:10433000CBA0DCA0EDA0FEA00FA118A50E94FA8AD8
:104340002B833C834D835E836F8378878F87988B25
:1043500029853A854B855C856D857E8589899A8915
:104360005201CB2EDA2E2296EFAC2297FF2E81013E
:104370000E94FA8A29873A874B875C876D877E87F8
:10438000898B9A8B2B893C894D895E896F89788DC1
:10439000898D9A8DA9ACBAACCBACDCACEDACFEACE3
:1043A0000FAD21961FAD21970E94FA8A2056304FFB
:1043B0004F4F5F4F6F4F7F4F8F4F9F4F243D304385
:1043C00041055105610571058105910521F018F040
:1043D0000FEF601A700A4DA95EA96FA978AD9A0116
:1043E000AB0160E070E0CB0122962FAF22972396BD
:1043F0003FAF239724964FAF249725965FAF25971D
:1044000026966FAF269727967FAF279728968FAF70
:10441000289729969FAF2997A984BA84CB84DC84F6
:10442000ED84FE8409891A8960E070E080E090E004
:104430000E945389122FD32EE42EB52FF62FE72F8B
:10444000F82E092FA0E00E940C8B84F42150310932
:10445000404E5F4F6F4F7F4F8F4F9F4F122FD32E86
:10446000E42EB52FF62FE72FF82E092F212F3D2D03
:104470004E2D5B2F6F2F7E2F8F2D902F05E10E94E9
:10448000C78AAB80BC80CD80DE80EF80F8840F854A
:1044900018890E94FA8A122FD32EE42EB52FF62FF8
:1044A000E72FF82E092FA0E00E940C8B84F42150F6
:1044B00030484F4F5F4F6F4F7F4F8F4F9F4F122F9F
:1044C000D32EE42EB52FF62FE72FF82E092F212F0C
:1044D0003D2D4E2D5B2F6F2F7E2F8F2D902F0FE0B8
:1044E0000E94C78A59016A017B018C01322E5B2C24
:1044F000B42FAD2DF62F4F2C4C01285E33404109CF
:1045000051096109710981099109283D304D4140E6
:104510005105610571058105910509F010F46728C1
:1045200069F09501A601B701C8010E94678A322E81
:10453000532EB42FA52FF62F472E4C01232D352DAA
:104540004B2F5A2F6F2F742DC4010E94A88C20E08E
:1045500030E048EC52E40E94FC8BC55BDF4F0FB6A5
:10456000F894DEBF0FBECDBFDF91CF911F910F91A9
:10457000FF90EF90DF90CF90BF90AF909F908F9083
:104580007F906F905F904F903F902F9008954F9243
:104590005F926F927F928F929F92AF92BF92CF92D3
:1045A000DF92EF92FF922B013C0169017A0123EC2B
:1045B00035EF4CE851E4C701B6010E94A88E4B01CB
:1045C0005C0128EB3EE143E753E4C701B6010E94DA
:1045D000198B9B01AC01C501B4010E94FC8B0E94A8
:1045E000768C4B015C0120E030E048EC52E4C301E2
:1045F000B2010E94FC8B21E835E943EC50E40E94B3
:10460000A88EA50194010E94A88E4B015C0123E3B2
:1046100033E948E853E4C701B6010E94198B9B01B6
:10462000AC01C501B4010E94FC8B23E333EB48E5E8
:1046300053E40E94A88EFF90EF90DF90CF90BF9040
:10464000AF909F908F907F906F905F904F90089564
:104650004F925F926F927F928F929F92AF92BF9292
:10466000CF92DF92EF92FF9269017A010E941C8E35
:1046700020E030E040E050E40E94188B22E93CE565
:104680004EED5EE30E94FC8B4B015C0123EC35EFA9
:104690004CE851E4C701B6010E94A88E2B013C01F1
:1046A00028EB3EE143E753E4C701B6010E94198BB2
:1046B0009B01AC01C301B2010E94FC8B9B01AC01C8
:1046C000C501B4010E94198B6B017C0128EB3EE10E
:1046D00043E753E40E94A88E4B015C01A7019601B9
:1046E00063EC75EF8CE891E40E94188B9B01AC01A0
:1046F000C501B4010E94FC8BFF90EF90DF90CF903A
:10470000BF90AF909F908F907F906F905F904F90F1
:1047100008954F925F926F927F928F929F92AF9285
:10472000BF92CF92DF92EF92FF922B013C01690181
:104730007A0123EC35EF4CE851E4C701B6010E9441
:10474000A88E4B015C0128EB3EE143E753E4C7012F
:10475000B6010E94198B9B01AC01C501B4010E94F6
:10476000FC8B0E94768C4B015C0120E030E048EC31
:1047700052E4C301B2010E94FC8BA50194010E9486
:10478000A88E20E030E040E251E40E94188B24EE35
:1047900038E34EE05FE30E94A88E9B01AC01C701A5
:1047A000B6010E94198BFF90EF90DF90CF90BF90E1
:1047B000AF909F908F907F906F905F904F900895F3
:1047C00080E80E94126181110DC08EEF0E941C6171
:1047D000811108C066E37CE980E090E00E9494606B
:1047E0000C9414610E9414618091D7309091D8305C
:1047F000A091D930B091DA300196A11DB11D8093FE
:10480000D7309093D830A093D930B093DA30089550
:10481000FC01DC01AC014E5F5F4F90E031E38D9114
:10482000982788E0292F220F97FF03C0922F932704
:1048300001C0922F8150B1F7A417B50781F721E08D
:1048400030E08281981711F020E030E0C90108952E
:10485000DF92EF92FF920F931F93CF93DF930E940B
:10486000E02380E80E94126181116DC08AEF0E94EE
:104870001C61811168C08FE00E941C61811163C0BE
:104880006AE67AE080E090E00E94946081E80E940D
:104890001261811158C00E942D61D82F0E942D6194
:1048A0000E942D61182F0E942D610E942D61082FFA
:1048B0000E942D610E943761F82E80E80E941261EB
:1048C000811141C08CEF0E941C6181113CC089ECB8
:1048D0000E941C61811137C06AE67AE080E090E0B6
:1048E0000E94946081E80E9412610E942D61E82E6E
:1048F0000E942D61D82E0E942D610E942D61C82F2B
:104900000E9437611F92DF921F92EF921F92FF92D7
:104910001F920F931F921F931F92DF931F928F93EB
:104920001F92CF9382EA93E09F938F930E941694F5
:104930000E9414618DB79EB742960FB6F8949EBF41
:104940000FBE8DBF17C00E9414618091D730909127
:10495000D830A091D930B091DA300196A11DB11DA7
:104960008093D7309093D830A093D930B093DA3079
:104970000E94E02320E030E040E050E060E070E0A2
:1049800080E090E0DF91CF911F910F91FF90EF9029
:10499000DF900895EF92FF920F931F93CF93DF93D1
:1049A00000D0CDB7DEB78C0180E80E941261811182
:1049B00054C00115110551F085EE0E941C61811152
:1049C0004CC062E07EE281E090E009C083EE0E948C
:1049D0001C61811142C062E375E783E090E00E94B0
:1049E000946081E80E941261811137C00E942D619C
:1049F000E82E89830E942D61F82E8A830E943761F8
:104A00008B830E941461CE0101960E940824892B99
:104A100021F16F2D70E07E296C7F80E090E0012B0A
:104A200069F00E94AE8C20E030E04AEF5AE30E9429
:104A3000A88E20E030E040EC50E40CC00E94AE8C28
:104A400022E538EB4FE25BE30E94A88E26E636E6CD
:104A50004BE352E40E94188B1BC00E9414618091AA
:104A6000D7309091D830A091D930B091DA300196FA
:104A7000A11DB11D8093D7309093D830A093D93029
:104A8000B093DA300E94E02360EF7FEF89E794E48F
:104A90000F900F900F90DF91CF911F910F91FF908A
:104AA000EF9008950F931F93CF93DF93729A8091A5
:104AB000660283FF08C08EE40E94B760811165C062
:104AC000C0E5D0E009C0C0E5D0E08FED97E00E94DE
:104AD000590E2197D1F7EFCF8FED97E00E94590E35
:104AE0002197D1F78FE40E94B7600E942D61D82FE3
:104AF000DF730E942D61082F0E942D61C82F0E9434
:104B00003761182F0E9414618091660283FF7298AA
:104B10006D2F70E0762F6627600F711D80E090E0AA
:104B20000E94AE8C20E134E048EC5BE30E94A88E4A
:104B30006093B9287093BA288093BB289093BC28BF
:104B40006C2F70E0762F6627610F711D7695679543
:104B50007695679580E090E00E94AE8C24EA3CEF69
:104B600044E25CE30E94A88E20E030E040E252E4A0
:104B70000E94188B60939A3570939B3580939C3577
:104B800090939D3580E090E002C081E090E0DF915D
:104B9000CF911F910F9108957298729A8EE40E949E
:104BA000B76080EA0E941C6180E00E941C6180E086
:104BB0000E941C618FE40E94B7600E942D618EE408
:104BC0000E94B76080E80E941C6180E00E941C6126
:104BD00080E00E941C610E94146180E090E00895D2
:104BE0008FE191E19F938F930E942A94809180029C
:104BF0000F900F90882361F01F928F938CE191E1C9
:104C00009F938F930E942A940F900F900F900F9074
:104C1000089587EF90E19F938F930E942A948FECE1
:104C200090E19F938F930E942A9488EA90E19F934A
:104C30008F930E942A948DE690E19F938F930E9418
:104C40002A9481E390E19F938F930E942A948FEF9F
:104C50009FE09F938F930E942A9483EC9FE09F9301
:104C60008F930E942A948DE99FE09F938F930E94D7
:104C70002A9487E69FE09F938F930E942A948091C5
:104C8000C52C9091C62C827091702DB73EB72E5EC8
:104C90003F4F0FB6F8943EBF0FBE2DBF892B41F09A
:104CA00087E39FE09F938F930E942A940F900F9029
:104CB0008BE09FE09F938F930E942A948FEC9EE05D
:104CC0009F938F930E942A9486EA9EE09F938F93EE
:104CD0000E942A948AE79EE09F938F930E942A94D1
:104CE0008BE49EE09F938F930E942A9489E19EE03B
:104CF0009F938F930E942A9488EE9DE09F938F93B9
:104D00000E942A948EEA9DE09F938F930E942A949A
:104D100088E79DE09F938F930E942A9488E49DE00A
:104D20009F938F930E942A948CE19DE09F938F9391
:104D30000E942A948DEE9CE09F938F930E942A9468
:104D400084EB9CE09F938F930E942A948BE79CE0D6
:104D50009F938F930E942A9484E49CE09F938F9367
:104D60000E942A9486E19CE09F938F930E942A944C
:104D70008DB79EB780960FB6F8949EBF0FBE8DBFBD
:104D800082EE9BE09F938F930E942A9481EB9BE09D
:104D90009F938F930E942A9482E89BE09F938F9326
:104DA0000E942A9483E59BE09F938F930E942A940C
:104DB0008CE29BE09F938F930E942A9486EF9AE067
:104DC0009F938F930E942A9480EC9AE09F938F93F5
:104DD0000E942A948AE89AE09F938F930E942A94D3
:104DE00081E69AE09F938F930E942A9489E29AE049
:104DF0009F938F930E942A948EEF99E09F938F93B5
:104E00000E942A942DB73EB72A5E3F4F0FB6F89402
:104E10003EBF0FBE2DBF089581ED93E00C945294D8
:104E20004F925F926F927F928F929F92AF92BF92BA
:104E3000CF92DF92EF92FF92CF93DF93CDB7DEB7A1
:104E400028970FB6F894DEBF0FBECDBF8091CB3050
:104E50009091CC30A091CD30B091CE3089839A839F
:104E6000AB83BC834090CB305090CC306090CD3041
:104E70007090CE308091CB309091CC30A091CD30DD
:104E8000B091CE308D839E83AF83B8876091CB3055
:104E90007091CC308091CD309091CE302CE3822E29
:104EA000912CA12CB12CA50194010E94D9887F934B
:104EB0006F9330E1C32E3EE0D32EE12CF12C6D81B7
:104EC0007E818F819885A70196010E94D988A501CE
:104ED00094010E94D9883F932F9340E8842E41E5A6
:104EE000942EAA24A394B12CC301B201A50194016C
:104EF0000E94D988A70196010E94D9883F932F93D9
:104F000069817A818B819C81A50194010E94D98855
:104F10003F932F9388ED99E09F938F930E942A945B
:104F20000FB6F894DEBF0FBECDBF28960FB6F8942B
:104F3000DEBF0FBECDBFDF91CF91FF90EF90DF902E
:104F4000CF90BF90AF909F908F907F906F905F9029
:104F50004F900895EDEFF9E380819181823492447E
:104F600079F0ED5FF943FF93EF938AEB99E09F931C
:104F70008F930E942A940F900F900F900F90089596
:104F80003A96E53F81E8F80738F30895CF93DF9329
:104F9000EC018C9A0E94CB109F938F937F936F9319
:104FA0008EEA99E09F938F930E942A940F900F901E
:104FB0000F900F900F900F90209719F00E94DC1126
:104FC00008C08CEA99E09F938F930E942A940F90D7
:104FD0000F9081E00E947D10209185023091860221
:104FE00040918702509188020E94A88E9F938F93D0
:104FF0007F936F9380EA99E09F938F930E942A9406
:105000000F900F900F900F900F900F90209719F026
:105010000E94DC1108C08EE999E09F938F930E9453
:105020002A940F900F9082E00E947D1020918102BF
:105030003091820240918302509184020E94A88E96
:105040009F938F937F936F9382E999E09F938F93C0
:105050000E942A940F900F900F900F900F900F9036
:10506000209719F00E94DC1108C080E999E09F9315
:105070008F930E942A940F900F9083E00E947D10DE
:105080009F938F937F936F9381E899E09F938F9382
:105090000E942A948C980F900F900F900F900F9071
:1050A0000F90209719F00E94DC1108C08FE799E05B
:1050B0009F938F930E942A940F900F908091C52CFC
:1050C00087FF83C021E042E161E080ED0E947E62C3
:1050D0009F938F937F936F9382E799E09F938F9332
:1050E0000E942A940F900F900F900F900F900F90A6
:1050F000209719F00E94DC1108C080E799E09F9387
:105100008F930E942A940F900F9021E042E162E079
:1051100080ED0E947E629F938F937F936F9383E6CF
:1051200099E09F938F930E942A940F900F900F9075
:105130000F900F900F90209719F00E94DC1108C07B
:1051400081E699E09F938F930E942A940F900F908D
:1051500021E042E163E080ED0E947E629F938F93A5
:105160007F936F9384E599E09F938F930E942A9495
:105170000F900F900F900F900F900F90CD2B19F074
:105180000E94DC1108C082E599E09F938F930E94F2
:105190002A940F900F9021E042E164E080ED0E949C
:1051A0007E629F938F937F936F9385E499E09F93A3
:1051B0008F930E942A940F900F900F900F900F9052
:1051C0000F90DF91CF910C94DC11CD2BD1F3DF91B7
:1051D000CF9108950F931F93CF93DF93882389F086
:1051E00049E050E06FEF70E08EE895E30E94649331
:1051F00049E050E06EE070E08EE895E30E94F5969D
:1052000013C0CEE8D5E300E419E089911F928F9393
:105210001F930F930E942A940F900F900F900F905E
:1052200085E3C639D80789F7DF91CF911F910F9198
:105230000C94DC11882311F0299A08952998089577
:10524000882311F02A9A08952A980895CF92DF9220
:10525000EF92FF92CF93DF936B017C0160FF11C04F
:105260008EE094E09F938F9384E391E19F938F93DB
:105270000E942A940F900F900F900F9081E090E081
:1052800002C080E090E0C1FE09C0EC01219648E236
:1052900059E063E174E00E944516CE01C2FE09C0E8
:1052A000EC01219648E259E06BE174E00E9445165A
:1052B000CE01C3FE09C0EC01219648E259E063E249
:1052C00074E00E944516CE01C4FE09C0EC0121968F
:1052D00048E259E063E975E00E944516CE01C5FE3B
:1052E00009C0EC01219648E259E067E274E00E94AF
:1052F0004516CE01C6FE09C0EC01219648E259E0F0
:105300006BE274E00E944516CE01C7FE09C0EC01B5
:10531000219648E259E061E374E00E944516CE010F
:10532000D0FE09C0EC01219648E259E069E374E03F
:105330000E944516CE01D1FE09C0EC01219648E23B
:1053400059E061E474E00E944516CE01D2FE09C026
:10535000EC01219648E259E065E474E00E944516AC
:10536000CE012091C52C3091C62C24703270232B95
:1053700059F0D3FE09C0EC01219648E259E06BE4F4
:1053800074E00E944516CE012091C52C23FF0BC06E
:10539000D4FE09C0EC01219648E259E060E574E0D2
:1053A0000E944516CE012091C52C24FF0BC0D5FECE
:1053B00009C0EC01219648E259E066E574E00E94DC
:1053C0004516CE01D6FE09C0EC01219648E259E00F
:1053D0006EE574E00E944516CE01D7FE09C0EC01CF
:1053E000219648E259E069E674E00E944516CE0134
:1053F000E0FE0CC048E259E06AE774E0DF91CF912B
:10540000FF90EF90DF90CF900C944516CD28CE28DA
:10541000CF2841F48BE399E09F938F930E942A94C5
:105420000F900F90DF91CF91FF90EF90DF90CF9092
:105430000895CF92DF92EF92FF92CF93DF93EC012A
:10544000C12CD12C7601209709F4A3C066E379E042
:10545000CE010E943693892B11F46894C0F86EE255
:1054600079E0CE010E943693892B11F46894C1F83B
:1054700066E279E0CE010E943693892B11F468949C
:10548000C2F862E279E0CE010E943693892B11F4D2
:105490006894C3F86FE179E0CE010E943693892BBE
:1054A00011F46894C4F86BE179E0CE010E94369360
:1054B000892B11F46894C5F865E179E0CE010E946A
:1054C0003693892B11F46894C6F86DE079E0CE012B
:1054D0000E943693892B11F46894C7F865E079E04F
:1054E000CE010E943693892B11F46894D0F861E0C4
:1054F00079E0CE010E943693892B11F46894D1F89B
:105500006BEF78E0CE010E943693892B11F46894FA
:10551000D2F866EF78E0CE010E943693892B11F421
:105520006894D3F860EF78E0CE010E943693892B1F
:1055300011F46894D4F868EE78E0CE010E943693B6
:10554000892B11F46894D5F86DED78E0CE010E94B6
:105550003693892B11F46894D6F86CEC78E0CE0180
:105560000E943693892B11F46894D7F867EC78E0A1
:10557000CE010E943693892B11F46894E0F8609173
:105580007E0270917F0280E090E00E944A93EC01DD
:105590005ACFC701B601DF91CF91FF90EF90DF9016
:1055A000CF900895AF92BF92CF92DF92EF92FF9289
:1055B0000F931F93CF93DF93D22FC32F8A01F62E21
:1055C000C72ED82EE92E217030E040E050E060E098
:1055D00070E080E090E0A0E00E940C8B89F08FE703
:1055E00094E09F938F9384E391E19F938F930E9424
:1055F0002A940F900F900F900F90E1E0F0E002C01E
:10560000E0E0F0E08091C52C80FF19C02D2F2470C0
:1056100030E040E050E060E070E080E090E0A0E04A
:105620000E940C8B61F05F018FEFA81AB80A48E264
:1056300059E063E874E0CF010E944516F5012D2F73
:10564000227030E040E050E060E070E080E090E008
:10565000A0E00E940C8B61F05F018FEFA81AB80ADE
:1056600048E259E067E874E0CF010E944516F50171
:105670002D2F287030E040E050E060E070E080E0E6
:1056800090E0A0E00E940C8B61F05F018FEFA81A00
:10569000B80A48E259E06FE974E0CF010E9445166C
:1056A000F5012D2F207130E040E050E060E070E027
:1056B00080E090E0A0E00E940C8B61F05F018FEF32
:1056C000A81AB80A48E259E06AE874E0CF010E94DB
:1056D0004516F5012D2F207230E040E050E060E0EB
:1056E00070E080E090E0A0E00E940C8B61F05F0130
:1056F0008FEFA81AB80A48E259E06DE874E0CF01CC
:105700000E944516F5012D2F207430E040E050E056
:1057100060E070E080E090E0A0E00E940C8B61F01F
:105720005F018FEFA81AB80A48E259E063E974E014
:10573000CF010E944516F5012D2F207830E040E082
:1057400050E060E070E080E090E0A0E00E940C8B10
:1057500061F05F018FEFA81AB80A48E259E069E9E1
:1057600074E0CF010E944516F50120E03C2F317016
:1057700040E050E060E070E080E090E0A0E00E9457
:105780000C8B61F05F018FEFA81AB80A48E259E06C
:105790006CE974E0CF010E944516F50120E03C2F32
:1057A000327040E050E060E070E080E090E0A0E027
:1057B0000E940C8B61F05F018FEFA81AB80A48E2D3
:1057C00059E061EA74E0CF010E944516F50120E03E
:1057D0003C2F347040E050E060E070E080E090E00A
:1057E000A0E00E940C8B61F05F018FEFA81AB80A4D
:1057F00048E259E068EA74E0CF010E944516F501DD
:1058000020E03C2F387040E050E060E070E080E045
:1058100090E0A0E00E940C8B61F05F018FEFA81A6E
:10582000B80A48E259E06BEA74E0CF010E944516DD
:10583000F50120E03C2F307140E050E060E070E086
:1058400080E090E0A0E00E940C8B61F05F018FEFA0
:10585000A81AB80A48E259E060EB74E0CF010E9450
:105860004516F50120E03C2F307240E050E060E04A
:1058700070E080E090E0A0E00E940C8B61F05F019E
:105880008FEFA81AB80A48E259E067EB74E0CF013D
:105890000E944516F50120E030E040E050E06F2D19
:1058A000647070E080E090E0A0E00E940C8B61F0FA
:1058B0005F018FEFA81AB80A48E259E06EEB74E076
:1058C000CF010E944516F5018091C52C81FF19C0BA
:1058D00020E03C2F307440E050E060E070E080E079
:1058E00090E0A0E00E940C8B61F05F018FEFA81A9E
:1058F000B80A48E259E062EC74E0CF010E94451614
:10590000F5018091C52C9091C62C90FF19C020E024
:1059100030E040E0512F507160E070E080E090E0B6
:10592000A0E00E940C8B61F05F018FEFA81AB80A0B
:1059300048E259E065EC74E0CF010E944516F5019C
:105940008091C52C9091C62C90FF19C020E030E0CA
:1059500040E0512F507260E070E080E090E0A0E005
:105960000E940C8B61F05F018FEFA81AB80A48E221
:1059700059E068EC74E0CF010E944516F501809172
:10598000C52C9091C62C90FF19C020E030E040E07B
:10599000512F507460E070E080E090E0A0E00E9441
:1059A0000C8B61F05F018FEFA81AB80A48E259E04A
:1059B0006EEC74E0CF010E944516F50120E03C2F0B
:1059C000307840E050E060E070E080E090E0A0E0FF
:1059D0000E940C8B61F05F018FEFA81AB80A48E2B1
:1059E00059E069ED74E0CF010E944516F50120E011
:1059F00030E0402F417050E060E070E080E090E0E7
:105A0000A0E00E940C8B61F05F018FEFA81AB80A2A
:105A100048E259E06EED74E0CF010E944516F501B1
:105A200020E030E0402F427050E060E070E080E025
:105A300090E0A0E00E940C8B61F05F018FEFA81A4C
:105A4000B80A48E259E061EE74E0CF010E944516C1
:105A5000F50120E030E040E050E06F2D687070E02C
:105A600080E090E0A0E00E940C8B61F05F018FEF7E
:105A7000A81AB80A48E259E064EE74E0CF010E9427
:105A80004516F50120E030E040E050E06F2D6071F8
:105A900070E080E090E0A0E00E940C8B61F05F017C
:105AA0008FEFA81AB80A48E259E068EE74E0CF0117
:105AB0000E944516F5018091C52C87FF19C020E092
:105AC00030E0402F487050E060E070E080E090E00F
:105AD000A0E00E940C8B61F05F018FEFA81AB80A5A
:105AE00048E259E06CEE74E0CF010E944516F501E2
:105AF0008091C52C87FF19C020E030E0402F407115
:105B000050E060E070E080E090E0A0E00E940C8B4C
:105B100061F05F018FEFA81AB80A48E259E060EF20
:105B200074E0CF010E944516F5018091C52C87FFD6
:105B300019C020E030E0402F407250E060E070E09B
:105B400080E090E0A0E00E940C8B61F05F018FEF9D
:105B5000A81AB80A48E259E064EF74E0CF010E9445
:105B60004516F5018091C52C87FF19C020E030E073
:105B7000402F407450E060E070E080E090E0A0E0F2
:105B80000E940C8B61F05F018FEFA81AB80A48E2FF
:105B900059E068EF74E0CF010E944516F50180914D
:105BA000C52C82FF19C020E030E0402F407850E043
:105BB00060E070E080E090E0A0E00E940C8B61F07B
:105BC0005F018FEFA81AB80A48E259E066E276E072
:105BD000CF010E944516F5018091C52C82FF19C0A6
:105BE00020E030E040E0512F517060E070E080E054
:105BF00090E0A0E00E940C8B61F05F018FEFA81A8B
:105C0000B80A48E259E06CEF74E0CF010E944516F3
:105C1000F5018091C52C9091C62C90FF19C020E011
:105C200030E040E0512F527060E070E080E090E0A2
:105C3000A0E00E940C8B61F05F018FEFA81AB80AF8
:105C400048E259E06FEF74E0CF010E944516F5017C
:105C50008091C52C9091C62C90FF19C020E030E0B7
:105C600040E0512F547060E070E080E090E0A0E0F0
:105C70000E940C8B61F05F018FEFA81AB80A48E20E
:105C800059E067E075E0CF010E944516F50180916B
:105C9000C52C9091C62C91FF1EC020E030E040E062
:105CA000512F587060E070E080E090E0A0E00E942A
:105CB0000C8B89F048E259E060E175E0CF01DF919B
:105CC000CF911F910F91FF90EF90DF90CF90BF90F9
:105CD000AF900C9445162D2F3C2FA8016F2D7C2DD5
:105CE0008D2D9E2DA0E00E940C8B41F482EC98E05B
:105CF0009F938F930E942A940F900F90DF91CF91E2
:105D00001F910F91FF90EF90DF90CF90BF90AF90D9
:105D10000895AF92BF92DF92EF92FF920F931F937D
:105D2000CF93DF93EC015B01FB0110826DEB78E018
:105D30000E943693892B59F58091C52C3DE4F32EB2
:105D400000E882FF03C024E8E22E02C094E0E92EBE
:105D500010E0D12C81FD00EC26E04AE250E06BE23D
:105D600070E089E290E00E945C5E81E090E00E9439
:105D70007411882311F08DE5F82E8091C52C909137
:105D8000C62C90FD16E091FF07C0186005C0F12CED
:105D900000E0E12C10E0D12C6BEB78E0CE010E940A
:105DA0003693892B61F481E0F501808360917E0256
:105DB00070917F0280E090E00E944A93EC0169EBD1
:105DC00078E0CE010E943693892B61F48FEFF501C4
:105DD000808360917E0270917F0280E090E00E945B
:105DE0004A93EC01209709F438C165EB78E0CE01C5
:105DF0000E943693892B19F4FF2DF160FF2E61EB81
:105E000078E0CE010E943693892B19F48F2D84609F
:105E1000F82E6EEA78E0CE010E943693892B19F4B1
:105E2000EF2DE260FE2E6CEA78E0CE010E94369300
:105E3000892B19F4FF2DF860FF2E69EA78E0CE0176
:105E40000E943693892B19F48F2D8061F82E63EA16
:105E500078E0CE010E943693892B19F4EF2DE06291
:105E6000FE2E6DE978E0CE010E943693892B19F45D
:105E7000FF2DF064FF2E6AE978E0CE010E94369390
:105E8000892B19F48F2D8068F82E65E978E0CE0112
:105E90000E943693892B09F401606EE878E0CE0108
:105EA0000E943693892B09F402606BE878E0CE01FA
:105EB0000E943693892B09F4046066E878E0CE01ED
:105EC0000E943693892B09F408606FE778E0CE01D1
:105ED0000E943693892B09F4006168E778E0CE01CF
:105EE0000E943693892B09F4006264E778E0CE01C2
:105EF0000E943693892B19F4ED2DE460DE2E61E7C4
:105F000078E0CE010E943693892B09F400646CE698
:105F100078E0CE010E943693892B09F4006869E687
:105F200078E0CE010E943693892B19F4FE2DF160A2
:105F3000EF2E66E678E0CE010E943693892B19F4A5
:105F40008E2D8260E82E63E678E0CE010E943693C3
:105F5000892B19F4EE2DE460EE2E6FE578E0CE018A
:105F60000E943693892B19F4FE2DF860EF2E6BE515
:105F700078E0CE010E943693892B19F48E2D806132
:105F8000E82E67E578E0CE010E943693892B19F45C
:105F9000EE2DE062EE2E63E578E0CE010E943693AE
:105FA000892B19F4FE2DF064EF2E61E578E0CE0127
:105FB0000E943693892B19F48E2D8068E82E6EE4AA
:105FC00078E0CE010E943693892B09F4116066E4D3
:105FD00078E0CE010E943693892B09F412606DE3BC
:105FE00078E0CE010E943693892B09F4146064E3B3
:105FF00078E0CE010E943693892B09F4186061E3A2
:1060000078E0CE010E943693892B09F410616BE28F
:1060100078E0CE010E943693892B09F4106260E289
:1060200078E0CE010E943693892B09F410646CE16C
:1060300078E0CE010E943693892B19F4ED2DE860AB
:10604000DE2E68E178E0CE010E943693892B09F0BC
:10605000C0CEFD2DF061DF2EBCCE2F2D302F4E2D6A
:10606000512F6D2D70E080E090E0DF91CF911F9176
:106070000F91FF90EF90DF90BF90AF9008955F92E7
:106080006F927F928F929F92AF92BF92CF92DF9248
:10609000EF92FF920F931F93CF93DF93782EC8EA6E
:1060A000DCE100E010E082E1E82E88E0F82E872DA8
:1060B0008170582E872D8270682E9DEFC92E97E033
:1060C000D92E25E0A22E28E0B22E33E0832E38E030
:1060D000932E772051F01F930F93FF92EF920E941F
:1060E0002A940F900F900F900F905520A1F0898562
:1060F0008F9388858F93BF92AF920E942A940F90BE
:106100000F900F900F906620C1F09F928F920E9487
:106110002A940F900F90662081F0DF92CF920E9418
:106120002A94288139814A815B816C817D818E81AD
:106130009F810E94D22A0F900F900E94DC110F5F66
:106140001F4F2A960430110521F6DF91CF911F9140
:106150000F91FF90EF90DF90CF90BF90AF909F9006
:106160008F907F906F905F90089588EF97E09F9356
:106170008F930E942A948091B5289091B628A0917F
:10618000B728B091B8280F900F90813027EA920776
:106190002EE1A207B10519F48AEE97E01DC0823006
:1061A00026EA92072EE1A207B10519F48DED97E0DA
:1061B00013C0823027EA92072EE1A207B10519F435
:1061C0008FEC97E009C0823028EA92072EE1A207FF
:1061D000B10549F481EC97E09F938F930E942A9434
:1061E0000F900F900895BF93AF939F938F938BEB76
:1061F00097E09F938F930E942A940F900F900F9097
:106200000F900F900F9008958BEA97E09F938F93D4
:106210000E942A940E940C270E94B5300E94DC1133
:106220008FE89CE19F938F9383EA97E09F938F93EE
:106230000E942A94609160027091610280916202D2
:106240009091630228EE33E040E050E00E94D9884C
:106250005F934F933F932F9383E997E09F938F939F
:106260000E942A948AE897E09F938F930E942A9431
:106270000E946E168091C52C2DB73EB7225F3F4F0E
:106280000FB6F8943EBF0FBE2DBF80FF05C041E0A2
:1062900061E081E00E94511886E897E09F938F9318
:1062A0000E942A9480E00E94EA280E941027809190
:1062B00065021F928F938DE797E09F938F930E94C3
:1062C0002A9480919C131F928F9384E797E09F9369
:1062D0008F930E942A94809190028F9380918F02D5
:1062E0008F9380918E028F9380918D028F9386E69B
:1062F00097E09F938F930E942A941F9280E48F933C
:106300008EE497E09F938F930E942A948091A43704
:106310001F928F938091A3371F928F938BE397E007
:106320009F938F930E942A94809164021F928F936F
:1063300082E397E09F938F930E942A948091660254
:1063400090916702A0916802B09169022DB73EB7A3
:10635000225E3F4F0FB6F8943EBF0FBE2DBF96FD95
:1063600003C08CE195E002C089E195E09F938F9393
:1063700088E297E09F938F930E942A9483E00E9483
:106380003F300F900F900F900F901D9903C08CE13C
:1063900095E002C089E195E09F938F938CE197E0AF
:1063A0009F938F930E942A9482E197E09F938F930B
:1063B0000E942A94809166020F900F900F900F9088
:1063C0000F900F9081FF09C08CE097E09F938F930F
:1063D0000E942A940F900F9013C080FD03C08CE19F
:1063E00095E002C089E195E09F938F9388E097E064
:1063F0009F938F930E942A940F900F900F900F906D
:106400008091660290916702A0916802B091690242
:1064100097FD03C08CE195E002C089E195E09F9370
:106420008F938FEF96E09F938F930E942A9488EF2B
:1064300096E09F938F930E942A9460919F1370918E
:10644000A0138091A1139091A2130E9426290E946B
:10645000DC110F900F900F900F900F900F90779B83
:1064600003C08CE195E002C089E195E09F938F9392
:106470008FEE96E09F938F930E942A940E945F0E66
:106480000E9430119F938F937F936F9381EE96E0DC
:106490009F938F930E942A940E94DF109F938F9363
:1064A0007F936F9383ED96E09F938F930E942A943E
:1064B00081E090E00E94C6278091743590917535F7
:1064C000A0917635B0917735BF93AF939F938F931B
:1064D00085EC96E09F938F930E942A948091893552
:1064E0008F93809188358F93809187358F9380919A
:1064F00086358F9381EB96E09F938F930E942A9429
:106500008091783590917935A0917A35B0917B352D
:10651000BF93AF939F938F9383EA96E09F938F935C
:106520000E942A948DB79EB782960FB6F8949EBFAC
:106530000FBE8DBF80918D358F9380918C358F9359
:1065400080918B358F9380918A358F938FE896E079
:106550009F938F930E942A9461E070E080E090E026
:106560000E94E51161E070E081E090E00E94E51199
:106570000F900F900F900F900F900F90299903C0DC
:106580008CE195E002C089E195E09F938F9387E8C5
:1065900096E09F938F930E942A940F900F900F90F4
:1065A0000F902A9903C08CE195E002C089E195E043
:1065B0009F938F938FE796E09F938F930E942A94E7
:1065C0008091660290916702A0916802B091690281
:1065D0000F900F900F900F9094FD03C08CE195E009
:1065E00002C089E195E09F938F9387E796E09F93A0
:1065F0008F930E942A940F900F900F900F90089500
:10660000F89491E2E0E0F0E0909357008491E2E0AA
:10661000F0E0909357002491E4E0F0E0909357006D
:10662000E49190E0A0E0B0E0BC0155274427822F20
:1066300090E0A0E0B0E0BA2FA92F982F8827840F10
:10664000951FA61FB71F8E0F911DA11DB11D809311
:10665000B5289093B628A093B728B093B82878941B
:106660000895CF93DF93CDB7DEB761970FB6F89457
:10667000DEBF0FBECDBF48E250E062E270E088EAC4
:106680009CE10E94D7962091A81C3091A91C4091B2
:10669000AA1C5091AB1C6091AC1C7091AD1C8091F8
:1066A000AE1C9091AF1CAFEF0E940C8B09F05DC047
:1066B0008DE48093A81C80E88093A91C84E08093DB
:1066C000AA1C1092AB1C1092AC1C1092AD1C109224
:1066D000AE1C1092AF1C8CE390E09093B11C8093A1
:1066E000B01C1092B21C1092B31C1092B41C1092E9
:1066F000B51C1092B61C1092B71C1092B81C1092C8
:10670000B91C1092BB1C1092BA1C1092BC1C1092A7
:10671000BD1C1092BE1C1092BF1C1092C01C109287
:10672000C11C1092C21C1092C31C1092C51C109266
:10673000C41C1092C61C1092C71C1092C81C109248
:10674000C91C1092CA1C1092CB1C1092CC1C109227
:10675000CD1C1092CF1C1092CE1C48E250E062E299
:1067600070E088EA9CE10E94F59644E050E06EE11A
:1067700070E0CE010B960E94D7968B859C85AD85E7
:10678000BE858F3F2FEF9207A207B207A9F48AE0D8
:1067900090E4A0E0B0E08093660290936702A0933B
:1067A0006802B093690244E050E06EE170E086E672
:1067B00092E00E94F59608C080936602909367026B
:1067C000A0936802B093690280916602909167027B
:1067D000A0916802B0916902A2FF02C02A9A03C088
:1067E00080E00E94202944E050E06AE570E0CE019C
:1067F0000B960E94D7968B859C85AD85BE858F3F75
:106800002FEF9207A207B20789F410929F131092FC
:10681000A0131092A1131092A21344E050E06AE575
:1068200070E08FE993E10E94F59608C080939F1372
:106830009093A013A093A113B093A21349E050E04A
:106840006EE070E08EE895E30E94D7960E941313E5
:1068500044E050E06EE470E0CE010B960E94D796C3
:106860008B859C85AD85BE8544E050E06EE470E08C
:106870008F3F9F4FAF4FBF4F29F485E892E00E94B2
:10688000F59604C085E892E00E94D79644E050E077
:106890006AE470E0CE010B960E94D7968B859C85AA
:1068A000AD85BE8544E050E06AE470E08F3F9F4FC5
:1068B000AF4FBF4F29F481E892E00E94F59604C0E3
:1068C00081E892E00E94D79644E050E062E570E0F3
:1068D000CE010B960E94D7968B859C85AD85BE8593
:1068E00044E050E062E570E08F3F9F4FAF4FBF4FF5
:1068F00029F489E892E00E94F59604C089E892E0C4
:106900000E94D79641E050E06DE170E0CE014196E3
:106910000E94D796898941E050E06DE170E08F3F99
:1069200029F48CE993E10E94F59604C08CE993E187
:106930000E94D79641E050E06CE170E0CE014196B4
:106940000E94D796898941E050E06CE170E08F3F6A
:1069500029F485E692E00E94F59604C085E692E06F
:106960000E94D79641E050E06BE170E0CE01419685
:106970000E94D796898941E050E06BE170E08F3F3B
:1069800029F484E692E00E94F59604C084E692E041
:106990000E94D7964AE050E064E070E0CE01019694
:1069A0000E94D79689814AE050E064E070E08F3F12
:1069B00029F48FE89CE10E94F59604C08FE89CE1E1
:1069C0000E94D79644E050E066E570E0CE010B9659
:1069D0000E94D7968B859C85AD85BE8544E050E0AE
:1069E00066E570E08F3F9F4FAF4FBF4F29F48DE8B2
:1069F00092E00E94F59604C08DE892E00E94D7963E
:106A000044E050E067E170E0CE010B960E94D7961B
:106A10008B859C85AD85BE8544E050E067E170E0E4
:106A20008F3F9F4FAF4FBF4F29F480E692E00E9407
:106A3000F59604C080E692E00E94D79680916002AD
:106A400090916102A0916202B091630281389A41F3
:106A5000A640B105A0F083EF92E09F938F930E9430
:106A60002A9480E197E2A0E0B0E0809360029093E6
:106A70006102A0936202B09363020F900F90609145
:106A800060027091610280916202909163020E94A3
:106A9000A16042E050E062E070E0CE010F960E94FB
:106AA000D7968F85988942E050E062E070E08F3F92
:106AB000910529F485E993E10E94F59604C085E9E2
:106AC00093E10E94D79642E050E060E070E0CE0192
:106AD0000F960E94D7968F85988942E050E060E03B
:106AE00070E08F3F910529F483E993E10E94F596C8
:106AF00004C083E993E10E94D79661960FB6F8949B
:106B0000DEBF0FBECDBFDF91CF910895CF92DF9250
:106B1000EF92FF9260917E0270917F0280E090E0A0
:106B20000E944A9360E275E00E946B93892B09F002
:106B30003BC18DE48093A81C80E88093A91C84E06D
:106B40008093AA1C1092AB1C1092AC1C1092AD1C2E
:106B50001092AE1C1092AF1C8CE390E09093B11C8D
:106B60008093B01C1092B21C1092B31C1092B41CF3
:106B70001092B51C1092B61C1092B71C1092B81C43
:106B80001092B91C1092BB1C1092BA1C1092BC1C23
:106B90001092BD1C1092BE1C1092BF1C1092C01C03
:106BA0001092C11C1092C21C1092C31C1092C51CE2
:106BB0001092C41C1092C61C1092C71C1092C81CC4
:106BC0001092C91C1092CA1C1092CB1C1092CC1CA3
:106BD0001092CD1C1092CF1C1092CE1C48E250E0B7
:106BE00062E270E088EA9CE10E94F5968AE090E417
:106BF000A0E0B0E08093660290936702A0936802E1
:106C0000B093690244E050E06EE170E086E692E005
:106C10000E94F59610929F131092A0131092A11348
:106C20001092A21344E050E06AE570E08FE993E12E
:106C30000E94F59682E2C82EDD24DA948CECE82ED0
:106C40008BE3F82EC0928502D0928602E0928702F2
:106C5000F092880244E050E06EE470E085E892E053
:106C60000E94F596C0928102D0928202E092830245
:106C7000F092840244E050E06AE470E081E892E03F
:106C80000E94F59687ED94E3AFEEBCE38093890212
:106C900090938A02A0938B02B0938C0244E050E060
:106CA00062E570E089E892E00E94F5968AE999E948
:106CB000A9E1B0E480938D0290938E02A0938F029D
:106CC000B093900244E050E066E570E08DE892E019
:106CD0000E94F59610929C1380E00E94116B41E097
:106CE00050E06DE170E08CE993E10E94F5968AE155
:106CF000809365020E94EA6941E050E06CE170E037
:106D000085E692E00E94F5968FE08093640241E070
:106D100050E06BE170E084E692E00E94F5968AE034
:106D2000EFE8FCE1DF011D928A95E9F74AE050E0C7
:106D300064E070E0CF010E94F59680E197E2A0E068
:106D4000B0E08093600290936102A0936202B093DE
:106D5000630244E050E067E170E080E692E00E9468
:106D6000F596109296131092951342E050E062E06F
:106D700070E085E993E10E94F596109294131092C9
:106D8000931342E050E060E070E083E993E10E94F9
:106D9000F59681E00E94EA2880E090E0FF90EF9075
:106DA000DF90CF900C942813FF90EF90DF90CF905E
:106DB00008950E9408676C9A6B9A6A9A6F9A729A01
:106DC000749A739A779A809880B3897F80BB8398EE
:106DD000849887E080937E00549A0E9400330E943A
:106DE00031338091660290916702A0916802B09160
:106DF000690294FD0E9417670E94CD0E80E090E02A
:106E00000E94281360916002709161028091620279
:106E1000909163020E94A1600E94DF106093C730CE
:106E20007093C8308093C9309093CA3080916602C5
:106E300086FD239A219A229A239A0E94E20E1D9B94
:106E400005C010929E1310929D13089581E090E06A
:106E500090939E1380939D130895CF93DF9390E0BA
:106E600040919F135091A0136091A1137091A213B0
:106E700041FD08C02091660220FD04C021FF8CC0A6
:106E80001D9B8AC02DE8289FE001299FD00D112469
:106E9000CE018B54924E9F938F9387E295E09F9300
:106EA0008F930E941694FE01E255F24EDF01AA571D
:106EB000BF4F2C910F900F900F900F9043815481F2
:106EC000658176818091CB309091CC30A091CD308E
:106ED000B091CE30841B950BA60BB70B2223D1F1BA
:106EE000BF93AF939F938F93DF01A257BF4F11962C
:106EF0008C9111978F938C918F93129711968C91FF
:106F000011978F938C918F9313978C911F928F93DE
:106F100011978C911F928F9313968C911F928F9340
:106F200011978C911F928F93E957FF4F80811F9289
:106F30008F931F922F938DE295E09F938F930E94E2
:106F400016948DB79EB746960FB6F8949EBF0FBEA7
:106F50008DBF10C0BF93AF939F938F9384E795E04D
:106F60009F938F930E9416940F900F900F900F9005
:106F70000F900F900E94DC1180918002882361F0B5
:106F80001F928F9380EF92E09F938F930E942A9499
:106F90000F900F900F900F90DF91CF9108958091F7
:106FA000AE1D882341F08091AF1D90E00E942D37E7
:106FB0000E94D30FF4CF0895CF93DF93EC01888123
:106FC00099818C3F2EE09207F1F018F4892BC1F0E3
:106FD0004BC084302FE0920709F44CC088309F40AA
:106FE00009F042C086E59AE00E944F6F892B09F4B0
:106FF0003FC086E59AE00E943B6F80E00E941A291C
:107000008CEF9EE02EC0623199F5299A409193133E
:10701000509194135695542F44275795479560E007
:1070200070E086E59AE00E94316F80919F13909105
:10703000A013A091A113B091A213A0FF10C0809142
:1070400094138F93809193138F9389ED91E19F9384
:107050008F930E942A940F900F900F900F9084E0CE
:107060009FE09983888304C01982188283E019C045
:1070700081E017C086E59AE00E944F6F892BC1F32B
:1070800086E59AE00E943B6F0E94CF3740E250E0D5
:1070900060E070E086E59AE00E94316F88E09FE052
:1070A000E0CFDF91CF9108952F923F924F925F9260
:1070B0006F927F928F929F92AF92BF92CF92DF9208
:1070C000EF92FF920F931F93CF93DF93CDB7DEB76D
:1070D0002B970FB6F894DEBF0FBECDBF9B878A8774
:1070E0003A01FC0180819181892B11F00C948B4C29
:1070F00060917E0270917F02CA010E944A9360E80B
:1071000070E0C3010E948A93009759F46091F739A7
:107110007091F8398AE090E00E94DE9381E00C944F
:10712000904C8130910561F4F3011081912E990CFE
:107130009908892C092D292C392C492C592CB9C096
:1071400082309105B9F4F3018081082E000C990B6F
:10715000982F88272181820F911D27FD9A95182F3E
:10716000992E892E880C8808082D282C382C482C1C
:10717000582C9FC083309105B1F5F3012081922FE7
:10718000990F990B392F492F592F692F792F892F53
:1071900000E10E94AE8A19012A014B01B82FA92FE4
:1071A0002181922F990F990B392F492F592F692F30
:1071B000792F892F08E00E94AE8A59016A017B016C
:1071C0008C019101A201B4018B2F9A2F0E94E58AB4
:1071D000A2801A2D110F110BB12EC12ED12EE12E2E
:1071E000F12E012F55C004970CF45BC0F3012081F0
:1071F000922F990F990B392F492F592F692F792FDA
:10720000892F08E10E94AE8A19012A014B01B82F8B
:10721000A92F2181922F990F990B392F492F592F7F
:10722000692F792F892F00E10E94AE8A59016A01E6
:107230007B018C019101A201B4018B2F9A2F0E9436
:10724000E58AA3801A2D110F110BB12EC12ED12E5C
:10725000E12EF12E012F0E94E58A19012A014B012E
:10726000B82FA92F2281922F990F990B392F492FCF
:10727000592F692F792F892F08E00E94AE8A590172
:107280006A017B018C019101A201B4018B2F9A2F1D
:107290000E94E58A122F932E842E052F1B012C01AC
:1072A00008C01AE0912C812C00E0212C312C412CBB
:1072B000512C0E94DC11212F392D482D502FB10166
:1072C000C2012537F3E63F07FDE64F07510561058B
:1072D00071058105910511F40C946A472537E3E6A1
:1072E0003E07EDE64E0751056105710581059105E3
:1072F00011F008F0B2C12337F2E73F07410551050D
:10730000610571058105910511F40C94034A233739
:10731000E2E73E07410551056105710581059105CB
:1073200011F008F0B9C02536F4E63F0741055105D4
:10733000610571058105910509F4D1C72536E4E69B
:107340003E0741055105610571058105910511F063
:1073500008F041C0A6E70E940C8B11F40C94F14395
:107360000E940C8B09F070F4A8E60E940C8B11F4BB
:107370000C94C041A5E70E940C8B11F40C94DB43E4
:107380000C94894C212F392D482D502FB101C20169
:107390002436F1E63F074105510561057105810578
:1073A000910511F40C942B4A2537E2E63E0741057E
:1073B0005105610571058105910509F431C52A332F
:1073C000364241055105610571058105910509F4B4
:1073D00030C30C94894C212F392D482D502FB101E9
:1073E000C2012737EFE63E074105510561057105EA
:1073F0008105910511F40C94D0472737FFE63F072C
:1074000041055105610571058105910509F0C8F433
:107410002436E9E63E074105510561057105810500
:10742000910511F40C94B44325363E4641055105AF
:10743000610571058105910511F40C9404480C94C3
:10744000894C212F392D482D502FB101C2012536ED
:10745000E2E73E074105510561057105810591058A
:1074600011F40C94D0482936F2E73F074105510545
:10747000610571058105910511F40C94B24923331E
:10748000314741055105610571058105910511F0EF
:107490000C94894C0C942B4A212F392D482D502FB8
:1074A000B101C2012236F5E63F07F4E64F07510568
:1074B000610571058105910509F411C72236E5E6DC
:1074C0003E07E4E64E07510561057105810591050A
:1074D00011F008F05BC02133F4E63F07F1E64F07F7
:1074E0005105610571058105910509F4B6C2213385
:1074F000E4E63E07E1E64E075105610571058105A9
:10750000910509F0C0F42337F3E73F074105510522
:10751000610571058105910511F40C94174A28370E
:10752000344741055105610571058105910509F44F
:1075300080C20C94894C212F392D482D502FB10138
:10754000C2012837F4E63F07F1E64F075105610510
:1075500071058105910509F47CC22C36E5E73E07EB
:10756000E2E64E075105610571058105910509F4B3
:1075700057C42336344641465105610571058105DE
:10758000910511F00C94894C0C942B4A212F392D24
:10759000482D502FB101C2012D36E5E73E07E8E640
:1075A0004E075105610571058105910511F40C9493
:1075B000414A2D36F5E73F07F8E64F0751056105CB
:1075C00071058105910509F0E0F42237E2E73E07F5
:1075D000E5E64E075105610571058105910511F438
:1075E0000C941B4723363D464846510561057105FD
:1075F0008105910511F00C94894C0E94AE1C0C94ED
:107600008B4C212F392D482D502FB101C20124362A
:10761000E3E63E07ECE64E0751056105710581057D
:10762000910511F40C947E462736FFE63F07FCE6F1
:107630004F075105610571058105910511F40C9401
:10764000814623363243494651056105710581055E
:10765000910511F00C94894C20C2212F392D482D11
:10766000502FB101C2012037FCE63F07F5E64F0776
:10767000F8E65F07610571058105910509F480C68B
:107680002037ECE63E07E5E64E07E8E65E076105D3
:1076900071058105910511F008F0E0C02437F8E785
:1076A0003F07F4E74F075105610571058105910515
:1076B00011F40C945D442437E8E73E07E4E74E07F5
:1076C0005105610571058105910511F008F05DC056
:1076D0002033F1E33F07F1E74F07510561057105DD
:1076E0008105910511F40C941B472033E1E33E071B
:1076F000E1E74E075105610571058105910509F026
:10770000C0F42133F2E63F07F0E74F07510561056A
:1077100071058105910509F498C22233324640472C
:107720005105610571058105910509F4E3C20C94C9
:10773000894C212F392D482D502FB101C2012037FE
:10774000F5E63F07F2E74F07510561057105810531
:10775000910511F40C94D0482C36E4E73E074E070F
:107760005105610571058105910511F40C94A64B35
:10777000213331434147510561057105810591056B
:1077800011F00C94894C0C946A47212F392D482D07
:10779000502FB101C2012B36ECE63E07E5E74E075C
:1077A000E2E65E07610571058105910509F438C3BC
:1077B0002B36FCE63F07F5E74F07F2E65F0761056A
:1077C00071058105910509F0E0F42437E4E63E07F0
:1077D000E7E74E075105610571058105910511F433
:1077E0000C94F44B24373F464F46524661057105D1
:1077F0008105910511F00C94894C0C9400000C94B7
:107800008B4C212F392D482D502FB101C2012E361E
:10781000E1E63E07E8E64E07E3E65E07610571052F
:107820008105910511F40C9431442633F9E63F07A4
:10783000F5E74F07F5E65F076105710581059105DD
:1078400009F4A2C529363C464146534661057105F7
:107850008105910511F00C94894C7FC3212F392D9E
:10786000482D502FB101C2012437F3E73F07F5E659
:107870004F07F2E75F07610571058105910511F476
:107880000C9480482437E3E73E07E5E64E07E2E73D
:107890005E07610571058105910511F008F062C070
:1078A0002337F5E63F07F2E74F07F0E75F0761058B
:1078B00071058105910511F40C94F14A2337E5E631
:1078C0003E07E2E74E07E0E75E07610571058105C7
:1078D000910509F0D0F42136FDE63F07F5E74F07A3
:1078E000F8E65F07610571058105910511F40C94B7
:1078F000EE472237374740475047610571058105FC
:10790000910509F45CC20C94894C212F392D482D26
:10791000502FB101C2012436FDE63F07F3E64F07C1
:10792000F2E75F07610571058105910509F437C626
:107930002136ECE63E07E5E64E07E2E75E07610525
:1079400071058105910509F43CC523373247474746
:107950005047610571058105910511F00C94894C22
:107960000C948348212F392D482D502FB101C2018D
:107970002437E2E73E07E1E64E07E5E75E076105EB
:1079800071058105910509F465C62437F2E73F07C3
:10799000F1E64F07F5E75F07610571058105910580
:1079A00009F0C8F42437E3E73E07E5E64E07E4E7CD
:1079B0005E07610571058105910509F4A9C727379F
:1079C000304748475447610571058105910509F421
:1079D0001EC70C94894C212F392D482D502FB101F1
:1079E000C2012F36ECE63E07EFE54E07E6E75E07FD
:1079F000610571058105910509F47CC52C36F1E618
:107A00003F07F4E74F07F8E75F0761057105810558
:107A1000910511F40C94734B223737464047554774
:107A2000610571058105910511F00C94894C0C9448
:107A30005A4683E080937C3510927E3510927D35D6
:107A40004CE755E362E182E492E00E94C1700C943D
:107A50008B4C0E94371C0C948B4C21E042E161E07E
:107A600080ED0E947E6221E042E161E080ED0E94B3
:107A70007E6221E042E161E080ED0E947E6221E0D1
:107A800042E161E080ED0E947E6221E042E161E03E
:107A900080ED0E947E620C948B4C60917E0270910E
:107AA0007F0280E090E00E944A9360E875E00E94C7
:107AB0006B93892B09F0C5C060917E0270917F02A3
:107AC00080E090E00E944A938C01009709F497C0EF
:107AD00064E673E00E946B93892BE1F488EE93E0F7
:107AE000A0E0B0E08093600290936102A0936202F4
:107AF000B093630268EE73E080E090E00E94A160C2
:107B000044E050E067E170E080E692E00E94F59684
:107B10000C948B4C66E875E0C8010E946B93892B2E
:107B2000E1F480E197E2A0E0B0E0809360029093FE
:107B30006102A0936202B093630260E177E280E0A9
:107B400090E00E94A16044E050E067E170E080E6D0
:107B500092E00E94F5960C948B4C69E875E0C801A0
:107B60000E946B93892BE1F480EA96E8A1E0B0E0F3
:107B70008093600290936102A0936202B0936302CB
:107B800060EA76E881E090E00E94A16044E050E085
:107B900067E170E080E692E00E94F5960C948B4CD1
:107BA0006DE875E0C8010E946B93892BE1F480E8D1
:107BB0009AE1A6E0B0E08093600290936102A09306
:107BC0006202B093630260E87AE186E090E00E948E
:107BD000A16044E050E067E170E080E692E00E943E
:107BE000F5960C948B4C8FEA94E09F938F930E94B0
:107BF0002A940E94DC110F900F900C948B4C609192
:107C0000600270916102809162029091630228EE9D
:107C100033E040E050E00E94D9885F934F933F9358
:107C20002F938BEA94E09F938F930E942A940E9453
:107C3000DC110F900F900F900F900F900F900C94FD
:107C40008B4C0E946E160C948B4C60917E0270914E
:107C50007F0280E090E00E944A938C0169E175E028
:107C60000E946B93892BA1F4809166029091670228
:107C7000A0916802B0916902A2608093660290931D
:107C80006702A0936802B0936902299A0C948B4C06
:107C90006CE175E0C8010E946B93892BB1F480916F
:107CA000660290916702A0916802B0916902AD7F6F
:107CB0008093660290936702A0936802B093690272
:107CC00080E00E941A290C948B4C299903C08CE106
:107CD00095E002C089E195E09F938F9383EA94E059
:107CE0009F938F930E942A940F900F900F900F9064
:107CF0000C948B4C60917E0270917F0280E090E04A
:107D00000E944A938C0169E175E00E946B93892B74
:107D1000E1F48091660290916702A0916802B091AF
:107D20006902A4608093660290936702A093680240
:107D3000B09369022A9A44E050E06EE170E086E672
:107D400092E00E94F5960C948B4C6CE175E0C801B2
:107D50000E946B93892BF1F48091660290916702E7
:107D6000A0916802B0916902AB7F80936602909304
:107D70006702A0936802B093690280E00E94202904
:107D800044E050E06EE170E086E692E00E94F596F5
:107D90000C948B4C2A9903C08CE195E002C089E1D8
:107DA00095E09F938F938BE994E09F938F930E942C
:107DB0002A940F900F900F900F900C948B4C609121
:107DC0007E0270917F0280E090E00E944A938C01D5
:107DD00069E175E00E946B93892B19F477980C94F4
:107DE0008B4C6CE175E0C8010E946B93892B19F4F0
:107DF000779A0C948B4C779B03C08CE195E002C082
:107E000089E195E09F938F9381E696E09F938F930E
:107E10000E942A940F900F900F900F900C948B4C0F
:107E200060917E0270917F0280E090E00E944A9310
:107E30008C0161E975E00E946B93892BD1F48091EC
:107E4000AE1D1F928F938091B01D1F928F938091D2
:107E5000AF1D1F928F931F9284E18F9381E794E06F
:107E60009F938F930E942A940FB6F894DEBF0FBEA3
:107E7000CDBF66E975E0C8010E946B93892B19F4A8
:107E80000E94CF3766C06EE975E0C8010E946B930F
:107E9000892BF1F560917E0270917F0280E090E085
:107EA0000E944A93009709F454C00E94379285318A
:107EB000910528F5909396138093951342E050E036
:107EC00062E070E085E993E10E94F59660917E02A0
:107ED00070917F0280E090E00E944A930097C9F180
:107EE0000E943792909394138093931342E050E052
:107EF00060E070E083E993E10E94F5962AC08FE587
:107F000094E09F938F930E942A940F900F9021C02A
:107F1000809196138F93809195138F9386E594E0CB
:107F20009F938F930E942A940E94DC118091941356
:107F30008F93809193138F9387E494E09F938F9313
:107F40000E942A940E94DC110FB6F894DEBF0FBE87
:107F5000CDBF0E94DC110C948B4C60917E0270911D
:107F60007F0280E090E00E944A938C016EED74E005
:107F70000E946B93892B09F077C060917E0270910B
:107F80007F0280E090E00E944A938C01009711F4F8
:107F90000C948B4C6CE975E00E946B93892BB1F4C7
:107FA00082E29FEFACECBBE3809385029093860264
:107FB000A0938702B093880244E050E06EE470E042
:107FC00085E892E00E94F5960C948B4C62EA75E08D
:107FD000C8010E946B93892BB1F482E29FEFACEC55
:107FE000BAE38093850290938602A0938702B093B0
:107FF000880244E050E06EE470E085E892E00E9480
:10800000F5960C948B4CC8010E9433922B013C01D5
:1080100020E030E0A9010E94F78B8823D9F081E0AD
:108020000E947D109B01AC01C301B2010E94FC8B38
:1080300060938502709386028093870290938802F2
:1080400044E050E06EE470E085E892E00E94F5962E
:108050000C948B4C8AE394E09F938F930E942A9414
:108060000F900F900C948B4C61EE74E0C8010E944D
:108070006B93892B09F077C060917E0270917F022B
:1080800080E090E00E944A938C01009711F40C94D8
:108090008B4C6CE975E00E946B93892BB1F482E202
:1080A0009FEFACECBBE38093810290938202A0939C
:1080B0008302B093840244E050E06AE470E081E817
:1080C00092E00E94F5960C948B4C62EA75E0C80130
:1080D0000E946B93892BB1F482E29FEFACECBAE380
:1080E0008093810290938202A0938302B0938402D2
:1080F00044E050E06AE470E081E892E00E94F59686
:108100000C948B4CC8010E9433922B013C0120E05F
:1081100030E0A9010E94F78B8823D9F082E00E9409
:108120007D109B01AC01C301B2010E94FC8B6093E6
:10813000810270938202809383029093840244E0D0
:1081400050E06AE470E081E892E00E94F5960C94B9
:108150008B4C8DE294E09F938F930E942A940F9012
:108160000F900C948B4C69ED74E0C8010E946B93E6
:10817000892B09F073C060917E0270917F0280E0CC
:1081800090E00E944A938C01009711F40C948B4C60
:108190006CE975E00E946B93892BB1F487ED94E351
:1081A000AFEEBCE38093890290938A02A0938B0286
:1081B000B0938C0244E050E062E570E089E892E020
:1081C0000E94F5960C948B4C62EA75E0C8010E94FF
:1081D0006B93892B51F48EE194E09F938F930E94CF
:1081E0002A940F900F900C948B4CC8010E943392EC
:1081F0002B013C0120E030E0A9010E94F78B88238D
:1082000019F180E00E947D104B015C0121EE3AE7FC
:1082100044E95EE3C301B2010E94188BA5019401F9
:108220000E94FC8B6093890270938A0280938B0278
:1082300090938C0244E050E062E570E089E892E0BF
:108240000E94F5960C948B4C81E194E09F938F9360
:108250000E942A940F900F900C948B4C0E94CB108C
:108260009F938F937F936F938AE094E09F938F9374
:108270000E942A9482E00E947D1020918102309118
:10828000820240918302509184020E94A88E162F90
:10829000072FF82EE92E81E00E947D10EF92FF92C9
:1082A0000F931F932091850230918602409187029F
:1082B000509188020E94A88E9F938F937F936F9313
:1082C0008EEF93E09F938F930E942A940E94DC117B
:1082D0000FB6F894DEBF0FBECDBF0C948B4C6091EF
:1082E0007E0270917F0280E090E00E944A930097A6
:1082F00011F10E94192A00919F131091A01320914F
:10830000A1133091A213601771078207930739F107
:1083100060939F137093A0138093A1139093A21363
:1083200044E050E06AE570E08FE993E10E94F59641
:108330008AE596E002C083E596E09F938F930E94C2
:108340002A9460919F137091A0138091A113909132
:10835000A2130E9426290E94DC110F900F9088E43E
:1083600096E09F938F930E942A946FEF7FEFCB014B
:108370000E9426290E94DC110F900F900C948B4CC8
:108380000E9409260C948B4CF3018481843329F4D8
:1083900040E061E080E00E945118809180028823D3
:1083A00011F40C948B4C1F928F9385E496E09F936D
:1083B0008F930E942A940F900F900F900F900C941F
:1083C0008B4CF3018481893709F080C060917E0273
:1083D00070917F0280E090E00E944A938C0169E1F5
:1083E00075E00E946B93892B51F480916602909105
:1083F0006702A0916802B0916902906410C06CE1BC
:1084000075E0C8010E946B93892BD1F480916602BC
:1084100090916702A0916802B09169029F7B80935E
:10842000660290936702A0936802B093690244E0E9
:1084300050E06EE170E086E692E00E94F59646C05C
:1084400067EA75E0C8010E946B93892B21F5809142
:10845000A71C8F938091A61C8F938091A51C8F934E
:108460008091A41C8F938091A31C8F938091A21C58
:108470008F938091A11C8F938091A01C8F9383ED8B
:1084800093E09F938F930E942A940FB6F894DEBFD7
:108490000FBECDBF1BC08091660290916702A09174
:1084A0006802B091690296FD03C08CE195E002C0BC
:1084B00089E195E09F938F938FEC93E09F938F9347
:1084C0000E942A940F900F900F900F90809180023D
:1084D000882311F40C948B4C1F928F9382E496E0C6
:1084E0009F938F930E942A940F900F900F900F905C
:1084F0000C948B4CF30184818737E9F560917E02FF
:1085000070917F0280E090E00E944A930097D9F03A
:108510000E9433922B013C0120E030E0A9010E942F
:10852000F78B882381F040928D0250928E026092E8
:108530008F027092900244E050E066E570E08DE8B2
:1085400092E00E94F596809190028F9380918F0225
:108550008F9380918E028F9380918D028F9381EC07
:1085600093E09F938F930E942A940F900F900F9007
:108570000F900F900F9080918002882311F40C943B
:108580008B4C1F928F938FE396E09F938F930E9463
:108590002A940F900F900F900F900C948B4C609139
:1085A0007E0270917F0280E090E00E944A938C01ED
:1085B00069E175E00E946B934090660250906702FB
:1085C0006090680270906902892B19F4689457F8DA
:1085D00009C06CE175E0C8010E946B93892B99F486
:1085E000E89457F8409266025092670260926802DF
:1085F0007092690244E050E06EE170E086E692E03D
:108600000E94F59613C057FC03C08CE195E002C0B0
:1086100089E195E09F938F938DEB93E09F938F93E8
:108620000E942A940F900F900F900F9080918002DB
:10863000882311F40C948B4C1F928F938CE396E05B
:108640009F938F930E942A940F900F900F900F90FA
:108650000C948B4C60917E0270917F0280E090E0E0
:108660000E944A938C016DEA75E00E946B93892BFE
:1086700011F489E108C061EB75E0C8010E946B93B9
:10868000892B49F480E18093C4001092C50082E0F8
:108690008093C00055C065EB75E0C8010E946B93E4
:1086A000892B11F488E0EFCF6AEB75E0C8010E94D6
:1086B0006B93892B39F06FEB75E0C8010E946B93C7
:1086C000892B11F483E0DFCF8091C400893141F41C
:1086D00088EB93E09F938F930E942A940F900F90C2
:1086E0008091C400803141F483EB93E09F938F939A
:1086F0000E942A940F900F908091C400883041F41A
:108700008DEA93E09F938F930E942A940F900F908D
:108710008091C400833041F487EA93E09F938F9364
:108720000E942A940F900F908091C400883041F4E9
:1087300081EA93E09F938F930E942A940F900F9069
:1087400080918002882311F40C948B4C1F928F939C
:1087500089E396E09F938F930E942A940F900F9045
:108760000F900F900C948B4C60917E0270917F0261
:1087700080E090E00E944A936CE975E00E946B9360
:10878000892B11F481E001C080E00E94EA288091E9
:108790008002882311F40C948B4C1F928F9386E3F4
:1087A00096E09F938F930E942A940F900F900F90C2
:1087B0000F900C948B4C0E9410278091800288238C
:1087C00011F40C948B4C1F928F9383E396E09F934C
:1087D0008F930E942A940F900F900F900F900C94FB
:1087E0008B4C0E940C2780918002882311F40C94FA
:1087F0008B4C1F928F9380E396E09F938F930E9400
:108800002A940F900F900F900F900C948B4C6091C6
:108810007E0270917F0280E090E00E944A930E9465
:108820003792803170F480939C130E94116B41E069
:1088300050E06DE170E08CE993E10E94F5960C94B4
:108840008B4C80919C131F928F9387E993E09F93A9
:108850008F930E942A940F900F900F900F900C947A
:108860008B4C60917E0270917F0280E090E00E94CC
:108870004A930E94379295EF980F903170F480934D
:1088800065020E94EA6941E050E06CE170E085E633
:1088900092E00E94F5960C948B4C809165021F9299
:1088A0008F938EE893E09F938F930E942A940F906A
:1088B0000F900F900F900C948B4C60917E027091F2
:1088C0007F0280E090E00E944A93009789F04AE09E
:1088D00050E0BC018FE89CE10E947B934AE050E0AD
:1088E00064E070E08FE89CE10E94F5960C948B4C5C
:1088F0008FE89CE19F938F9384EC95E09F938F93F7
:108900000E9416940F900F900F900F900C948B4C28
:1089100060917E0270917F0280E090E00E944A9315
:108920008C0164E673E00E946B93892BE1F4219A39
:108930008091660290916702A0916802B0916902ED
:1089400080618093660290936702A0936802B0935F
:10895000690244E050E06EE170E086E692E00E9439
:10896000F5960C948B4C62EE74E0C8010E946B93F8
:10897000892BD9F4229A8091660290916702A09186
:108980006802B091690280628093660290936702E8
:10899000A0936802B093690244E050E06EE170E099
:1089A00086E692E00E94F596B6C766E473E0C801D9
:1089B0000E946B93892BD9F4239A8091660290913F
:1089C0006702A0916802B091690280648093660298
:1089D00090936702A0936802B093690244E050E06C
:1089E0006EE170E086E692E00E94F59694C765E835
:1089F00074E0C8010E946B93892BD9F4239A80916B
:108A0000660290916702A0916802B0916902806845
:108A10008093660290936702A0936802B093690204
:108A200044E050E06EE170E086E692E00E94F59648
:108A300072C76AE779E0C8010E946B93892B71F5D0
:108A400081E08093E03088EA9CE19093E23080936B
:108A5000E1301092E4301092E33080916602909100
:108A60006702A0916802B0916902916080936602EA
:108A700090936702A0936802B093690244E050E0CB
:108A80006EE170E086E692E00E94F59640EE50E3DB
:108A900062E182E492E00E94C1703DC76DE673E03E
:108AA000C8010E946B93892B11F5E8EDFCE111924E
:108AB00011922CE1E83FF207D1F780916602909184
:108AC0006702A0916802B091690292608093660289
:108AD00090936702A0936802B093690244E050E06B
:108AE0006EE170E086E692E00E94F59614C76CE1B4
:108AF00075E0C8010E946B93409166025091670235
:108B00006091680270916902892BC1F44F705C7F9B
:108B10004093660250936702609368027093690203
:108B20002B9A44E050E06EE170E086E692E00E940D
:108B3000F596809185350E94FF69EDC644FD03C01E
:108B40008CE195E002C089E195E09F938F9383E8E3
:108B500093E09F938F930E942A94809166020F90D6
:108B60000F900F900F9085FD03C08CE195E002C03F
:108B700089E195E09F938F9388E793E09F938F938C
:108B80000E942A94809166020F900F900F900F9090
:108B900086FD03C08CE195E002C089E195E09F93DA
:108BA0008F938DE693E09F938F930E942A948091F8
:108BB00066020F900F900F900F9087FD03C08CE11D
:108BC00095E002C089E195E09F938F9382E693E060
:108BD0009F938F930E942A948091660290916702DE
:108BE000A0916802B09169020F900F900F900F90C2
:108BF00090FD03C08CE195E002C089E195E09F9370
:108C00008F9387E593E09F938F930E942A9480919E
:108C1000660290916702A0916802B09169020F907C
:108C20000F900F900F9091FD03C08CE195E002C072
:108C300089E195E09F938F938CE493E09F938F93CA
:108C40000E942A948091660290916702A091680226
:108C5000B09169020F900F900F900F9091FF5BC63B
:108C60008CEC95E00E94529498EDE92E9CE1F92E4F
:108C700000E010E024ED822E25E0922EF7018081A5
:108C80009181F2E0EF0EF11C9F938F93C8010B9638
:108C90009F938F939F928F920E9416940F5F1F4F06
:108CA0000F900F900F900F900F900F9000311105C3
:108CB00029F731C68CE296E09F938F930E942A9405
:108CC000809180020F900F90882361F01F928F9304
:108CD00089E296E09F938F930E942A940F900F90C1
:108CE0000F900F90F89498E088E10FB6F894A8954B
:108CF000809360000FBE90936000FFCF0E942F62B0
:108D00000AC660917E0270917F0280E090E00E942E
:108D10004A938C0169E175E00E946B93892BE9F419
:108D20000E94EE688091660290916702A0916802AD
:108D3000B09169028D7F8160809366029093670293
:108D4000A0936802B093690244E050E06EE170E0E5
:108D500086E692E00E94F596DEC56CE175E0C801FA
:108D60000E946B93892BE1F40E9424688091660233
:108D700090916702A0916802B09169028C7F809304
:108D8000660290936702A0936802B093690244E080
:108D900050E06EE170E086E692E00E94F596BBC579
:108DA0006FED75E0C8010E946B93892BE9F40E9476
:108DB00024688091660290916702A0916802B09148
:108DC00069028E7F82608093660290936702A0930F
:108DD0006802B093690244E050E06EE170E086E61C
:108DE00092E00E94F59697C58091660281FF0FC0C0
:108DF0008FED95E09F938F9388E493E09F938F93FB
:108E00000E942A940F900F900F900F9084C580FDC0
:108E100003C08CE195E002C089E195E09F938F93B8
:108E200084E493E09F938F930E942A940F900F9075
:108E30000F900F9070C58091DE308F938091DD3060
:108E40008F938091DC308F938091DB308F93809172
:108E5000DA308F938091D9308F938091D8308F936F
:108E60008091D7308F938091D6308F938091D53079
:108E70008F938091D4308F938091D3308F93809152
:108E8000D2308F938091D1308F938091D0308F9357
:108E90008091CF308F938DEF95E09F938F930E94B9
:108EA0002A940E94DC11809180020FB6F894DEBFF4
:108EB0000FBECDBF882309F42EC51F928F938AEF72
:108EC00095E09F938F930E942A940F900F900F909C
:108ED0000F9021C5F89489E021E030E0F9018093FA
:108EE0005700C895E02C20E030E0F901809357004E
:108EF000C895F02C7894F89423E030E0F901809341
:108F00005700C895002D22E030E0F901809357000A
:108F1000C895102D78948091B8288F938091B728A8
:108F20008F938091B6288F938091B5288F9380EF8F
:108F300095E09F938F930E942A941F92EF921F9225
:108F4000FF921F920F931F921F9389EC95E09F93BE
:108F50008F930E942A940E94AA27809166001F92F4
:108F60008F938DEB95E09F938F930E942A940E949C
:108F7000DC11809180020FB6F894DEBF0FBECDBF2A
:108F8000882309F4C8C41F928F938AEB95E09F93BE
:108F90008F930E942A940F900F900F900F90BBC454
:108FA00060E070E080E090E00E94E51160E070E039
:108FB00081E090E00E94E51180918002882309F40D
:108FC000AAC41F928F9387EB95E09F938F930E9483
:108FD0002A940F900F900F900F909DC40E94CC2563
:108FE0000E94DC1180918002882309F494C41F92AE
:108FF0008F9384EB95E09F938F930E942A940F9018
:109000000F900F900F9087C460917E0270917F0245
:1090100080E090E00E944A9366E975E00E946B93BD
:10902000892B31F5F89481E99AE00E949A718C01BC
:10903000892B69F0C8010F960E94076EB80188E07D
:1090400092E00E944B72C8010E94FF71F0CF81E94B
:109050009AE00E94F271892B29F081E99AE00E943E
:10906000AE71F5CF81E99AE00E949671789436C08E
:1090700081E99AE00E949A718C0184EEE82E85E0E5
:10908000F82E0115110551F1F80186811F928F9379
:1090900080851F928F9385811F928F9381851F9268
:1090A0008F9387811F928F9384811F928F938381E7
:1090B0001F928F9382811F928F9382851F928F932D
:1090C000FF92EF920E941694C8010E94FF718C01DA
:1090D0000FB6F894DEBF0FBECDBFD3CF8091800214
:1090E000882309F418C41F928F9381EB95E09F9316
:1090F0008F930E942A940F900F900F900F900BC4A3
:109100000E94863508C460917E0270917F0280E0E3
:1091100090E00E944A938C0163E276E00E946B9398
:10912000892BD1F48091660290916702A091680228
:10913000B0916902977F8093660290936702A09333
:109140006802B093690244E050E06EE170E086E6A8
:1091500092E00E94F596DFC362EA75E0C8010E94C2
:109160006B93892BD1F48091660290916702A09154
:109170006802B091690298608093660290936702DA
:10918000A0936802B093690244E050E06EE170E0A1
:1091900086E692E00E94F596BEC30E945F0EBBC3B6
:1091A00060917E0270917F0280E090E00E944A937D
:1091B000FC0120812332C1F44AE050E060E070E01D
:1091C00001960E94D18F7B836A8360917E027091A9
:1091D0007F0280E090E00E944A932A813B81243004
:1091E00031050CF096C002C01B821A82009709F468
:1091F00090C01982BE016F5F7F4F0E94892E1901B6
:109200003A014B01B82FA92F8AE02A813B81829F26
:10921000F001839FF00D1124E855F34E40805180FA
:1092200032813C8383818D8394819E8325812F832A
:1092300036813887878189879101A301B4018B2FFB
:109240009A2F5201CC80DD80EE80FF800885198541
:109250000E94038B09F460C08981811103C02082C0
:1092600031822AC0181684F4422853289C81692A26
:109270002D81722A3E81832A8F81982A9885B92B65
:109280002985A22B408217C020943094609470945A
:1092900080949094B095A095242053203C81632223
:1092A0008D8178229E8189222F8192223885B32355
:1092B0008985A8232082518262827382848295826A
:1092C000B683A78348E250E062E270E088EA9CE15E
:1092D0000E94F59689EA95E09F938F930E942A94C5
:1092E0008AE02A813B81829FF001839FF00D112447
:1092F000E855F34E2081318142815381648175812B
:10930000868197810E94D22A0E94DC110F900F90D3
:1093100003C082E00E943F308DE995E09F938F93D8
:109320000E942A942FEF3FEF4FEF5FEF6FEF7FEF39
:109330008FEF9FEF0E94D22A0E94DC118091800261
:109340000F900F90882309F4E6C21F928F938AE949
:1093500095E09F938F930E942A940F900F900F9007
:109360000F90D9C260917E0270917F0280E090E000
:109370000E944A93FC0120812332A1F44AE050E08C
:1093800060E070E001960E94D18F8B0160917E02B7
:1093900070917F0280E090E00E944A9304301105B2
:1093A000ECF402C000E010E00097C1F04AE050E0A9
:1093B00060E070E00E94FC902AE0209FF001219F75
:1093C000F00D1124E855F34E7187608748E250E0B4
:1093D00062E270E088EA9CE10E94F59681E00E94DA
:1093E0003F3080918002882309F495C21F928F93A9
:1093F00087E995E09F938F930E942A940F900F9096
:109400000F900F9088C20E948E72809180028823F4
:1094100009F481C21F928F9384E995E09F938F9303
:109420000E942A940F900F900F900F9074C20E9488
:10943000043180918002882309F46DC21F928F93BA
:1094400081E995E09F938F930E942A940F900F904B
:109450000F900F9060C280E090E00E94C62780913C
:109460008002882309F457C21F928F938EE895E0FB
:109470009F938F930E942A940F900F900F900F90BC
:109480004AC28091C52C81FF2DC00E945225892B94
:1094900049F58091BC288F938091BB288F93809150
:1094A000BA288F938091B9288F9383E895E09F9392
:1094B0008F930E942A9480919D358F9380919C3543
:1094C0008F9380919B358F9380919A358F9386E708
:1094D00095E09F938F930E942A940FB6F894DEBF75
:1094E0000FBECDBF0E94DC118091C52C9091C62C7F
:1094F00090FF63C081E090E00E94CA247B011C01C0
:1095000080E090E00E94CA244B018C010E94282434
:109510003F922F92FF92EF9285E695E09F938F9373
:109520000E942A941F930F939F928F9285E595E056
:109530009F938F930E942A94240138019401A801DB
:1095400047018101B701C1010E94C7229F938F93F8
:109550007F936F938AE495E09F938F930E942A9460
:10956000242D352D462D572D6E2D792D822D912FA1
:109570000E9428239F938F937F936F938CE395E0B2
:109580009F938F930E942A94242D352D462D572D7D
:109590006E2D792D822D912F0E9489239F938F9379
:1095A0007F936F9389E295E09F938F930E942A9413
:1095B0000FB6F894DEBF0FBECDBF0E94DC118091C4
:1095C0008002882309F4A7C11F928F9386E295E059
:1095D0009F938F930E942A940F900F900F900F905B
:1095E0009AC18091C52C82FF2BC021E048E061E048
:1095F00083E00E94BC198091AC1D8F938091AB1DBC
:109600008F938091AA1D8F938091A91D8F93809134
:10961000A81D8F938091A71D8F938091A61D8F9376
:109620008091A51D8F938FE095E09F938F930E946B
:109630002A940E94DC110FB6F894DEBF0FBECDBF96
:109640008091C52C9091C62C91FF3BC00E94211E99
:1096500020E030E048EC52E4162F072FF82EE92ED8
:109660000E94A88E20E836EE45EC57E40E94FC8B61
:1096700021E03EED42E45EE30E94158F9B01AC01C8
:1096800060E070E080E89FE30E94188B2BE43AE3EF
:109690004DEB57E30E94FC8B9F938F937F936F93C7
:1096A000EF92FF920F931F9386EF94E09F938F9317
:1096B0000E942A940E94DC110FB6F894DEBF0FBE00
:1096C000CDBF80918002882309F425C11F928F931A
:1096D00083EF94E09F938F930E942A940F900F90B2
:1096E0000F900F9018C160917E0270917F0280E010
:1096F00090E00E944A9368E276E00E946B93892B87
:1097000099F460917E0270917F0280E090E00E9467
:109710004A93009709F4FFC00E943792909152013A
:10972000892B80935201F7C0809152018F701F9254
:109730008F9387E393E09F938F930E942A940E94D4
:10974000DC110F900F900F900F90E5C060917E029A
:1097500070917F0280E090E00E944A93009711F19F
:109760004AE050E060E070E00E94D18F603198F4F0
:10977000609364021F926F9386EE94E09F938F93A1
:109780000E942A9441E050E06BE170E084E692E0B0
:109790000E94F59611C0809164021F928F938DED07
:1097A00094E006C0809164021F928F9384ED94E050
:1097B0009F938F930E942A940F900F900F900F9079
:1097C0000E94DC1180918002882309F4A4C01F92BA
:1097D0008F9381ED94E09F938F930E942A940F9032
:1097E0000F900F900F9097C060917E0270917F0252
:1097F00080E090E00E944A938C0169E175E00E944C
:109800006B93892BE1F40E94176780916602909117
:109810006702A0916802B09169029061809366022C
:1098200090936702A0936802B093690244E050E00D
:109830006EE170E086E692E00E94F5966CC06CE105
:1098400075E0C8010E946B93892B99F5F8940E94EA
:1098500024670FB6F894A895809160008861809382
:109860006000109260000FBE84B7877F84BF809134
:10987000600088618093600010926000789480910D
:10988000660290916702A0916802B09169029F7E82
:109890008093660290936702A0936802B093690276
:1098A00044E050E06EE170E086E692E00E94F596BA
:1098B00032C06DE276E0C8010E946B93409166026F
:1098C000509167026091680270916902892B69F476
:1098D00054FF02C0F894FFCF86E293E09F938F93EA
:1098E0000E942A940F900F9016C054FD03C08CE183
:1098F00095E002C089E195E09F938F9382E293E027
:109900009F938F930E942A940F900F900F900F9027
:1099100002C00E94F025EA85FB851182108283E057
:109920002B960FB6F894DEBF0FBECDBFDF91CF915F
:109930001F910F91FF90EF90DF90CF90BF90AF906D
:109940009F908F907F906F905F904F903F902F905F
:109950000895CF93DF93EC0188819981009741F0BE
:109960008830924109F48CC01982188283E093C038
:109970000E94D9368091660280FD05C081FF01C03A
:109980001D9B0E942468809170008C7F80937000E2
:109990008091B60080628093B6001092B20082E09F
:1099A0008093B1008091B6008770E1F780917000DC
:1099B0008160809370006DE77EE080E090E00E941F
:1099C000F1660E940C2780E00E94EA2885E092E17F
:1099D0009F938F930E942A940E946E168091C52CAB
:1099E0000F900F9086FD0E94DB618091C52C9091B5
:1099F000C62C90FD0E94E0238091C52C87FF06C0F5
:109A000021E04CE061E080ED0E947E6280919C1339
:109A10000E94116B809165020E94EA690E94E769C9
:109A20008093810A809165020E94EA6980919C136B
:109A30001F928F938091810A1F928F9382E396E009
:109A40009F938F930E9416941092830A1092820A19
:109A50000F900F900F900F900F900F9086E592E06F
:109A6000909398358093973583E290E09093981384
:109A70008093971388E092E19983888381E00BC0FB
:109A80006332E1F744EF50E360E070E082E89AE08F
:109A90000E945438E3CFDF91CF9108950F931F9325
:109AA000CF93DF93EC018A0188819981009711F1AE
:109AB0008D31924121F01982188283E020C06231F9
:109AC000E9F4A80162E170E082E89AE00E9454386B
:109AD00084E080937C3510927E3510927D35109312
:109AE000803500937F354CE755E362E182E492E0F4
:109AF0000E94C1708DE192E19983888381E0DF91BA
:109B0000CF911F910F9108958436910514F19F9381
:109B10008F9388E896E09F938F930E94169480918C
:109B2000CF309091D030A091D130B091D230019609
:109B3000A11DB11D8093CF309093D030A093D13030
:109B4000B093D2300F900F900F900F9081E090E083
:109B5000089580E090E008952F923F924F925F9297
:109B60006F927F928F929F92AF92BF92CF92DF922D
:109B7000EF92FF920F931F93CF93DF93CDB7DEB792
:109B8000CC59D1090FB6F894DEBF0FBECDBFCB566E
:109B9000DF4F99838883C559D0408A01633871F4B7
:109BA00086E89AE0C456DF4F6883CC59D0400E94C3
:109BB000DF73C456DF4F6881CC59D040CB56DF4F9E
:109BC000A881B981C559D0402D913C91253BB1E187
:109BD0003B0711F40C94795B40F42115310581F0B9
:109BE0002B3D3F4009F43BC42FC4273C41E13407DF
:109BF00009F409C42E3C314111F40C94815B24C456
:109C00004AE259E061E870E086E89AE00E94C47395
:109C10008BED9FE0EFC35A01E3E0F0E0EC0FFD1F96
:109C2000E40FF51F1082CA010E94844D892B81F731
:109C300020E030E040E050E0CC56DF4F6881C4596E
:109C4000D040627070E080E090E0A0E00E940C8B59
:109C500009F0A0C6212F287030E040E050E060E01D
:109C600070E080E090E0A0E00E940C8B99F127E08A
:109C70004AE250E06BE270E089E290E00E945C5EB4
:109C80008EE895E30E942D60BC01990F880B990B1B
:109C90000E94B08C20E030E048EC52E40E94FC8B43
:109CA0009F938F937F936F938CEB96E09F938F930B
:109CB0001F9287E78F93CE018A0D9B1D03969F937A
:109CC0008F930E948294A80EB91E0FB6F894DEBF3F
:109CD0000FBECDBF212F207130E040E050E060E0AA
:109CE00070E080E090E0A0E00E940C8BE9F126E0BB
:109CF0004AE250E06BE270E089E290E00E945C5E34
:109D000081E090E00E94741180939B1381E09DE1BB
:109D10000E942D60BC01990F880B990B0E94B08C9A
:109D200020E030E048EC52E40E94FC8B9F938F933C
:109D30007F936F9386EC96E09F938F931F9287E7B4
:109D40008F93C501029621E030E02C0F3D1F820F5A
:109D5000931F9F938F930E948294A80EB91E0FB6F3
:109D6000F894DEBF0FBECDBFC257DF4F2881CE585B
:109D7000D04030E040E050E060E070E080E090E013
:109D8000A0E00E940C8B01F10E9430119F938F93F1
:109D90007F936F9381ED96E09F938F931F9287E758
:109DA0008F93C5010296A1E0B0E0AC0FBD1F8A0FF2
:109DB0009B1F9F938F930E948294A80EB91E0FB68B
:109DC000F894DEBF0FBECDBF212F207430E040E0FD
:109DD00050E060E070E080E090E0A0E00E940C8B3A
:109DE00031F18091CA308F938091C9308F938091E7
:109DF000C8308F938091C7308F938FED96E09F93FB
:109E00008F931F9287E78F93C501029621E030E080
:109E10002C0F3D1F820F931F9F938F930E9482945C
:109E2000A80EB91E0FB6F894DEBF0FBECDBF212F0E
:109E3000207830E040E050E060E070E080E090E0CA
:109E4000A0E00E940C8B41F1F894809174359091C0
:109E50007535A0917635B09177357894BF93AF93EF
:109E60009F938F938DEE96E09F938F931F9287E73A
:109E70008F93C5010296A1E0B0E0AC0FBD1F8A0F21
:109E80009B1F9F938F930E948294A80EB91E0FB6BA
:109E9000F894DEBF0FBECDBF20E0302F317040E020
:109EA00050E060E070E080E090E0A0E00E940C8B69
:109EB00009F082C520E0302F327040E050E060E0D1
:109EC00070E080E090E0A0E00E940C8B09F0F2C509
:109ED00020E0302F347040E050E060E070E080E03F
:109EE00090E0A0E00E940C8B09F015C620E0302F16
:109EF000387040E050E060E070E080E090E0A0E08A
:109F00000E940C8B09F036C620E0302F307140E003
:109F100050E060E070E080E090E0A0E00E940C8BF8
:109F200009F0A6C620E0302F307240E050E060E03B
:109F300070E080E090E0A0E00E940C8B09F0C8C6C1
:109F400020E030E040E050E0CC56DF4F6881C4595B
:109F5000D040647070E080E090E0A0E00E940C8B44
:109F600009F0E4C620E0C856DF4F3881C859D04018
:109F700040E050E060E070E080E090E0A0E00E940F
:109F80000C8B09F040C720E0C756DF4F3881C95914
:109F9000D04040E050E060E070E080E090E0A0E081
:109FA0000E940C8B09F05DC7CE56DF4F5881C25915
:109FB000D0405170952E20E030E0452F50E060E019
:109FC00070E080E090E0A0E00E940C8B09F077C781
:109FD00020E030E0CE56DF4F4881C259D040427079
:109FE00050E060E070E080E090E0A0E00E940C8B28
:109FF00009F098C720E030E0C657DF4F4881CA58C3
:10A00000D04050E060E070E080E090E0A0E00E948E
:10A010000C8B09F0BAC720E030E040E050E0CC56AD
:10A02000DF4F6881C459D040687070E080E090E0F4
:10A03000A0E00E940C8B09F0D2C720E030E040E0A5
:10A0400050E0CC56DF4F6881C459D040607170E059
:10A0500080E090E0A0E00E940C8B09F0ECC720E0CB
:10A0600030E0CE56DF4F4881C259D040487050E0B2
:10A0700060E070E080E090E0A0E00E940C8B11F0C6
:10A080000C94475820E030E0CE56DF4F4881C2594B
:10A09000D040407150E060E070E080E090E0A0E0EF
:10A0A0000E940C8B11F00C947A5820E030E0CE56D0
:10A0B000DF4F4881C259D040407250E060E070E00C
:10A0C00080E090E0A0E00E940C8B11F00C94AD5861
:10A0D00020E030E0CE56DF4F4881C259D040407476
:10A0E00050E060E070E080E090E0A0E00E940C8B27
:10A0F00011F00C94E058CE56DF4FF881C259D04091
:10A10000F0787F2E20E030E04F2F50E060E070E0EC
:10A1100080E090E0A0E00E940C8B11F00C941359A9
:10A12000CD56DF4F2881C359D0402170622E20E0E8
:10A1300030E040E0562D60E070E080E090E0A0E08C
:10A140000E940C8B11F40C94945B8091C52C82FDC1
:10A1500002C00C945B5921E046E061E083E00E947C
:10A16000BC1920E030E0472D50E060E070E080E076
:10A1700090E0A0E00E940C8B11F40C945B5980914C
:10A18000C52C82FF02C00C94205920E030E040E052
:10A19000CD56DF4F5881C359D040527060E070E017
:10A1A00080E090E0A0E00E940C8B11F00C9490599C
:10A1B00020E030E040E0CD56DF4F5881C359D04019
:10A1C000547060E070E080E090E0A0E00E940C8BB2
:10A1D00011F00C94C35920E030E040E0CD56DF4F41
:10A1E0005881C359D040507160E070E080E090E049
:10A1F000A0E00E940C8B11F00C94F65920E030E0A6
:10A2000040E0CD56DF4F5881C359D040507260E0D6
:10A2100070E080E090E0A0E00E940C8B11F00C94C4
:10A22000355A20E030E040E0CD56DF4F5881C35929
:10A23000D040507460E070E080E090E0A0E00E94C8
:10A240000C8B11F00C94745A20E030E040E0CD56B5
:10A25000DF4F5881C359D040587060E070E080E013
:10A2600090E0A0E00E940C8B11F00C94B35A20E017
:10A2700030E040E0C656DF4F5881CA59D04060E018
:10A2800070E080E090E0A0E00E940C8B11F00C9454
:10A29000E45A20E030E0492D50E060E070E080E0DA
:10A2A00090E0A0E00E940C8B11F00C941B5B212F1E
:10A2B000302FCE56DF4F4881C259D040CD56DF4FA8
:10A2C0005881C359D040CC56DF4F6881C459D04023
:10A2D0007D2DC956DF4F8881C759D0409C2DA0E005
:10A2E0000E940C8B11F00C94265B809164028061BB
:10A2F000898380917A0A8A83FE01EA0DFB1D13820D
:10A3000080919F139091A013A091A113B091A213DB
:10A3100085010D5F1F4F80FF0CC01F930F938DE8C9
:10A3200098E09F938F930E9416940F900F900F9038
:10A330000F90B801CE0101960E94CE758091660201
:10A3400082FF0AC024E731E3A801BE016F5F7F4F9F
:10A350008EE692E00E94416180919F139091A0133C
:10A36000A091A113B091A21382FD73980E94EE6890
:10A3700086E89AE00E94E1738091660290916702FC
:10A38000A0916802B091690290FD02C00C945D5BDF
:10A390003FEFA31AB30A0E94E769F82E89E10E94F1
:10A3A000FF698091660290916702A0916802B09166
:10A3B000690290FD02C00C94595B739880917A0AEF
:10A3C0008F5F80937A0A8A83B5016F5F7F4FCE01DA
:10A3D00001960E94CE7586E89AE00E94E17340E003
:10A3E00050E065E88091E1149091E2140E94C17000
:10A3F00085EB91E1CB56DF4FA881B981C559D0409B
:10A400008D939C931EC08EE69AE00E944F6F892B1D
:10A41000C1F00E94EE688091660287FD2B9840E4AF
:10A4200050E060E070E08EE69AE00E94316F8EECC2
:10A4300091E1CB56DF4FE881F981C559D040918336
:10A44000808381E00C94A45BCB56DF4FA881B98157
:10A45000C559D0401D921C9283E00C94A45B6231DC
:10A4600081F78090660290906702A0906802B09099
:10A47000690291FCCDCBF8018081813021F501800A
:10A48000F281E02D108101812281CE56DF4F288399
:10A49000C259D0403381CD56DF4F3883C359D040A5
:10A4A0004481CC56DF4F4883C459D040D580568173
:10A4B000C956DF4F5883C759D040C780E084F18424
:10A4C000212C312C52C08230B9F423803480E12C0D
:10A4D000F12C11E000E0CE56DF4F1882C259D04077
:10A4E000B0E8CD56DF4FB883C359D040CC56DF4FCC
:10A4F0001882C459D04032C08330D1F0843009F082
:10A5000087CBE12CF12C212C312C15E000E0CE562C
:10A51000DF4F1882C259D040CD56DF4F1882C35941
:10A52000D040E2E0CC56DF4FE883C459D04016C09B
:10A53000E12CF12C212C312C15E000E0CE56DF4F20
:10A540001882C259D040CD56DF4F1882C359D0402F
:10A55000F1E0CC56DF4FF883C459D040D12CC95616
:10A56000DF4F1882C759D040C12C4090C73050905F
:10A57000C8306090C9307090CA3020918D023091FF
:10A580008E0240918F0250919002C657DF4F288370
:10A5900039834A835B83CA58D0402DEC3CEC4CE4B1
:10A5A0005EE3C657DF4F688179818A819B81CA58F3
:10A5B000D0400E94198B9B01AC01C301B2010E94E3
:10A5C000D58D87FD0BC0E894A0F88092660290922A
:10A5D0006702A0926802B092690246C0C657DF4F78
:10A5E000288139814A815B81CA58D040C301B201B8
:10A5F0000E94F78B87FF38C08091D3309091D43080
:10A60000A091D530B091D6300196A11DB11D809397
:10A61000D3309093D430A093D530B093D630A0FCF3
:10A62000F7CA6894A0F88092660290926702A0929E
:10A630006802B092690215E400E2CE56DF4F18823C
:10A64000C259D040CD56DF4F1882C359D04034E0B4
:10A65000CC56DF4F3883C459D040D12CC956DF4F78
:10A660001882C759D040C12CCE56DF4F4881C259FD
:10A67000D0404470C657DF4F4883CA58D04020E0CE
:10A6800030E050E060E070E080E090E0A0E00E9408
:10A690000C8B09F08C9A512F5072C257DF4F5883A0
:10A6A000CE58D040252F30E040E050E060E070E030
:10A6B00080E090E0A0E00E940C8B11F00E9430112D
:10A6C000802F8074C856DF4F8883C859D04020E05F
:10A6D000382F40E050E060E070E080E090E0A0E0E3
:10A6E0000E940C8B11F00E945225902F9078C75633
:10A6F000DF4F9883C959D04020E0392F40E050E027
:10A7000060E070E080E090E0A0E00E940C8B51F0EF
:10A710000E94CB106093813570938235809383358E
:10A7200090938435212F217030E040E050E060E0CC
:10A7300070E080E090E0A0E00E940C8BF1F08FE8E8
:10A740009CE19F938F938CE996E09F938F931F9248
:10A7500087E78F93CE0103969F938F930E948294F5
:10A760004C010E94844D0FB6F894DEBF0FBECDBFE2
:10A77000892B09F04DCA540102C0A12CB12C212F04
:10A78000227030E040E050E060E070E080E090E077
:10A79000A0E00E940C8BD1F1C501029664EA76E03C
:10A7A000E1E0F0E0EC0FFD1F8E0F9F1F0E947493FD
:10A7B000F3E0AF0EB11C2EE8622E25E3722E36E7D1
:10A7C000832E33E0932E47E7542ED3018D913D0124
:10A7D0001F928F939F928F921F925F92C501029654
:10A7E000E1E0F0E0EC0FFD1F8E0F9F1F9F938F9312
:10A7F0000E948294A80EB91E0FB6F894DEBF0FBE59
:10A80000CDBF36E9631635E37306F9F6212F2470C0
:10A8100030E040E050E060E070E080E090E0A0E0F8
:10A820000E940C8B09F450C0C501029668EA76E0DC
:10A8300041E050E04C0F5D1F840F951F0E94749300
:10A8400054E0A50EB11C2E018AE7480E511C80E190
:10A85000D2011D928A95E9F728E0A20168E980EB10
:10A860000E9407183201B8E06B0E711C96E7892E22
:10A8700093E0992E27E7F20181912F011F928F9388
:10A880009F928F921F922F93C501029641E050E054
:10A890004C0F5D1F840F951F9F938F93C556DF4FFD
:10A8A0002883CB59D0400E948294A80EB91E0FB6BF
:10A8B000F894DEBF0FBECDBFC556DF4F2881CB5900
:10A8C000D04046145704B9F6CD56DF4F9881C3598E
:10A8D000D0409078C656DF4F9883CA59D04020E0C8
:10A8E00030E040E0592F60E070E080E090E0A0E0D0
:10A8F0000E940C8BE1F480919D1390919E139F9385
:10A900008F938DEA96E09F938F931F9287E78F93A3
:10A91000CE018A0D9B1D03969F938F930E94829474
:10A92000A80EB91E0FB6F894DEBF0FBECDBF20E053
:10A9300030E040E050E0CC56DF4F6881C459D04051
:10A94000617070E080E090E0A0E00E940C8B09F460
:10A950006FC9E3E0F0E0EC0FFD1FEA0DFB1D80E2A4
:10A960008083A50183E090E08A199B09FC01E40F34
:10A97000F51FEC50FF4C20814F5F5F4F222309F4FD
:10A980004AC92081E1E0F0E0EC0FFD1FE40FF51F64
:10A990002283ECCFCE018A0D9B1D64EB76E00396FB
:10A9A0000E947493B7E0AB0EB11CC5010E94844DA8
:10A9B000892B09F02DC94EC9E114F10409F47ACAB2
:10A9C000F89440907435509075356090763570905D
:10A9D000773578948091F91C9091FA1CA091FB1C1A
:10A9E000B091FC1CA3019201281B390B4A0B5B0B95
:10A9F000CA01B9010E94AE8CC257DF4F68837983C8
:10AA00008A839B83CE58D040B70180E090E00E94BB
:10AA1000AE8C9B01AC01C257DF4F688179818A817E
:10AA20009B81CE58D0400E94FC8B4C019F928F930B
:10AA30007F936F9388EF96E09F938F931F9287E7A2
:10AA40008F939E012A0D3B1D2D5F3F4F3F932F9308
:10AA5000C456DF4F6883CC59D040C556DF4F78834A
:10AA6000CB59D0400E948294A80EB91EC456DF4F25
:10AA70006881CC59D040C556DF4F7881CB59D04042
:10AA8000862F972FA82DB92D8093863590938735E3
:10AA9000A0938835B09389354092F91C5092FA1CE6
:10AAA0006092FB1C7092FC1C0FB6F894DEBF0FBEC8
:10AAB000CDBF00CAE114F10409F40ACAF8948091E8
:10AAC000D01C9091D11CA091D21CB091D31C789431
:10AAD0009F938F9380916D028F9380916C028F93DF
:10AAE00085E097E09F938F931F9287E78F93C5012F
:10AAF0000296A1E0B0E0AC0FBD1F8A0F9B1F9F9391
:10AB00008F930E948294A80EB91E0FB6F894DEBFF0
:10AB10000FBECDBFDDC9F89480917835909179351D
:10AB2000A0917A35B0917B357894BF93AF939F9382
:10AB30008F9385E197E09F938F931F9287E78F9381
:10AB4000C501029621E030E02C0F3D1F820F931FBC
:10AB50009F938F930E948294A80EB91EC5010E94F4
:10AB6000844D0FB6F894DEBF0FBECDBF892B09F020
:10AB70004FC8BCC9E114F10409F4C6C9F894409067
:10AB800078355090793560907A3570907B3578942F
:10AB90008091FD1C9091FE1CA091FF1CB091001DA6
:10ABA000A3019201281B390B4A0B5B0BCA01B901A7
:10ABB0000E94AE8CC257DF4F688379838A839B8360
:10ABC000CE58D040B70180E090E00E94AE8C9B014F
:10ABD000AC01C257DF4F688179818A819B81CE5851
:10ABE000D0400E94FC8B4C019F928F937F936F9378
:10ABF00080E297E09F938F931F9287E78F939E0148
:10AC00002A0D3B1D2D5F3F4F3F932F93C456DF4FBF
:10AC10006883CC59D040C556DF4F7883CB59D0409C
:10AC20000E948294A80EB91EC456DF4F6881CC5989
:10AC3000D040C556DF4F7881CB59D040862F972F13
:10AC4000A82DB92D80938A3590938B35A0938C35A0
:10AC5000B0938D354092FD1C5092FE1C6092FF1CFB
:10AC60007092001D0FB6F894DEBF0FBECDBF4CC969
:10AC7000EF2809F457C9F8948091D41C9091D51C01
:10AC8000A091D61CB091D71C78949F938F938091FC
:10AC90006B028F9380916A028F938DE297E09F936E
:10ACA0008F931F9287E78F93C5010296A1E0B0E0D2
:10ACB000AC0FBD1F8A0F9B1F9F938F930E9482949E
:10ACC000A80EB91E0FB6F894DEBF0FBECDBF2AC9BD
:10ACD0008091CB309091CC30A091CD30B091CE30DE
:10ACE000BF93AF939F938F938DE397E09F938F9341
:10ACF0001F9287E78F93C501029621E030E02C0F69
:10AD00003D1F820F931F9F938F930E948294A80EE2
:10AD1000B91EC5010E94844D0FB6F894DEBF0FBE68
:10AD2000CDBF892B11F00C94084E0AC98091D63002
:10AD30008F938091D5308F938091D4308F93809171
:10AD4000D3308F938091D2308F938091D1308F9375
:10AD50008091D0308F938091CF308F9388E497E0AB
:10AD60009F938F931F9287E7982E9F92C50102961B
:10AD7000A1E0B0E0AC0FBD1F8A0F9B1F9F938F9384
:10AD80000E948294A80EB91EC5010E94844D0FB680
:10AD9000F894DEBF0FBECDBF892B11F00C94084E86
:10ADA0008091C52C9091C62C90FFDCC88091DA3040
:10ADB0008F938091D9308F938091D8308F938091E9
:10ADC000D7308F938CE697E09F938F931F929F923B
:10ADD000C501029621E030E02C0F3D1F820F931F2A
:10ADE0009F938F930E948294A80EB91EC5010E9462
:10ADF000844D0FB6F894DEBF0FBECDBF892B11F086
:10AE00000C94084EAFC88091BC288F938091BB28CA
:10AE10008F938091BA288F938091B9288F938EE772
:10AE200097E09F938F931F9287E78F93C5010296B8
:10AE3000A1E0B0E0AC0FBD1F8A0F9B1F9F938F93C3
:10AE40000E948294A80EB91EC5010E94844D0FB6BF
:10AE5000F894DEBF0FBECDBF892B11F00C94084EC5
:10AE600092C8809184358F93809183358F938091A0
:10AE700082358F93809181358F9389E897E09F93F6
:10AE80008F931F9287E78F93C501029621E030E0F0
:10AE90002C0F3D1F820F931F9F938F930E948294CC
:10AEA000A80EB91EC5010E94844D0FB6F894DEBFEE
:10AEB0000FBECDBF892B11F00C94084E75C881E0F0
:10AEC0000E947D1020918502309186024091870278
:10AED000509188020E94A88E9F938F937F936F93C7
:10AEE00086E997E09F938F931F9287E78F93C50121
:10AEF0000296A1E0B0E0AC0FBD1F8A0F9B1F9F938D
:10AF00008F930E948294A80EB91EC5010E94844DA1
:10AF10000FB6F894DEBF0FBECDBF892B11F00C9495
:10AF2000084E56C882E00E947D1020918102309127
:10AF3000820240918302509184020E94A88E9F93C6
:10AF40008F937F936F9383EA97E09F938F931F92E2
:10AF500087E78F93C501029621E030E02C0F3D1F5B
:10AF6000820F931F9F938F930E948294A80EB91E05
:10AF7000C5010E94844D0FB6F894DEBF0FBECDBF51
:10AF8000892B11F00C94084E35C883E00E947D1087
:10AF90009F938F937F936F9380EB97E09F938F9313
:10AFA0001F9287E78F93C5010296A1E0B0E0AC0F36
:10AFB000BD1F8A0F9B1F9F938F930E948294A80EA0
:10AFC000B91E8C98C5010E94844D0FB6F894DEBF5F
:10AFD0000FBECDBF892B11F00C94084E1CC82999C7
:10AFE00003C08CE195E002C089E195E09F938F93C7
:10AFF0008DEB97E09F938F931F9287E78F93C50107
:10B00000029621E030E02C0F3D1F820F931F9F938B
:10B010008F930E948294A80EB91EC5010E94844D90
:10B020000FB6F894DEBF0FBECDBF892B11F00C9484
:10B03000084E0C941D502A9903C08CE195E002C083
:10B0400089E195E09F938F9385EC97E09F938F9391
:10B050001F9287E78F93C5010296A1E0B0E0AC0F85
:10B06000BD1F8A0F9B1F9F938F930E948294A80EEF
:10B07000B91EC5010E94844D0FB6F894DEBF0FBE05
:10B08000CDBF892B11F00C94084E0C942F50809159
:10B09000C52C87FD02C00C94425021E042E161E0E2
:10B0A00080ED0E947E629F938F937F936F938DECD0
:10B0B00097E09F938F931F9287E78F93C501029626
:10B0C00021E030E02C0F3D1F820F931F9F938F9341
:10B0D0000E948294A80EB91EC5010E94844D0FB62D
:10B0E000F894DEBF0FBECDBF892B11F00C94084E33
:10B0F0000C9442508091C52C87FD02C00C94555091
:10B1000021E042E162E080ED0E947E629F938F9396
:10B110007F936F938BED97E09F938F931F9287E7B9
:10B120008F93C5010296A1E0B0E0AC0FBD1F8A0F5E
:10B130009B1F9F938F930E948294A80EB91EC501F6
:10B140000E94844D0FB6F894DEBF0FBECDBF892B91
:10B1500011F00C94084E0C9455508091C52C87FD2D
:10B1600002C00C94685021E042E163E080ED0E944F
:10B170007E629F938F937F936F9389EE97E09F9367
:10B180008F931F9287E78F93C501029621E030E0ED
:10B190002C0F3D1F820F931F9F938F930E948294C9
:10B1A000A80EB91EC5010E94844D0FB6F894DEBFEB
:10B1B0000FBECDBF892B11F00C94084E0C94685033
:10B1C0008091C52C87FD02C00C947B5021E042E1A8
:10B1D00064E080ED0E947E629F938F937F936F93D4
:10B1E00087EF97E09F938F931F9287E78F93C50117
:10B1F0000296A1E0B0E0AC0FBD1F8A0F9B1F9F938A
:10B200008F930E948294A80EB91EC5010E94844D9E
:10B210000FB6F894DEBF0FBECDBF892B11F00C9492
:10B22000084E0C947B508091C52C82FD02C00C947A
:10B23000905046E061E083E00E94BC190C9490506D
:10B240008091A81D8F938091A71D8F938091A61D3B
:10B250008F938091A51D8F9385E098E09F938F93A6
:10B260001F9287E78F93C501029641E050E04C0F93
:10B270005D1F840F951F9F938F930E948294A80E49
:10B28000B91EC5010E94844D0FB6F894DEBF0FBEF3
:10B29000CDBF892B11F00C94084E20E030E040E047
:10B2A000562D60E070E080E090E0A0E00E940C8B02
:10B2B00011F40C94C5508091C52C82FD02C00C94F1
:10B2C000C5508091AC1D8F938091AB1D8F93809161
:10B2D000AA1D8F938091A91D8F938DE098E09F9375
:10B2E0008F931F9287E78F93C5010296E1E0F0E00C
:10B2F000EC0FFD1F8E0F9F1F9F938F930E948294D0
:10B30000A80EB91EC5010E94844D0FB6F894DEBF89
:10B310000FBECDBF892B11F00C94084E0C94C55074
:10B320008091C52C9091C62C90FD02C00C94D850F1
:10B3300080E090E00E94CA249F938F937F936F9345
:10B3400088E198E09F938F931F9287E78F93C501C1
:10B35000029641E050E04C0F5D1F840F951F9F93B4
:10B360008F930E948294A80EB91EC5010E94844D3D
:10B370000FB6F894DEBF0FBECDBF892B11F00C9431
:10B38000084E0C94D8508091C52C9091C62C90FDFD
:10B3900002C00C94EB5081E090E00E94CA249F937D
:10B3A0008F937F936F9388E298E09F938F931F9280
:10B3B00087E78F93C5010296E1E0F0E0EC0FFD1FF7
:10B3C0008E0F9F1F9F938F930E948294A80EB91E89
:10B3D000C5010E94844D0FB6F894DEBF0FBECDBFED
:10B3E000892B11F00C94084E0C94EB508091C52CD5
:10B3F0009091C62C90FD02C00C94FE5081E090E02C
:10B400000E94CA242B013C0180E090E00E94CA24E3
:10B410009B01AC01C301B2010E94C7229F938F938D
:10B420007F936F9389E398E09F938F931F9287E7B1
:10B430008F93C501029641E050E04C0F5D1F840FD1
:10B44000951F9F938F930E948294A80EB91EC501E9
:10B450000E94844D0FB6F894DEBF0FBECDBF892B7E
:10B4600011F00C94084E0C94FE508091C52C9091D4
:10B47000C62C90FD02C00C94115181E090E00E9416
:10B48000CA242B013C0180E090E00E94CA249B0169
:10B49000AC01C301B2010E9428239F938F937F9335
:10B4A0006F9384E498E09F938F931F9287E78F9325
:10B4B000C5010296E1E0F0E0EC0FFD1F8E0F9F1F2B
:10B4C0009F938F930E948294A80EB91EC5010E947B
:10B4D000844D0FB6F894DEBF0FBECDBF892B11F09F
:10B4E0000C94084E0C9411518091C52C9091C62C4F
:10B4F00090FD02C00C94245181E090E00E94CA2487
:10B500002B013C0180E090E00E94CA249B01AC0129
:10B51000C301B2010E9489239F938F937F936F93FE
:10B5200082E598E09F938F931F9287E78F93C501E1
:10B53000029641E050E04C0F5D1F840F951F9F93D2
:10B540008F930E948294A80EB91EC5010E94844D5B
:10B550000FB6F894DEBF0FBECDBF892B11F00C944F
:10B56000084E0C9424518091C52C9091C62C91FDCD
:10B5700002C00C9437510E94211E9F938F937F939A
:10B580006F9385E698E09F938F931F9287E78F9341
:10B59000C5010296E1E0F0E0EC0FFD1F8E0F9F1F4A
:10B5A0009F938F930E948294A80EB91EC5010E949A
:10B5B000844D0FB6F894DEBF0FBECDBF892B11F0BE
:10B5C0000C94084E0C943751D10116968C91169715
:10B5D0001F928F9315968C9115971F928F931396A8
:10B5E0008C9113971F928F9312968C911F928F9329
:10B5F00086E798E09F938F931F9287E78F93C5010B
:10B600000296E1E0F0E0EC0FFD1F8E0F9F1F9F936D
:10B610008F930E948294A80EB91EC5010E94844D8A
:10B620000FB6F894DEBF0FBECDBF892B11F00C947E
:10B63000084E0C944951779A80919F139091A013D2
:10B64000A091A113B091A21392FD749A80919F13BF
:10B650009091A013A091A113B091A21382FD0CC0F0
:10B660008091660280FD08C081FD02C00C94755176
:10B670001D9902C00C94755140E050E060E070E00C
:10B68000CE0101960E94E80E8091AE1D90E02091BF
:10B690009513309196138217930710F40C947551FB
:10B6A00040E050E062E180E192E00E94C1700C94C1
:10B6B00075518F2D0E94FF69739A80919D1390910F
:10B6C0009E13892B11F00E94246880917A0A8F5F63
:10B6D00080937A0A80919F139091A013A091A11357
:10B6E000B091A21382FD02C00C94084E739A0C9480
:10B6F000084E653811F00C942152A12CB12C0C94F9
:10B70000D1518EE69AE00E944F6F892B11F40C9470
:10B7100021520E9424688091660287FD02C00C9429
:10B72000084E2B9A0C94084E20E030E0472D50E054
:10B7300060E070E080E090E0A0E00E940C8B11F0EF
:10B740000C94BF500C94C550C456DF4F0FB6F894FC
:10B75000DEBF0FBECDBFDF91CF911F910F91FF9044
:10B76000EF90DF90CF90BF90AF909F908F907F90A1
:10B770006F905F904F903F902F9008950C94777347
:10B780004F925F926F927F929F92AF92BF92CF92B1
:10B79000DF92EF92FF920F931F93CF93DF93CDB77A
:10B7A000DEB760970FB6F894DEBF0FBECDBF5B016A
:10B7B0000E94E769E82FF0E0EE0FFF1FEE53F34E13
:10B7C0008081918101969183808380919F139091D4
:10B7D000A013A091A113B091A21381FD7498409081
:10B7E00066025090670260906802709069020E9441
:10B7F0002A756C01FC018081982F92959F70913081
:10B8000099F48F7051F48091A61C9091A71C019619
:10B810009093A71C8093A61C3CC1B50183EA97E3D3
:10B820000E94E374892B51F08091A41C9091A51C77
:10B8300001969093A51C8093A41C2BC1D301C20137
:10B840003EE0B695A795979587953A95D1F7F82F4D
:10B85000F1709F2E81E99AE00E949A717C01892BF8
:10B8600009F44BC0B501C70102960E94E374892B0D
:10B8700009F43FC0870127E93EE040E054E660E07C
:10B8800070E0C7010F960E94CF6DF6019181F7011C
:10B890008481981321C082858F5F82878091A21C4A
:10B8A0009091A31C01969093A31C8093A21C84E00A
:10B8B0000E941A76F701208530E02817390708F032
:10B8C00078C184E00E941A76F7018087F6018081B2
:10B8D0008F70F7018187DDC0F701128684E00E9436
:10B8E0001A76F7018087F60180818F70F7018187D2
:10B8F00061C1C7010E94FF71B1CF88E092E00E9450
:10B9000026727C01892B09F4C4C0B501C7010296D7
:10B910000E94DC74F60181818150F701848380E00C
:10B9200091E0A0E0B0E083879487A587B687128670
:10B9300084E00E941A76F7018087F60180818F707B
:10B94000F7018187B70181E99AE00E94D9718701E7
:10B9500027E93EE040E054E660E070E0C7010F9662
:10B960000E94CF6D11E0F6018181F7018483F60119
:10B9700080818F70F701878384E00E941A76F70137
:10B98000858383E00E941A76F701868387818F3052
:10B9900009F010E0F6014180F7018481481A512C2A
:10B9A000612C712C86E0440C551C661C771C8A9512
:10B9B000D1F72385348545855685A0ECB0E00E94FB
:10B9C0004089BB27A92F982F872F480E591E6A1E22
:10B9D0007B1E4386548665867686A501B701C6011F
:10B9E0000E94E80E8091AE1D90E020919513309159
:10B9F00096138217930738F040E050E062E180E14F
:10BA000092E00E94C17080919513909196130297D5
:10BA100008F44BC08091C52C86FF2AC00E94CD61DE
:10BA2000C60105960E949961F60181811F928F934C
:10BA3000F70186811F928F9385811F928F938EE9E4
:10BA400098E09F938F931F9280E18F93CE01019690
:10BA50005C019F938F930E94829482E00E94B36165
:10BA6000C5010E9499610FB6F894DEBF0FBECDBF2D
:10BA70008091660290916702A0916802B09169027C
:10BA800097FD4DC08091951390919613029708F4FD
:10BA90007AC080919F139091A013A091A113B091AF
:10BAA000A21381FF89C0749A87C080916602909129
:10BAB0006702A0916802B091690296FFABCF99200E
:10BAC00009F4A8CFF6018081982F9F709230E8F09A
:10BAD0009150807F892B808386E89AE00E94BE5B2C
:10BAE0008091A01C9091A11C01969093A11C809321
:10BAF000A01C80919F139091A013A091A113B091CD
:10BB0000A21396FF87CF739885CF8091A61C909142
:10BB1000A71C01969093A71C8093A61C7BCF8FE84F
:10BB20009CE120918F1C222309F4ACCF9F938F932B
:10BB300081EB98E09F938F93CE0101963C019F93F8
:10BB40008F930E94BF945C01B301C60102960E94CC
:10BB500095930F900F900F900F900F900F9000976C
:10BB600009F490CFEFEFAE1ABE0A8A0D9B1DAC010F
:10BB70000196FA0120812032D1F362E18AE192E05C
:10BB80000E94C1707FCF112309F483CF82E080939C
:10BB9000E0301092E2301092E130F092E430E09226
:10BBA000E33040EE50E362E182E492E00E94C17033
:10BBB00070CF912C10E0D7CE60960FB6F894DEBF10
:10BBC0000FBECDBFDF91CF911F910F91FF90EF90EE
:10BBD000DF90CF90BF90AF909F907F906F905F90DD
:10BBE0004F9008958115910511F00197F1F708958F
:10BBF000E091A135F091A23590818091A035892303
:10BC00000895E0919E35F0919F3590818091A03507
:10BC1000892B8083E091A335F091A43590818091A8
:10BC2000A035892B808308951F93CF93DF93E091F4
:10BC30009E35F0919F3590818091A0358095892324
:10BC40008083E091A335F091A43590818091A03557
:10BC5000892B80838FE897E00E94F25D1FB7F894EC
:10BC6000E091A335F091A43590818091A035809525
:10BC70008923808389E091E00E94F25DE091A13503
:10BC8000F091A235D081C091A0351FBF789485E88E
:10BC900096E00E94F25DE091A135F091A23580819D
:10BCA0009091A035982319F08D2F8C2301C081E04D
:10BCB000DF91CF911F9108955093A4354093A33500
:10BCC00070939F3560939E359093A2358093A135F4
:10BCD00081E001C0880F2A95EAF78093A0350C9483
:10BCE000145ECF93DF93C82FDFB7F894E091A335AC
:10BCF000F091A43590818091A035892B808387E0D5
:10BD000090E00E94F25DCC2351F0E091A335F091D8
:10BD1000A43590818091A03580958923808384E328
:10BD200090E00E94F25DE091A135F091A235908102
:10BD30008091A035892309F4C0E085EB90E00E9452
:10BD4000F25DE091A335F091A43590818091A0350A
:10BD5000809589238083DFBF88E790E00E94F25DB1
:10BD60008C2FDF91CF910895CF93DF93C82FD8E028
:10BD70008C2F81700E94715EC6958111C068D15070
:10BD8000B9F78C2FDF91CF9108958FEF0C94B45EAB
:10BD9000DF92EF92FF920F931F93CF93DF93E82EE2
:10BDA0008B010E94145E811135C080EF0E94B45E49
:10BDB000D0E0C0E488EFD82EDC0E81E00E94715EF6
:10BDC000F82E81E00E94715E882319F0FF2071F047
:10BDD00023C0F1100BC0CE1530F0F801808180FF38
:10BDE00005C0EC1619F0DC2FFF24F3948F2D0E9470
:10BDF000715EF80190819695FF2011F09068F8012E
:10BE00009083C150CD11D9CF0F5F1F4FC111D2CF39
:10BE10008D2F03C08FEF01C08EEFDF91CF911F9167
:10BE20000F91FF90EF90DF900895EF92FF921F9394
:10BE3000CF93DF93182FEB010E94145E209771F0CF
:10BE400085E50E94B45E7E0188E0E80EF11C8991D0
:10BE50000E94B45ECE15DF05D1F703C08CEC0E94C2
:10BE6000B45E812FDF91CF911F91FF90EF900C94E2
:10BE7000B45E0F931F93CF93DF93DB01EC91119688
:10BE80009C911197F0E0F92B803179F4EE7F63E01B
:10BE9000EE0FFF1F6A95E1F716969C9116976CE0DE
:10BEA00070E0691B7109E60FF71FF7FF07C091E00B
:10BEB000EA019883F195E195F10902C0EA0118823F
:10BEC000883279F414968C91982F9076903649F0B8
:10BED00086FF02C0EE7F05C085FF02C0EC7F01C077
:10BEE000E87FCF0144E0969587954A95E1F7D9011F
:10BEF0008C93EF70E801E88380E0DF91CF911F9190
:10BF00000F9108950F931F93CF93DF93EC018B0153
:10BF1000B80188810E94C85E88839FEF980F9D3F7B
:10BF200030F4F8019081983211F0903189F7DF9167
:10BF3000CF911F910F910895CF93DF93EC010E9451
:10BF4000145EBE0184EB0E94155F81E00E94715E69
:10BF5000C82F0E94145E81E0C11101C080E0DF9112
:10BF6000CF9108951F93CF93DF931F921F92CDB768
:10BF7000DEB7182F69837A830E94145E0E94F85DF1
:10BF800069817A81882341F084E40E94155F113031
:10BF900029F00E94015E02C082E001C080E00F90A3
:10BFA0000F90DF91CF911F9108955F926F927F92D2
:10BFB0008F929F92AF92BF92CF92DF92EF92FF92B9
:10BFC0000F931F93CF93DF93CDB7DEB729970FB6AB
:10BFD000F894DEBF0FBECDBF5C014B013A01890171
:10BFE0000E94145EB5018EEB0E94155FCE01019692
:10BFF0007C016C0199E0592E5E0C0E94C55EF60131
:10C0000081936F015E12F9CF69E070E0C7010E9471
:10C01000B979D82E811108C09301A401B701F501A7
:10C0200080810E94395F02C083E0D82E8D2D299631
:10C030000FB6F894DEBF0FBECDBFDF91CF911F9139
:10C040000F91FF90EF90DF90CF90BF90AF909F90B7
:10C050008F907F906F905F9008950F931F93CF9371
:10C06000DF93CDB7DEB72B970FB6F894DEBF0FBEC8
:10C07000CDBF182F092F682F792F88E0810F0E94DC
:10C08000B25F882319F084E391E243C06CE872E860
:10C090008EE190E00E9494609E01275F3F4FAE01C9
:10C0A000465F5F4FBE01655F7F4F812F902F0E94DB
:10C0B000D55F8111E8CF88E0E1EEF2E0DE01119674
:10C0C00001900D928A95E1F7298541E752E0249F7E
:10C0D000C001259F900D112464E670E00E94C58880
:10C0E0008A8594E6899F600D711D1124FE013196A9
:10C0F00088E08E0F9191291303C06F5F7F4F02C0BC
:10C100008E13F8CF8B85882319F07195619571098D
:10C11000CB012B960FB6F894DEBF0FBECDBFDF91DB
:10C12000CF911F910F910895DC01CB0181159105ED
:10C13000A105B10529F081509040A040B040D9F749
:10C1400008959B01AC011092B90060E074E284EFA5
:10C1500090E00E94D988DA01C9014097A109B1098C
:10C16000B695A795979587958093B800089594EA1A
:10C170009093BC0040EA56E861E070E09091BC000A
:10C1800097FD07C04150510961097109B9F781E074
:10C1900008959091B900987F983011F09031B9F7D7
:10C1A0008093BB0084E88093BC0080EA96E8A1E01D
:10C1B000B0E02091BC0027FD05C00197A109B1099D
:10C1C000C1F7E5CF8091B900887F883111F08034C4
:10C1D000F1F680E0089524EA34E844E92093BC00B5
:10C1E0009091BC0097FFFCCF9091B900987F983058
:10C1F00011F0903199F78093BB003093BC0090917F
:10C20000BC0097FFFCCF9091B900987F903211F05D
:10C21000983539F44093BC009091BC0094FDFCCF5C
:10C22000DDCF08950C94B76084E98093BC008091C1
:10C23000BC0084FDFCCF08958093BB0084E880930C
:10C24000BC008091BC0087FFFCCF9091B900987F23
:10C2500081E0983209F480E0089584EC8093BC007A
:10C260008091BC0087FFFCCF8091BB00089584E8DB
:10C270008093BC008091BC0087FFFCCF8091BB0005
:10C280000895CF93DF93FC017096EC01A991CE0144
:10C29000A0933F01CE17DF07C1F780913C018F7D4E
:10C2A00080933C0180913C01877F80933C01DB01BE
:10C2B0005096FB01819180933E01EA17FB07D1F76D
:10C2C00080913C01806880933C0180913D0180FF1A
:10C2D000FCCF4051510980913C01806280933C0128
:10C2E00080913C01877F80933C01141615069CF4D5
:10C2F000FB01819180933E01EA17FB07D1F7809102
:10C300003C01806880933C0180913D0180FFFCCF1F
:10C3100040515109EACFF901C901409620913E01EF
:10C320002193E817F907D1F781E090E0DF91CF91F1
:10C3300008950F931F93CF93DF93EC018CE70E9436
:10C34000EB608CE70E941C618E01005F1F4F89919A
:10C350000E941C61C017D107D1F7DF91CF911F91C7
:10C360000F910C941461813019F440E050E002C048
:10C3700040EC50E060E070E08CE790E00C94EF1748
:10C38000813019F44EE050E002C048E050E060E037
:10C3900070E08CE790E00C94EF1741E050E060E033
:10C3A00070E08CE790E00E94EF1764ED74E180E0AC
:10C3B00090E00C94946048E350E060E070E08CE71B
:10C3C00090E00E94EF1749E350E060E070E08CE7F6
:10C3D00090E00E94EF1744E150E060E070E08CE7ED
:10C3E00090E00E94EF1748E750E060E070E08CE7D3
:10C3F00090E00E94EF174EE550E060E070E08CE7BF
:10C4000090E00E94EF174DE650E060E070E08CE7AE
:10C4100090E00E94EF1768E374E38CE090E00E94E4
:10C4200094604CE050E060E070E08CE790E00E94A7
:10C43000EF1741E050E060E070E08CE790E00E9490
:10C44000EF1746E050E060E070E08CE790E00E947B
:10C45000EF1764ED74E180E090E00C949460CF936A
:10C46000DF93CDB7DEB7A2970FB6F894DEBF0FBE4D
:10C47000CDBF81E1E0E4F9E0DE01529601900D923A
:10C480008A95E1F781E1E1E5F9E0DE01119601909D
:10C490000D928A95E1F70E94DB61CE0142960E94DF
:10C4A000996182E00E94B36164ED74E180E090E004
:10C4B0000E949460CE0101960E94996160E27CE541
:10C4C00081E590E00E94946080E00E94C06160E29B
:10C4D0007CE581E590E00E9494604EE050E060E0F1
:10C4E00070E08CE790E00E94EF17A2960FB6F894E8
:10C4F000DEBF0FBECDBFDF91CF910895CF92DF9207
:10C50000EF92FF920F931F93CF93DF9300D0CDB79D
:10C51000DEB7042F122F213061F0223031F02430A9
:10C5200031F0283031F493E005C091E003C092E08F
:10C5300001C090E0E82FF0E08160F82E0C3009F4A3
:10C54000E0C00E3011F49460DCC0003111F498604A
:10C55000D8C0023109F0D5C0613009F4B7C09C6081
:10C56000623011F4906207C0633011F4906403C02C
:10C57000643009F490669068692F70E023E030E041
:10C58000AE014F5F5F4FCF010E94071862E174E375
:10C5900080E090E00E9494608F2D0E94B7600E941E
:10C5A0002D6189830E942D618A83023119F40E94D2
:10C5B0002D618B830E942D6187FDF1CF0E94376131
:10C5C0000E94146162E174E380E090E00E94946054
:10C5D0008F2D0E94B7600E942D6189830E942D617A
:10C5E0008A83023119F40E9437618B830E9437617C
:10C5F0000E94146169812A81023139F5862F90E009
:10C60000A0E0B0E04B81DC019927882730E0322F91
:10C610002227820F931FA11DB11D61FF09C0840F46
:10C62000911DA11DB11DBC01CD018C6F9F6F06C076
:10C63000BC01CD01640F711D811D911D0E94B08C44
:10C6400020E83FEF4FEF57E41FC070E0762F6627DA
:10C65000620F711D072E000C880B990B0E94B08C85
:10C660000C3029F420E030EE4FEF54E40DC00E30D2
:10C6700029F420E038EF4FEF55E406C0003131F4E3
:10C6800020E03EEF4FEF56E40E94FC8B2FE632E1B4
:10C6900043E050E40E94A88E6B017C01612F70E0A2
:10C6A00080E090E00E94B08C9B01AC01C701B60114
:10C6B0000E94FC8B0F900F900F90DF91CF911F91F4
:10C6C0000F91FF90EF90DF90CF9008959C68692FB5
:10C6D00070E023E030E0AE014F5F5F4FCF010E947A
:10C6E000071862E174E380E090E00E9494608F2D6F
:10C6F0000E94B7600E942D6189830E942D618A8308
:10C7000056CF613009F02CCF9068692F70E023E09C
:10C7100030E0AE014F5F5F4FCF010E94071862E12A
:10C7200074E380E090E00E9494608F2D0E94B760D7
:10C730000E942D6189830E942D618A833BCFCF9314
:10C74000E6E4F1E0208190818081C081C295C695A8
:10C75000C695C370207CC20F969596959073C90FAD
:10C7600082958C70C80F1F92CF9382E293E19F93C2
:10C770008F930E942A940F900F900F900F908C2F00
:10C78000CF9108951F93CF93DF9346E069E180E056
:10C790000E94AA6680E00E94FF660E948D6504B632
:10C7A00000FE08C081E193E19F938F930E942A9439
:10C7B0000F900F9004B601FE08C080E093E19F93B4
:10C7C0008F930E942A940F900F9004B602FE08C027
:10C7D0008FEE92E19F938F930E942A940F900F9077
:10C7E00004B603FE08C08EED92E19F938F930E94E2
:10C7F0002A940F900F9004B604FE08C081ED92E1D8
:10C800009F938F930E942A940F900F9082E699E055
:10C810009F938F9386EB92E19F938F930E942A942C
:10C820000E941C710E944D7060E070E085EB92E008
:10C830000E94EF700E94C36DE091A609F091A709D4
:10C8400019950E949F6390E00E9430670E94F474E3
:10C8500082E08093A3378093A4370E94856543EAE2
:10C8600057E3BC018DEC9BEA0E94046A0E94F564C8
:10C870000E94EA690E9489650E94116B0E943376CA
:10C88000E0911C0AF0911D0A1995E091F409F091CC
:10C89000F5091995E091E609F091E70919950E94CB
:10C8A000136B182FC091280AD091290AFE011995FF
:10C8B0000F900F900F900F90892B49F0FE01199562
:10C8C000BC0180E890E00E94B188EB0102C0C0E8A2
:10C8D000D0E00E94E7691F921F93DF93CF931F92CE
:10C8E0008F9380911B0A8F9380911A0A8F93809166
:10C8F000F3098F938091F2098F9384E892E19F93DB
:10C900008F930E942A9487E792E19F938F930E94CE
:10C910002A9486E692E19F938F930E942A9460E086
:10C9200070E087ED92E00E94EF708EE299E00E9445
:10C930004E6D8EE592E19F938F930E942A948DB75E
:10C940009EB742960FB6F8949EBF0FBE8DBFDF9183
:10C95000CF911F91089580E880936100109261004B
:10C960000E94C263CCE4D2E10BE312E18AE2E82E3A
:10C9700082E1F82E99E1C92E92E1D92E2BE0A22E68
:10C9800022E1B22E04B600FE06C0DF93CF930E94D0
:10C990002A940F900F9004B601FE06C01F930F93C8
:10C9A0000E942A940F900F9004B602FE06C0FF92D8
:10C9B000EF920E942A940F900F9004B603FE06C0D7
:10C9C000DF92CF920E942A940F900F9004B604FE3B
:10C9D00006C0BF92AF920E942A940F900F9014BE8F
:10C9E0000E945D700E942267CDCFDF92EF92FF928E
:10C9F0000F931F93CF93DF93CDB7DEB7A0970FB6FA
:10CA0000F894DEBF0FBECDBF83E690E00E94EF96A4
:10CA1000182F282F35EF380F303108F0982F9095C8
:10CA2000291709F463C081E393E19F938F930E94D8
:10CA30002A94E6E7F3E18E010F5F1F4F0F900F90EE
:10CA4000D801D02EE12EF02E88E0800F94919D9396
:10CA500031968A13FBCFF89448E050E06FE770E01E
:10CA6000C8010E94F596E8E6F3E1D8018EE08F0D4B
:10CA700094919D9331968A13FBCF4EE050E061E78D
:10CA800070E0C8010E94F596EEE5F3E12AE02F0D73
:10CA90008491D8018D938D0131962A13F9CF4AE004
:10CAA00050E067E670E08D2D9E2D0E94F5966DECAE
:10CAB0007BEA81E690E00E940D9760E070E08FE5F0
:10CAC00090E00E940D9760E08EE590E00E94FF9656
:10CAD00060E070E085E690E00E940D971AE16AE15F
:10CAE00075EE83E690E00E940D977894812FA096D2
:10CAF0000FB6F894DEBF0FBECDBFDF91CF911F916F
:10CB00000F91FF90EF90DF9008958FE590E00C94E7
:10CB1000EF968EE590E00C94E796F8941092B600AC
:10CB200016BC89E787BD82E084BD95E095BD95B3CD
:10CB300095BB80936E00789408950F931F93609136
:10CB4000A5137091A6138091A7139091A81300913B
:10CB5000A5131091A6132091A7133091A813601765
:10CB600071078207930759F71F910F9108950F934B
:10CB70001F936091AD357091AE358091AF35909136
:10CB8000B0350091AD351091AE352091AF35309173
:10CB9000B035601771078207930759F71F910F91FE
:10CBA00008951F920F920FB60F9211240BB60F9299
:10CBB0002F933F934F935F936F937F938F939F93A5
:10CBC000AF93BF93EF93FF938091A5139091A6131A
:10CBD000A091A713B091A8130196A11DB11D809338
:10CBE000A5139093A613A093A713B093A8138091B5
:10CBF000A4138F5F8093A41387FF15C01092A41312
:10CC00008091AD359091AE35A091AF35B091B035F2
:10CC10000196A11DB11D8093AD359093AE35A093C3
:10CC2000AF35B093B03580914C378823E1F08091D7
:10CC3000A3138F5F8093A31387FF15C01092A313D4
:10CC40008091A5359091A635A091A735B091A835D2
:10CC50000196A11DB11D8093A5359093A635A09393
:10CC6000A735B093A8350E945A6F892B11F00E9406
:10CC70007B6EFF91EF91BF91AF919F918F917F91CB
:10CC80006F915F914F913F912F910F900BBE0F903D
:10CC90000FBE0F901F9018951F920F920FB60F9214
:10CCA00011240BB60F922F933F934F935F936F9383
:10CCB0007F938F939F93AF93BF93EF93FF93809155
:10CCC000C600E091B335F091B435309709F019956D
:10CCD000FF91EF91BF91AF919F918F917F916F9154
:10CCE0005F914F913F912F910F900BBE0F900FBE10
:10CCF0000F901F9018951F920F920FB60F9211244C
:10CD00000BB60F922F933F934F935F936F937F9345
:10CD10008F939F93AF93BF93EF93FF938091CE0038
:10CD2000E091B135F091B235309709F01995FF9146
:10CD3000EF91BF91AF919F918F917F916F915F9193
:10CD40004F913F912F910F900BBE0F900FBE0F9000
:10CD50001F90189581110EC01092C5006093C400F9
:10CD600088E98093C1004093C2001092B4351092BC
:10CD7000B3350895813069F41092CD006093CC00F2
:10CD800088E98093C9004093CA001092B23510928E
:10CD9000B1350895811107C08091C00085FFFCCF97
:10CDA0006093C6000895813031F48091C80085FFFA
:10CDB000FCCF6093CE000895CF93C82F8A3031F412
:10CDC0006DE08091A9130E94CA6602C08D3029F0DF
:10CDD0006C2F8091A9130E94CA6680E090E0CF91E9
:10CDE0000895811105C07093B4356093B3350895EB
:10CDF000813021F47093B2356093B13508958093FA
:10CE0000A91383E992E09093F8398093F739089554
:10CE100084B7877F84BF0FB6F894A895809160008F
:10CE2000886180936000109260000FBE08959FE0BB
:10CE300088E10FB6F894A895809360000FBE909398
:10CE400060000895A89508950FB6F894A89580916C
:10CE50006000886180936000109260000FBE0895AA
:10CE60000C94C68F0C94C28F8091BA3590E00895CF
:10CE70008091390181FF09C0809139018D7F8093B4
:10CE8000390189E190E00197F1F723E040E06FE19B
:10CE900082E491E00E946E6C85E090E00197F1F7EA
:10CEA00008959091390191FD0AC0282F803108F032
:10CEB0002FE040E06FE085E491E00C946E6C089503
:10CEC0008091390181FD0EC040E06FE181E491E085
:10CED0000E94636C282F2F7E81E090E0213021F0AA
:10CEE00080E0089580E090E008958091390181FF0D
:10CEF00002C081E0089540E06FE181E491E00E948A
:10CF0000636C8F3121F08F7E8150823090F780E00A
:10CF100008958091390181FD04C00E9475678823BE
:10CF2000C1F3089510924C378091390181FD8BC077
:10CF30000E9489678091390181FD85C00E94386710
:10CF400080913901826080933901809184378823F0
:10CF5000D9F180919400909195004091953750912E
:10CF6000963784179507A0F48091613790916237C6
:10CF7000A0916337B0916437875F924CAF4FBF4F3A
:10CF80008093613790936237A0936337B09364378F
:10CF90002091940030919500241B350B80916137CE
:10CFA00090916237A0916337B0916437820F931FDD
:10CFB000A11DB11D8093613790936237A0936337B1
:10CFC000B093643710928437809186378823D9F1E3
:10CFD00080919400909195004091993750919A37A3
:10CFE00084179507A0F48091693790916A37A091D2
:10CFF0006B37B0916C37875F924CAF4FBF4F8093C8
:10D00000693790936A37A0936B37B0936C37209150
:10D01000940030919500241B350B809169379091D5
:10D020006A37A0916B37B0916C37820F931FA11DA7
:10D03000B11D8093693790936A37A0936B37B09393
:10D040006C3710928637089580914C37882321F0F1
:10D050000E9475670E94926780E090E0089522E048
:10D06000260F27FF0CC080914A3790914B370196CD
:10D0700090934B3780934A378FEF9FEF0895AB0122
:10D08000BC018AEA93E10E945B9380E090E00895FE
:10D0900040E06FE181E491E00C94636C282F40E064
:10D0A0006FEF86E591E00E946E6C0895CF93DF9359
:10D0B00098EF980F923038F0982F9F7E963019F0A5
:10D0C000893109F049C09091390191FD48C0C82FBC
:10D0D0000E9489670E944868D82FC81709F442C087
:10D0E000C83029F4809139010E94386727C0C931BE
:10D0F00019F4863181F404C0C63169F4893159F4D8
:10D1000029E040E06FE182E491E00E946E6C85E0EE
:10D1100090E00197F1F72C2F40E06FE182E491E07D
:10D120000E946E6CD83031F48FEF0E944E6881ED12
:10D1300092E002C085E090E00197F1F70E94486814
:10D140008C1781F0C63019F4813079F40BC0C631E8
:10D1500061F4813151F406C082E490E008C084E4B7
:10D1600090E005C080E490E002C083E490E0DF91AD
:10D17000CF910895809194009091950090939A3763
:10D180008093993781E08093863780934C379091D4
:10D19000390191FF1EC02091940030919500309389
:10D1A00096372093953780938437809347372FB7EE
:10D1B000789480913901809139018D7F8093390174
:10D1C00080E197E230914737332311F00197D1F78F
:10D1D0002FBF86E10E9456680C94896780914C3776
:10D1E000811102C00E94BA6881E090E008950F9317
:10D1F0001F93CF93DF931F92CDB7DEB780914C374B
:10D20000882361F08091390181FF02C080E07BC0FA
:10D210000E9475678823D1F300E003C00E94EE6886
:10D2200001E08091940090919500909394378093C1
:10D23000933711E01093833780E88093550186E09F
:10D240000E9456681093BB358FB7898378941092EB
:10D2500047018091BB358111FCCF89818FBF8091BF
:10D26000470111E08E3008F010E0119586E10E9430
:10D27000566810925501809183378823D9F18091A7
:10D280009400909195004091933750919437841772
:10D290009507A0F480915D3790915E37A0915F373C
:10D2A000B0916037875F924CAF4FBF4F80935D372F
:10D2B00090935E37A0935F37B093603720919400CE
:10D2C00030919500241B350B80915D3790915E372E
:10D2D000A0915F37B0916037820F931FA11DB11DE0
:10D2E00080935D3790935E37A0935F37B09360373C
:10D2F0001092833701110E942468812F82958695B0
:10D3000086958370817090E00F90DF91CF911F918F
:10D310000F9108958FEF80934E0121E044E060EF7C
:10D320008CE691E00E946E6C25E041E06EE08CE6B8
:10D3300091E00E946E6C80E880936F0180914601BD
:10D3400080936D0121E045E060E284E491E00C947B
:10D350006E6CCF93DF93C9EFD7E0CE010197F1F761
:10D360000E94626C1092C135109243361092C536FD
:10D370001092C0351092BF35E9E3F1E080818E7FD5
:10D38000808380818D7F808381EC93E00197F1F72A
:10D3900080818160808323E040E06FE182E491E05E
:10D3A0000E946E6C2197F1F780915D0180915E0182
:10D3B0000E948A6960E070E081EA92E00E94EF706A
:10D3C0000E94BA6881E090E0DF91CF91089580914A
:10D3D0002B140895CF93DF931F92CDB7DEB78983C7
:10D3E0000E948967898180932B14282F40E06FE188
:10D3F00088E491E00F90DF91CF910C946E6C0E94C5
:10D40000EA6986E00C945668EF92FF920F931F939F
:10D41000CF93DF931F921F92CDB7DEB78C017A01B5
:10D420007F936F931F938F938CE799E09F938F93D4
:10D4300069837A830E9416940093620110936301BA
:10D440006981609360017A81709361010F900F9000
:10D450000F900F900F900F90E114F104C9F0F701B5
:10D46000808180936B01818180936A0182818093A6
:10D47000690183818093680184818093670185813C
:10D480008093660186818093650187818093640122
:10D490000F900F90DF91CF911F910F91FF90EF9020
:10D4A000089581EA92E00E94107181E08093BA357C
:10D4B0008091BC359091BD3501969093BD35809398
:10D4C000BC3581E090E008950F931F93CF93209196
:10D4D000C035C2E8C29F90011124F901EF53FA4C04
:10D4E0004081442309F451C047FD09C0433038F05E
:10D4F00050E08A01025011096017710710F4108280
:10D5000044C0B9016E537A4C0E945B938091C03540
:10D51000C89FF0011124EF53FA4CDF01A058BF4F10
:10D520009C919093B53510828F5F833018F480936F
:10D53000C03502C01092C035E091C03582E8E89F46
:10D54000F0011124EF53FA4C8081882319F00E94D6
:10D55000516A02C01092BA35809147018093B63566
:10D560009091B935992311F0891710F48093B9354A
:10D570006091B63570E084E00E940F766091B53519
:10D5800070E083E00E940F7602C000E010E0C80166
:10D59000CF911F910F9108950F931F93CF93DF9316
:10D5A0001F92CDB7DEB78C01FC018081918100977D
:10D5B00009F18334954029F0F8011182108283E04B
:10D5C0002AC06238E1F40E94BB758FB78983F89452
:10D5D0000E942A7560E870E00E94646A29812FBF6A
:10D5E0001816190674F40E942575E091220AF0912C
:10D5F000230A199583E495E0F8019183808381E003
:10D600000AC08091B7359091B83501969093B8359E
:10D610008093B735EFCF0F90DF91CF911F910F918E
:10D6200008950C9451678091390181FD06C040E056
:10D630006FE085E491E00C94636C80E10895EF92D3
:10D64000FF921F93CF93DF931F92CDB7DEB7182FB2
:10D650008091390181FD07C00E94896780914C3714
:10D6600081111CC05AC080919400909195009093B4
:10D6700096378093953781E080938437809347373E
:10D68000809139018D7F8093390180E197E220916B
:10D690004737222309F30197D1F7DECF80918637F0
:10D6A0008823D9F180919400909195004091993709
:10D6B00050919A3784179507A0F48091693790911B
:10D6C0006A37A0916B37B0916C37875F924CAF4F40
:10D6D000BF4F8093693790936A37A0936B37B093AD
:10D6E0006C372091940030919500241B350B80916C
:10D6F000693790916A37A0916B37B0916C37820F80
:10D70000931FA11DB11D8093693790936A37A09331
:10D710006B37B0936C371092863789E10E94566858
:10D7200086E00E941A76892B51F00E94136BE82E36
:10D7300086E00E941A7681500E94516702C0E12C57
:10D74000F12C80919400909195009093983780935C
:10D75000973781E0809385378FB78983F8948091DC
:10D760003901826080933901809139018D7F8093E6
:10D77000390162E0610F8AEA93E10E94B56C898108
:10D780008FBF8091483790914937019690934937E0
:10D79000809348370E94896745E060EE82E491E01B
:10D7A0000E94636C182F86E00E941A76892B19F06C
:10D7B0008E2D0E945167809185378823D9F1809101
:10D7C0009400909195004091973750919837841725
:10D7D0009507A0F48091653790916637A0916737DF
:10D7E000B0916837875F924CAF4FBF4F80936537DA
:10D7F00090936637A0936737B09368372091940071
:10D8000030919500241B350B8091653790916637D8
:10D81000A0916737B0916837820F931FA11DB11D8A
:10D820008093653790936637A0936737B0936837D6
:10D830001092853780914C37882371F08091940045
:10D840009091950090939A378093993781E08093D7
:10D8500086370E94BA6802C00E949267123028F48C
:10D860008CE00E941A7610E00BC0133031F01530B6
:10D8700031F0173029F411E003C012E001C013E0C9
:10D88000812F90E00F90DF91CF911F91FF90EF904B
:10D890000895CF93DF93EB010E942F68009729F43E
:10D8A000CE010E941F6B009751F020914A373091B2
:10D8B0004B372F5F3F4F30934B3720934A37DF91E1
:10D8C000CF9108950895FC0180816823862F90E010
:10D8D00002C0959587954A95E2F70895CF93DF9317
:10D8E0001F92CDB7DEB7FC01922F8FB78983F894D2
:10D8F0002081362F3095522F5323292F01C0220F1C
:10D900004A95EAF72623252B208389818FBF0F9024
:10D91000DF91CF910895CF93DF93E0917B012DEFBD
:10D920002E0F2D3740F0FC011082E058FF4F10827F
:10D930003196108217C0EC01E993A0E8B1E020E82D
:10D940002E0F3C91399311962A13FBCFE150F0E052
:10D95000E058FE4F2181FC01E058FF4F20833196B3
:10D9600081E08083DF91CF91089560938001E1E8A9
:10D97000F1E06158DC012D91CD01208331966E13C9
:10D98000F9CF08951F920F920FB60F9211240BB684
:10D990000F922F933F934F935F936F937F938F9348
:10D9A0009F93AF93BF93EF93FF9380914701809331
:10D9B000B6358091BF3522E8829FC00111248F5374
:10D9C0009A4C0E948B6C8091BF358F5F833018F426
:10D9D0008093BF3502C01092BF350E94516AFF91FB
:10D9E000EF91BF91AF919F918F917F916F915F91D7
:10D9F0004F913F912F910F900BBE0F900FBE0F9044
:10DA00001F9018951F920F920FB60F9211240F902E
:10DA10000FBE0F901F9018951F920F920FB60F9286
:10DA200011240F900FBE0F901F9018951F920F9208
:10DA30000FB60F9211240F900FBE0F901F901895E4
:10DA40001F920F920FB60F921124109247370F902A
:10DA50000FBE0F901F9018951F920F920FB60F9246
:10DA600011241092BE350F900FBE0F901F90189585
:10DA70001F920F920FB60F9211240F900FBE0F90AE
:10DA80001F9018951F920F920FB60F9211241092AB
:10DA9000BB350F900FBE0F901F901895CF93DF935B
:10DAA000EC0189919991009729F060E070E00E9463
:10DAB000EF70F7CFDF91CF910895EF92FF920F9320
:10DAC0001F93CF93DF938C017A01FC0180819181B8
:10DAD000009741F08A34910511F1F801118210820A
:10DAE00083E04AC08DE294E10E949A71EC01209794
:10DAF00061F04E815F8168857985CE0102960E9432
:10DB0000316F0990D881C02DF2CF81E080932C1421
:10DB10008AE490E0F8019183808381E02DC0683829
:10DB2000E1F78DE294E10E949A71EC01209781F374
:10DB3000CE010296E816F906D9F4BE018DE294E111
:10DB40000E94BA71E090E114F090E2148E859F85F6
:10DB50009093E2148093E114E889F989309719F0E1
:10DB60008A899B891995F092E214E092E114D0CF52
:10DB70000990D881C02DDACFDF91CF911F910F91FD
:10DB8000FF90EF90089510922C148DE294E10E9482
:10DB9000967160E070E08BEA92E00C94EF70EF9287
:10DBA000FF920F931F93CF93DF93EC01E090E1146A
:10DBB000F090E214FF86EE86398B288B1B8B0A8B44
:10DBC00080912C14882379F08BEA92E09093E214F0
:10DBD0008093E114CE0102960E94316FF092E2141C
:10DBE000E092E11404C04E835F8368877987BE01A9
:10DBF0008DE294E10E94BA71BE018DE294E1DF9161
:10DC0000CF911F910F91FF90EF900C94D971CF930A
:10DC1000DF93EC0180912C14882329F0CE01029629
:10DC20000E94656F04C01B861A861D861C86BE0175
:10DC30008DE294E1DF91CF910C94BA71CF92DF9293
:10DC4000EF92FF920F931F938091331490913414AD
:10DC5000892B49F410922F14109230141092311421
:10DC60001092321441C00E949D658B019C01E0918D
:10DC70003314F09134144481558166817781808119
:10DC80009181A281B381840F951FA61FB71F801BAE
:10DC9000910BA20BB30B0084F185E02D3097C1F0FE
:10DCA000C480D580E680F780408151816281738194
:10DCB0004C0D5D1D6E1D7F1D401B510B620B730BC8
:10DCC000481759076A077B0730F7DB01CA01E3CF22
:10DCD000800F911FA21FB31F80932F1490933014B5
:10DCE000A0933114B09332141F910F91FF90EF90D5
:10DCF000DF90CF90089585EB92E00C941071EF9235
:10DD0000FF920F931F93CF93DF938C01FC018081CF
:10DD10009181009799F089359105D9F0F801118228
:10DD2000108283E068C0828593858417950709F087
:10DD300049C00084F185E02D3097A9F71092341482
:10DD40001092331489E590E0F8019183808381E09B
:10DD500052C0673891F16238A9F7C0913314D0915D
:10DD60003414E12CF12C209769F3CE010E946B71E1
:10DD7000892BF1F0AE0168E88A859B850E94C1700D
:10DD8000892BA1F41B861A8688859985E114F104F4
:10DD900021F0F7019187808704C090933414809319
:10DDA0003314198618860E941E6ED7CF0E947B6E90
:10DDB0007E010884D985C02DD6CFE0913314F0912F
:10DDC0003414BACFF0933414E0933314A085B185A2
:10DDD000109709F4B7CF1A968D919C911B978417D1
:10DDE000950739F418968D919C91199791878087A2
:10DDF000EDCFFD01EBCFDF91CF911F910F91FF9000
:10DE0000EF900895CF93DF93EC010E947B6E2A85FB
:10DE10003B859091331480913414232B91F0E92F9A
:10DE2000F82F309771F0EC17FD0739F48091E11469
:10DE30009091E2149387828710C00084F185E02DD1
:10DE4000F0CF2091E1143091E2143B872A87988724
:10DE50008987D0933414C0933314DF91CF910C94FD
:10DE60001E6ECF93DF93EC010E943D71CE01DF91D6
:10DE7000CF910C94026FCF93DF93EC010E944D7110
:10DE8000CE01DF91CF910C94026FCF93DF93EC0121
:10DE90000E945F71CE01DF91CF910C94026F21E05F
:10DEA00030E0FC0182859385892B11F020E030E081
:10DEB000C901089581E090E0209133143091341429
:10DEC000232B11F480E090E00895CF93DF93EC01D1
:10DED000E0913314F09134148E179F0769F488850C
:10DEE000998590933414809333140DC08085918567
:10DEF0008C179D0721F0FC013097C1F706C088857B
:10DF00009985918780870E941E6E198618861B86C8
:10DF10001A86DF91CF9108951F93CF93DF93DC0191
:10DF20001496ED91FC9115973097E1F0162FEC01C6
:10DF30009093E2148093E11482E08887CD010696E5
:10DF40001995082E000C990B0297029710F01338C0
:10DF500039F4BE01CE01DF91CF911F910C94BC6FBB
:10DF600081E08887DF91CF911F910895FC01208582
:10DF700020FD0C948C6F0895CF92DF92EF92FF9268
:10DF80000F931F93CF93DF93E090E114F090E2148E
:10DF9000C090E314D090E414F601E817F90739F0C3
:10DFA000309709F44BC00190F081E02DF6CF009737
:10DFB00009F444C08B01EC018885882309F1188697
:10DFC000C114D10461F0CC15DD0529F0AE0167E87C
:10DFD000C6010E94B66FF601C080D180F1CFEC81FE
:10DFE000FD81309769F0C017D10751F0D093E2144A
:10DFF000C093E11440E050E063E8CE010696199525
:10E00000E091E314F091E414CE17DF0741F4888126
:10E0100099819093E4148093E3140CC0FC01309731
:10E0200049F0808191818C179D07C1F78881998182
:10E0300091838083F092E214E092E114DF91CF911A
:10E040001F910F91FF90EF90DF90CF9008951F9355
:10E05000CF93DF9310923D14C091E314D091E41458
:10E0600011E0209779F08985882341F01887198677
:10E0700040E050E062E8CE010E948C6F0990D881A8
:10E08000C02DEFCFDF91CF911F9108958091E014C3
:10E0900091E0980F9093E01408958AE88093E0143B
:10E0A0001092DE141092DF141092E4141092E31414
:10E0B0001092E2141092E114089580913D148111A0
:10E0C0000E9427705091DF14552309F452C0E0914B
:10E0D000DE142E2F30E085E0E89FF0011124E25C91
:10E0E000FB4E608160933C14A181B281B0933B14DC
:10E0F000A0933A14838194819093391480933814B7
:10E100002F5F3F4F2F7133272093DE1451505093D0
:10E11000DF14009731F58091E3149091E41490930B
:10E120003714809336148091361490913714892BCC
:10E1300001F180913D1481110E94277040913A14A1
:10E1400050913B1460913C14809136149091371497
:10E150000E94B66FE0913614F0913714808191815E
:10E16000DECF613819F421E0FC012087AD010E9467
:10E17000B66F80913D142091DF1490E0820F911DC5
:10E1800008959C019091DF149032B9F0E091DE1473
:10E19000E90FEF71E093351485E0E89FF001112459
:10E1A000E25CFB4E608352834183348323839F5F11
:10E1B0009093DF1480E090E0089581E090E008956E
:10E1C000CF93DF93C091E114D091E2140E94B66F17
:10E1D000D093E214C093E114DF91CF910895AB0185
:10E1E0003091E3142091E414E32FF22FE817F9079C
:10E1F000B1F0309721F00190F081E02DF7CF00973A
:10E2000071F0FC01308321839093E4148093E31434
:10E2100021E020871782168261E80C94E07008954F
:10E22000009749F0FC0120852150223020F421E0A4
:10E23000218720933D1408950C94497A8091E51428
:10E240009091E6140097C1F01092E6141092E51434
:10E25000DC0114966D917C9115971296ED91FC91CD
:10E2600013971995E091E514F091E614309721F099
:10E27000808191810C94637A0895CF93DF93EC01B0
:10E280004C835D836E837F830E949D656883798361
:10E290008A839B83DF91CF910895FC014081518156
:10E2A0006281738184819581A681B781840F951FD6
:10E2B000A61FB71F80839183A283B3830895CF9352
:10E2C000DF93EC010E949D65688379838A839B8339
:10E2D000DF91CF910895CF92DF92EF92FF92CF938B
:10E2E000DF93EC010E949D65C880D980EA80FB80A5
:10E2F000DC01CB018C199D09AE09BF090196A11D56
:10E30000B11D21E030E0CC80DD80EE80FF80C816BA
:10E31000D906EA06FB0610F020E030E0C901DF91E3
:10E32000CF91FF90EF90DF90CF900895FC01118284
:10E3300010820895FC01808191810895DC01ED91A6
:10E34000FC91309741F080819181009711F0FC01A0
:10E35000FACFCF01089580E090E00895DC01ED91BF
:10E36000FC911197309721F0208131812D933C93BE
:10E37000CF010895DC01ED91FC913097C9F0A0E048
:10E38000B0E0E617F70761F4FB01208131811097B7
:10E3900009F4DC012D933C93FB0111821082089556
:10E3A00020813181DF012115310511F0F901E9CF1B
:10E3B00008950F931F93CF93DF938C01EB010E947D
:10E3C000BA7119821882C8010E949E71009711F4D7
:10E3D000F80101C0FC01D183C083DF91CF911F916F
:10E3E0000F910895DC01ED91FC9180E090E0309771
:10E3F00029F001960190F081E02DF9CF0895009762
:10E4000021F0FC0180819181089580E090E00895E1
:10E41000CF93DF93EC014A815B8160E070E08C81F7
:10E420009D810E9464932A813B8188819981289FE4
:10E43000A001299F500D389F500D112460E070E01D
:10E440008E819F81DF91CF910C946493FC01828136
:10E45000938120E030E028173907D1F0A481B581FD
:10E46000A20FB31F4C91411110C081E08C938081A9
:10E470009181289FA001299F500D389F500D112494
:10E4800086819781840F951F08952F5F3F4FE3CFBB
:10E4900080E090E00895FC0186819781428153815C
:10E4A00020E030E024173507D1F08617970781F474
:10E4B000A481B581A20FB31F8C91181614F481505A
:10E4C0008C9384819581FC01E20FF31F8081089574
:10E4D000A081B1818A0F9B1F2F5F3F4FE3CF8FEF4A
:10E4E0000895FC012681378162177307A0F0A0818F
:10E4F000B18142815381A49FC001A59F900DB49F1B
:10E50000900D1124280F391F81E090E062177307E6
:10E5100020F080E0089580E090E008952F923F92EF
:10E520004F925F926F927F928F929F92AF92BF9223
:10E53000CF92DF92EF92FF920F931F93CF93DF93CF
:10E54000CDB7DEB768970FB6F894DEBF0FBECDBF6C
:10E55000EDE4F7E324A535A546A557A550A441A4AD
:10E5600032A423A4948C858C768C678C808D8983CF
:10E57000918D9A83828D8B83938D9C8384898D83E7
:10E5800095899E8386898F839789988780898987D3
:10E5900091899A8782898B8793899C8784858D87C7
:10E5A00095859E8786858F879785988B8085898BB3
:10E5B00091859A8BB284A384F480E580D680C7804D
:10E5C00080818F8B9181988F128103812B8B3C8B63
:10E5D0004D8B5E8B0E94B7655E895F934D894F932B
:10E5E0003C893F932B892F932F923F924F925F92BA
:10E5F0006F927F928F929F922C812F932B812F93DA
:10E600002A812F9329812F9328852F932F812F9350
:10E610002E812F932D812F932C852F932B852F9334
:10E620002A852F9329852F9328892F932F852F9320
:10E630002E852F932D852F93AF92BF922A892F93EA
:10E6400029892F93CF92DF92EF92FF920F931F931E
:10E65000288D2F932F892F939F938F937F936F9361
:10E66000E3EAF7E381811F928F9380811F928F935A
:10E670008EE793E19F938F930E942A940FB6F894AC
:10E68000DEBF0FBECDBF68960FB6F894DEBF0FBEDB
:10E69000CDBFDF91CF911F910F91FF90EF90DF9051
:10E6A000CF90BF90AF909F908F907F906F905F9032
:10E6B0004F903F902F900895EF92FF920F931F93EA
:10E6C000CF93DF938C01EB017A010E94F273F80182
:10E6D000F086E78265ED79E0CE01DF91CF911F9161
:10E6E0000F91FF90EF900C9416740C94FA730C94A5
:10E6F000AE74DC011796ED91FC9118970190F081B2
:10E70000E02D309709F019940895DC011796ED91EA
:10E71000FC9118970280F381E02D309709F019944D
:10E720000895DC011996ED91FC911A970280F3810E
:10E73000E02D309709F0199408950F931F93CF930C
:10E74000DF931F921F92CDB7DEB78C0188E10E9444
:10E750002D76BC01CE0101960E94DC74D801199679
:10E76000ED91FC911A970190F081E02D309729F0FE
:10E77000BE016F5F7F4FC80119950F900F90DF9119
:10E78000CF911F910F910895EF92FF920F931F93D6
:10E79000CF93DF938C01EB017A0147ED59E00E94A2
:10E7A0005C73F801F286E1866BED79E0CE01DF91D2
:10E7B000CF911F910F91FF90EF900C9416740C94D1
:10E7C0007573CF93DF93EC0163EA77E388E10E94EE
:10E7D0002376CE01DF91CF910C94777387EE94E18D
:10E7E0000C949671FC0173836283BC0187EE94E103
:10E7F0000C94D971BC0187EE94E10C94BA71CF935B
:10E80000DF93EC0187EE94E10E949A71009749F042
:10E81000FC01228133812C173D0729F00E94FF71F2
:10E82000F5CF80E090E0DF91CF9108950F931F9393
:10E83000CF93DF938B010E94FF73EC01892B31F0A2
:10E840001D830C83C8010E9416848E83DF91CF91B3
:10E850001F910F910895CF92DF92EF92FF920F9345
:10E860001F93CF93DF937C018B016A0189EE94E1C2
:10E870000E949A71EC01892B51F0EC81FD81309757
:10E8800011F0C8011995CE010E94FF71F3CFA601C6
:10E89000B801C701DF91CF911F910F91FF90EF90C9
:10E8A000DF90CF900C9485730F931F93CF93DF93DA
:10E8B0001F921F92CDB7DEB70E94E8838C0189EECC
:10E8C00094E10E949A71009779F0DC011296ED9123
:10E8D000FC911397309729F089839A8319959A812F
:10E8E00089810E94FF71EFCF0115110549F0C80120
:10E8F0000F900F90DF91CF911F910F910C9479732E
:10E900000F900F90DF91CF911F910F910895CF92AB
:10E91000DF92EF92FF920F931F930E9433760E9433
:10E92000BB750E947D820E94E683C12C88E0D82EB0
:10E9300087E0E82EF12C00E01EE120E030E040E02E
:10E9400052E060E070E082E090E00E94AD831F91B1
:10E950000F91FF90EF90DF90CF900895CF93DF93CA
:10E96000EC010E94FB83009761F00E944375E091E7
:10E97000F609F091F709BE018BE294E7199581E061
:10E9800090E0DF91CF910895E0911E0AF0911F0A67
:10E990001994E091E809F091E9091994E091240AA9
:10E9A000F091250A1994E091260AF091270A19940A
:10E9B00080E090E008950895FB0120813181FC0101
:10E9C00031832083089542E050E00E944E9321E07D
:10E9D00030E0892B11F020E030E0C9010895BC013E
:10E9E00083EA97E30C94DC74E091A609F091A709FF
:10E9F0001995E0911C0AF0911D0A1995E091F4090E
:10EA0000F091F5091995E091E609F091E70919945B
:10EA10002091A2153091A3152817390798F040913D
:10EA2000A0155091A115480F591F5093A11540935F
:10EA3000A015281B390B3093A3152093A21581E054
:10EA400090E0089580E090E008959093A31580935E
:10EA5000A21508958091A0159091A115835E9A4EFC
:10EA6000089580919F1590E083519B4E089581E019
:10EA700090E02091EB143091EC142D51354111F4BC
:10EA800080E090E008950E943775892B61F06091D5
:10EA9000EB147091EC144091A2155091A3158DE1E7
:10EAA00095E10C945B932091A0153091A11521154F
:10EAB0003105B9F08091A2159091A315C096EDE1B2
:10EAC000F5E1AF014D5E54414817590734F4DF01B9
:10EAD000A20FB31F4C914193F4CF1092A115109245
:10EAE000A01508958091A2159091A3150895809185
:10EAF0009F1590E3981B2091A2153091A315A901B1
:10EB0000490F511DCA0108950F931F93CF938C0194
:10EB1000C0919F158C2F90E0801791076CF00E9498
:10EB20007775800F911F8138910530F4C01BC09319
:10EB30009F1581E090E002C080E090E0CF911F91AE
:10EB40000F910895CF93DF93EDEAF7E311921192BD
:10EB500087E3ED3DF807D1F7C5EAD7E360E07AE057
:10EB6000CE010E94DC74229687E3CD3AD807B1F734
:10EB7000DF91CF9108951092A1151092A0151092D7
:10EB8000A3151092A21580E380939F158DE195E166
:10EB90009093EC148093EB140C94A275EF92FF9277
:10EBA0000F931F93CF93DF931F921F92CDB7DEB7C2
:10EBB0008C0169837A830E94BB756981E62E7A8114
:10EBC000F72E81E8E816F10418F080E8E82EF12C21
:10EBD000A701B8018091EB149091EC140E945B9313
:10EBE000F092A315E092A215C7010F900F90DF914C
:10EBF000CF911F910F91FF90EF900895FC0190E34A
:10EC0000ADEAB7E301900D929A95E1F788E0FB0138
:10EC1000A5EAB7E301900D928A95E1F70895E82FF0
:10EC2000F0E0EE0FFF1FE355F84C7183608381E045
:10EC300090E00895E82FF0E0EE0FFF1FE355F84C49
:10EC400080819181089590E0880F991F8B58984C8E
:10EC50000E94DC7481E090E0089590E0880F991F95
:10EC60008B58984C08958FEB92E00E9408728FECBD
:10EC700092E00E94087287EC92E00C9408720F9365
:10EC80001F93CF93DF93EC01BC018FEC92E00E94C5
:10EC90007172892BA9F00990D881C02DFE01619174
:10ECA0007191CF010E94CE75BE016E547F4FCE018F
:10ECB0008E579F4FDF91CF911F910F910C94FE754E
:10ECC000BE0187EC92E00E947172892BD1F00E9404
:10ECD000BB75688179818A819B810E94CE758CA9E0
:10ECE00090E00E9484750CA910E00E943175BE016D
:10ECF0006C5F7F4FA801DF91CF911F910F910C9412
:10ED00005B93DF91CF911F910F91089587E19CE173
:10ED10000E944F6F892B21F087E19CE10C94456F95
:10ED20000895E091031CF091041C309709F01994A8
:10ED300080E00895EF92FF920F931F93CF93DF939C
:10ED40008C01EA01FC0180819181009741F08A33B6
:10ED5000934081F1F8011182108283E0F8C080E0D5
:10ED600024E0829FF0011124EB5FF34E11821082A8
:10ED70008F5F8430A9F78093021C8091E1149091F9
:10ED8000E2149093161C8093151C0E944670809389
:10ED9000DD3740E450E060E070E087E19CE10E94F4
:10EDA000316F0E942A7B8AE393E0F801918380838C
:10EDB00081E0CDC06230D9F48091DE379091DF37A9
:10EDC000892B89F38091EF37863029F480910738B9
:10EDD00081FD0E94867681E00E94717B8091DE3702
:10EDE0009091DF37892BF9F20E94F477DCCF633002
:10EDF00060F5611114C02097B1F2D093DC38C09354
:10EE0000DB3883E00E94717B8091DE379091DF37A1
:10EE1000892B11F00E9491760E948676C4CF6130D2
:10EE200011F6209709F4BFCFD093D838C093D738C4
:10EE300085E00E94717B8091DE379091DF37892BCE
:10EE400009F4B1CF0E949176AECF673809F040C087
:10EE50001092011C85E0E82E8CE1F82E8091011CB7
:10EE60008430C0F4F701828193818C179D0749F4A7
:10EE7000808191810E94567BF7011182108213825A
:10EE80001282F4E0EF0EF11C8091011C8F5F8093E1
:10EE9000011CE4CFE6EFF8E3838194818C179D0792
:10EEA00019F4148213821082B09629E3E637F20730
:10EEB00099F7E3E7F9E3818592858C179D0711F4B3
:10EEC000158214823D9689E3E53FF807A1F76BCFE1
:10EED000683809F068CFC751DC4109F064CF87E199
:10EEE0009CE10E944F6F892B09F45DCF1092011CA9
:10EEF000E091011CE43008F056CF20E2E29FF001DF
:10EF00001124E352F74C818D8823D9F087E19CE1ED
:10EF10000E94456F8091011CE0E28E9FC001112488
:10EF20008352974C9093DC388093DB3882E00E94C8
:10EF3000717B8091DE379091DF37892B11F00E9431
:10EF400091768091011C8F5F8093011CD1CFDF915E
:10EF5000CF911F910F91FF90EF900895CF93DF9382
:10EF6000A091DB38B091DC38109719F0ED016C9668
:10EF700005C0C091D738D091D83829968091D6381D
:10EF800086FF23C01092001C80E0E5E0FCE18430A5
:10EF9000C1F04081518114962D913C9115974217F3
:10EFA000530761F4228133812115310539F08093B3
:10EFB000001C398328831B821A8205C034968F5F18
:10EFC000E6CF8093001C0E94867688819981009705
:10EFD00041F04A815B816091DD37DF91CF910C94E4
:10EFE000E070DF91CF9108950F931F93CF93DF933C
:10EFF0008091EF37863009F07AC08091DE379091AA
:10F00000DF37803F910508F472C08897EC01D695F0
:10F01000C7959E01220F331F8E012817390710F460
:10F020000F5F1F4FCE0188969093DF378093DE37B6
:10F030009093E8378093E93710920B3810920A3892
:10F040000E94247B8095909590930B3880930A388A
:10F050001092F1371092F0370E94137B80959095B3
:10F060009093F1378093F0370E949176C80188968B
:10F070009093DF378093DE379093E8378093E937BA
:10F080008091D9389091DA38BC016C0F7D1FA801AE
:10F090000E945B93BE018EEF97E30E94C07A80913D
:10F0A000E2378093FE378091E3378093FF3780917A
:10F0B000E437809300388091E537809301381092CF
:10F0C0000B3810920A380E94247B8095909590937B
:10F0D0000B3880930A381092F1371092F0370E9463
:10F0E000137B809590959093F1378093F037DF9163
:10F0F000CF911F910F910C949176E091B609F09108
:10F10000B709199480E090E00895AF92BF92CF9232
:10F11000DF92EF92FF920F931F93CF93DF93CDB7C0
:10F12000DEB7E1970FB6F894DEBF0FBECDBF7C010E
:10F130006B01CE0101965C0181E3F50111928A9584
:10F14000E9F781E089838CE00E941A768C831D8226
:10F150001F828091231C91E0980F9093231C898734
:10F1600013E018878DEC9BEA9B878A8789E10E94D0
:10F170002D7660E07AE00E94E374892B31F082E022
:10F180008E838FEF8C878D8709C089E10E942D7651
:10F19000BC01CE010C960E94DC741E838DEC9BEAB0
:10F1A0009D8B8C8B63EA77E3CE0146960E94DC74DC
:10F1B0000E942A759FA78EA70E94727599AB88AB93
:10F1C000C5010E945E848C011127C8010E948475CC
:10F1D000892B31F10E943175A801BC01C5010E9443
:10F1E00081840091AC091091AD090E9477755C0192
:10F1F0000E943175B501F8011995E114F10481F00F
:10F20000009739F0019761F441E050E064E070E06C
:10F2100004C041E050E060E070E0C601F7011995DC
:10F22000E1960FB6F894DEBF0FBECDBFDF91CF9150
:10F230001F910F91FF90EF90DF90CF90BF90AF9014
:10F2400008950F931F93CF93DF934115510579F0E4
:10F25000FA018B01EC01828193810E943F76B80113
:10F26000CE01DF91CF911F910F910C948578DF91A2
:10F27000CF911F910F9108950F931F93CF93DF9319
:10F28000CDB7DEB7E1970FB6F894DEBF0FBECDBFA6
:10F290000E9472758C010E942A75AE014F5F5F4F0C
:10F2A000B8010E947485892B09F443C088A999A9E3
:10F2B0009801281B390BC9010E940875892BC9F1D7
:10F2C0008E8181110CC0BE016A5E7F4F88E10E9471
:10F2D0002376E091F809F091F90919952AC02A8559
:10F2E0003B852D3C9BEA390719F02F3F3F4F09F52D
:10F2F000823019F088E090E002C082E090E001974F
:10F3000010F3E1E0F0E0EC0FFD1FE80FF91F23859B
:10F310002F3FA9F3BE01645F7F4F89E10E942376EE
:10F3200089E10E942D7663EA77E30E94E374892BDA
:10F3300051F6E1960FB6F894DEBF0FBECDBFDF9158
:10F34000CF911F910F9108950E9432678093231CE3
:10F35000E091B609F091B7091994892B29F0E09151
:10F36000B609F091B70904C0E091B809F091B90964
:10F370001994FC01680F791F80E048E1E617F70750
:10F3800081F0219198E0322F3827532F517030FDB2
:10F3900084278695513009F480682695915099F715
:10F3A000EDCF08951F920F920FB60F9211240BB656
:10F3B0000F922F933F934F935F936F937F938F930E
:10F3C0009F93AF93BF93EF93FF938091940090919D
:10F3D00095009093903780938F3781E080938137A9
:10F3E00080917100807D809371000E941E718091D8
:10F3F00081378823D9F180919400909195004091B4
:10F400008F375091903784179507A0F48091553726
:10F4100090915637A0915737B0915837875F924CEB
:10F42000AF4FBF4F8093553790935637A0935737C0
:10F43000B09358372091940030919500241B350BE0
:10F440008091553790915637A0915737B0915837E2
:10F45000820F931FA11DB11D80935537909356378E
:10F46000A0935737B093583710928137FF91EF919F
:10F47000BF91AF919F918F917F916F915F914F91CC
:10F480003F912F910F900BBE0F900FBE0F901F90CA
:10F4900018959FB7F894E1E7F0E08081807D808344
:10F4A00088B38F6288BB10929000E1E9F0E010828F
:10F4B00010929200109295001092940080818560C5
:10F4C00080839FBF08959C019FB7F8943093990063
:10F4D0002093980088B38F6288BBE1E7F0E08081D9
:10F4E000826080839FBF0895FB0141505109460F00
:10F4F000571FE417F50778F4208130E0322F2227D8
:10F500006181260F311D820F931F8217930708F424
:10F5100001963296EECFE417F50751F4208130E0E2
:10F52000322F2227820F931F8217930708F4019628
:10F530000895CF93DF93C091E937D0E0649720918D
:10F54000E83730E0322F2227C20FD31F48E050E0C7
:10F5500062EF77E39E01280F311DC9010E94747A82
:10F56000AE016AEF77E30E94747A009721F0982742
:10F570008927982702C08FEF9FEFDF91CF910895E1
:10F58000FC012381260F2093E537A72FBB2792810B
:10F590009A0F9093E43731813093E3374081409361
:10F5A000E237E92FF0E0EA17FB0748F481E0830F28
:10F5B0008093E337811103C04F5F4093E23730E01F
:10F5C00077272617370788F49F5F9093E4379111C8
:10F5D0000CC08091E3378F5F8093E337811105C0C2
:10F5E0008091E2378F5F8093E23708952091DB3876
:10F5F0003091DC38BC01C90108960E94C07AE091C4
:10F60000DB38F091DC38A2EEB7E38C91808711965D
:10F610008C911197818712968C91129782871396FD
:10F620008C918387089544E150E066EE77E380E0B3
:10F6300090E00E94747A009721F0982789279827F4
:10F6400008958FEF9FEF089586E00C94997A81E1F9
:10F650000C94997A80E0E82FF0E0EE0FFF1FE35A58
:10F66000F64C118210828F5F8430A9F780E090E21F
:10F67000899FF0011124E352F74C118E8F5F843083
:10F68000B1F780E094E09093291C8093281C80E0DF
:10F690009DE0989FF0011124ED58F64C15821482DC
:10F6A0008F5F8A30B1F78093271C08959C0190E00A
:10F6B0009430A1F0E92FF0E081E0890FEE0FFF1FF9
:10F6C000E35AF64C408151814217530729F4909335
:10F6D000271C118210820895982FEACF9093271C3F
:10F6E0000895AF92BF92CF92DF92EF92FF920F9365
:10F6F0001F93CF93DF93C091DB38D091DC388430F7
:10F7000009F4DBC12EE038E33093DA382093D9389E
:10F710003093E1372093E037833059F4898D8F702F
:10F72000833009F06AC088899989892B09F0D4C689
:10F730007EC0823009F07FC080912D1C8F5F809346
:10F740002D1C811113C080912C1C8F5F80932C1C69
:10F7500081110CC080912B1C8F5F80932B1C811119
:10F7600005C080912A1C8F5F80932A1C1092DF377E
:10F770001092DE371092723910927139898D982F5C
:10F780009D7F953041F48A8D8F5F8A8F843109F097
:10F79000A3C6198EA1C6882309F49EC62889398973
:10F7A000232B09F440C09A8D2FEF290F2A8F911136
:10F7B00093C69B8D983031F02FEF280F223048F4FC
:10F7C000953039F4198E80E88093D6380E94AE7750
:10F7D0003DC5953038F423E0092E01C0220F0A946C
:10F7E000EAF701C020E32A8F9F5F9B8F8F708330E1
:10F7F000A1F048F4813009F444C3823009F06CC6AA
:10F800001092073841C3863009F4BCC4883009F42B
:10F81000B9C4843009F060C6B5C484E08093D6389A
:10F820000E94AE7745C58F70833009F055C688E0D9
:10F830008093D63800C5853019F5E091D738F0911E
:10F84000D83884819581892B09F446C61092DC381A
:10F850001092DB3882E098E39093DA388093D938BD
:10F860009093E1378093E03710927239109271399A
:10F870001092DF371092DE3788E08093D6381BC1B4
:10F880008091E637853409F027C60091E83710E00B
:10F89000102F00278091E937080F111D8091DE3766
:10F8A0009091DF378017910708F416C61093DF3761
:10F8B0000093DE378091EC378F7309F00DC6F0901E
:10F8C000ED37F11009C680916D3990916E39C09174
:10F8D0002A0AD0912B0A8C179D0759F440916F3951
:10F8E0005091703920912C0A30912D0A42175307FC
:10F8F000A1F02091F6373091F7372817390709F032
:10F90000EBC52091F8373091F93780916F3990919C
:10F9100070392817390709F0DFC50E94137B01965B
:10F9200009F0DAC58091EF37863009F429C18131B9
:10F93000E9F1813009F0D0C58091FA37883009F0BB
:10F94000CBC51092FA378091FC379091FD37873FF5
:10F950006FEF960710F0099601C008969093FD3757
:10F960008093FC378091F2379091F337A091F43770
:10F97000B091F5378093F6379093F737A093F83727
:10F98000B093F93780916D3990916E39A0916F39AC
:10F99000B09170398093F2379093F337A093F43796
:10F9A000B093F53780E48093EE3773C50C5111099D
:10F9B0001093DF370093DE3782E098E39093DA38D4
:10F9C0008093D9388091003890910138892B29F0A3
:10F9D0000E94277B019609F07FC52091FC3730916A
:10F9E000FD372115310509F477C583E799E3909335
:10F9F000D8388093D738A090FA37B090FB37409131
:10FA00002E0A50912F0A6091300A7091310AA0910C
:10FA1000F237B091F3370091F4371091F537E09059
:10FA20002C0AF0902D0AE091D738F091D83889E36C
:10FA3000E53FF80708F050C584819581009721F1D2
:10FA40002817390709F586819781009719F0A816BC
:10FA5000B906D1F4808191818C179D0729F4C28069
:10FA6000D380CE14DF04B1F08417950729F4C28047
:10FA7000D380C616D70671F0A817B90729F482817A
:10FA800093810817190731F03D96F093D838E09329
:10FA9000D738C9CF1092DC381092DB3882E08093DF
:10FAA000D63882E098E39093E1378093E037109264
:10FAB0007239109271390E94AE77809171399091AC
:10FAC0007239009709F408C59C01245E3F4F3093BA
:10FAD000DF372093DE373093E8372093E937E09122
:10FAE000D738F091D83820852093EE3721E1209344
:10FAF000EF3708969827892798279093FF378093A8
:10FB0000FE371092013810920038848195819093CD
:10FB1000FB378093FA37868197819093FD378093E6
:10FB2000FC3780916D3990916E39A0916F39B09109
:10FB300070398093F2379093F337A093F437B093F2
:10FB4000F53780819181A281B3818093F6379093BC
:10FB5000F737A093F837B093F9378EE098E3909396
:10FB6000DA388093D9380E94277B8095909500974A
:10FB700011F48FEF9FEF909301388093003889C480
:10FB80000E94247B019609F0A7C44091FC37509154
:10FB9000FD374115510509F49FC48091FA379091C2
:10FBA000FB37009709F498C46091F2377091F337EE
:10FBB000E091F437F091F537CDEDD8E3298D22238C
:10FBC000A9F0AC81BD814A175B0781F4AE81BF818A
:10FBD0008A179B0759F4A881B9816A177B0731F40A
:10FBE000AA81BB81EA17FB0709F466C1A09629E345
:10FBF000CD35D20719F7809107388F738230D9F449
:10FC00005093251C4093241C80E0843091F0E82F11
:10FC1000F0E0EE0FFF1FE35AF64C208131818F5F39
:10FC20004217530791F71092271C80E0C0E0D0E004
:10FC30007CC08093271C8091073882FD4DC484E1ED
:10FC40008093073888E290E09093DF378093DE3727
:10FC500080E5809306383091013880910538809393
:10FC60000138209100388091043880930038209327
:10FC700004389091FF37809103388093FF37909339
:10FC800003388091FE378093271C409102384093BF
:10FC9000FE37809302383F5F3093053831110DC035
:10FCA0002F5F20930438211108C09F5F9093033881
:10FCB000911103C08F5F809302388091FA37909141
:10FCC000FB379093251C8093241C2091FC373091A6
:10FCD000FD373093FB372093FA379093FD378093AD
:10FCE000FC378091F2379091F337A091F437B091BF
:10FCF000F5378093F6379093F737A093F837B093A2
:10FD0000F93780916D3990916E39A0916F39B0912A
:10FD100070398093F2379093F337A093F437B09310
:10FD2000F5379CC3973089F08F5F8430C1F060E273
:10FD3000869F90011124F901E352F74C918D9111A6
:10FD4000F1CF8093271CEF010CC0209721F0428D4A
:10FD50009A8D941748F7E901C352D74CE5CF8093A9
:10FD6000271C209709F4B8C3D093DC38C093DB3844
:10FD700083E08A8F888F1E8A84E08F8B1B8E809110
:10FD8000FC379091FD379D838C838091FA37909159
:10FD9000FB379F838E838091F2379091F337A09148
:10FDA000F437B091F53788839983AA83BB8381E0C8
:10FDB000898F80912A1C8C8780912B1C8D87809144
:10FDC0002C1C8E8780912D1C8F8781E090E0998B71
:10FDD000888B809101388B87809100388A87809149
:10FDE000FF3789878091FE37888781E090E00E9405
:10FDF000F67A80910638982F907F913508F441C0AB
:10FE000082958F7090E00597880F991F880F991F32
:10FE10002091261CEF2DF0E0E817F90774F5EA5160
:10FE2000F84C20A5211103C01092261C28C02130B7
:10FE300011F4F394EFCF2230D9F431A53430C1F46A
:10FE40002093261CF092271C82A590E0982F8827EB
:10FE500023A5822B9093251C8093241C893C91051B
:10FE600010F088EC90E09B8B8A8B9D8B8C8B09C06B
:10FE700031A5332311F0F30ECDCF2093261CF09241
:10FE8000271C80E180930738809107388260809337
:10FE9000073882E080930E3884E080930F38109208
:10FEA000103888EC809311388CE290E09093DF3723
:10FEB0008093DE3780E680C2D093DC38C093DB3895
:10FEC0001092D63880910738782F7470F72E82FF01
:10FED00003C0198E80E219C29091063892959F70E6
:10FEE000990F990F9093271C091B110904511109AF
:10FEF0001093DF370093DE37922F9F70923029F4F2
:10FF0000982F9F73923139F41FC0913021F4982FAC
:10FF10009F739230C9F0012B19F4982F9370A1F0C0
:10FF20002091FE37988529133DC22091FF3799858E
:10FF3000291338C2209100389A85291333C22091A1
:10FF400001389B8529132EC284FF49C068897989AD
:10FF50006115710509F443C0CE010C960E94C07A68
:10FF6000309102388091E237381339C0209103383C
:10FF70008091E337281333C0909104388091E4379F
:10FF800098132DC0809105384091E537841327C020
:10FF90003C872D879E878F878B8D811119C09E8905
:10FFA000888D2A8D821B292F269526952695821BC2
:10FFB000980F9E8B87FD81952F89322F3695369528
:10FFC000231B820F8F8B969596959695890F888F18
:10FFD00081E08093D638888D8A8F198A188A298D76
:10FFE000E22FEF708E2F90E0FC013197E830F105A1
:10FFF00008F072C28827E656FF4F8F4F0C941A897B
:020000021000EC
:100000008091D63880FF14C083E0898F80E480938C
:10001000D638198A188A8091DE379091DF37009799
:1000200009F405C122E42093D6380E94F67AFFC075
:10003000809107388F73823009F04EC222CF8091B1
:10004000D63880FF6AC0809107388F73823109F0FB
:1000500064C080910638982F907F913508F441C094
:1000600082958F7090E00597880F991F880F991FD0
:100070002091261CEF2DF0E0E817F90774F5EA51FE
:10008000F84C20A5211103C01092261C28C0213055
:1000900011F4F394EFCF2230D9F431A53430C1F408
:1000A0002093261CF092271C82A590E0982F882789
:1000B00023A5822B9093251C8093241C893C9105B9
:1000C00010F088EC90E09B8B8A8B9D8B8C8B09C009
:1000D00031A5332311F0F30ECDCF2093261CF092DF
:1000E000271C83E0898F8091FE3788878091FF37B6
:1000F0008987809100388A87809101388B8781E0D9
:1001000090E00E94F67A82E48093D638198A188AA1
:100110001092DF371092DE378AC080E28093D638A3
:100120000E94AE77E091DB38F091DC38118E83CD00
:100130008091073880FF28C024FD26C088899989CE
:10014000892B09F0C9C18091DE379091DF37019684
:100150000E94F67A8091D638982F90619093D63885
:100160002091DE373091DF37232B19F082618093A5
:10017000D6380E94AE7781E090E0998B888B88E03A
:10018000898F1B8E81E10FC185FF1DC080910C38C6
:1001900090E0982F882730910D38832B4091D938E3
:1001A0005091DA38480F591F5093DA384093D938B4
:1001B0004091DE375091DF37BA01681B790B70939D
:1001C000DF376093DE374091DE375091DF374115DE
:1001D000510551F024FD08C09091D638926090935B
:1001E000D638CA010E94F67A8091083890E0982F9C
:1001F000882720910938820F911D9093251C8093A8
:10020000241C2C893D892817390710F0892B21F4EB
:100210003093251C2093241C8091241C9091251C34
:100220009B8B8A8B8091D638837009F455C11092CC
:100230007239109271390E94AE778091D63885FF5D
:1002400007C01092723910927139198E84E1ABC0D7
:1002500084FF0AC0109272391092713981E090E0E7
:10026000998B888B84E08CCF2091713930917239D1
:1002700021153105E1F080FF02C0198A188A8889AA
:100280009989009781F48A899B898217930720F4C2
:10029000909372398093713980917139909172394C
:1002A000998B888B04C090937239809371391B8E1F
:1002B0008091E0379091E1379093DA388093D93884
:1002C0008091713990917239892B59F08889998977
:1002D000009739F088969093DF378093DE3788E176
:1002E0000BC08091D63881FFF7C088E290E09093F0
:1002F000DF378093DE3780E1809307385CC08091E0
:10030000D63880FFE9C0198E80E18093D6380E94EC
:10031000AE77E2C08091DE379091DF37009711F021
:100320000E94F67A909107388091D63890FF0BC0E2
:1003300080FF06C087E0898F1A8E198A188A19C033
:1003400086E0898F16C080FF1EC085E0898F198ADC
:10035000188AC2C08091DE379091DF37009711F084
:100360000E94F67A8091073880FF0DC087E0898F60
:100370001A8E81E090E00E94F67A80E18093D63870
:100380000E94AE770FC08091DE379091DF37892BC6
:1003900049F4A2C08091D63880FF9EC087E0898F43
:1003A0001A8E9AC080E18093073888E290E090939B
:1003B000DF378093DE3780E5809306388885809329
:1003C00002388985809303388A85809304388B8529
:1003D000809305388C858093FE378D858093FF3719
:1003E0008E85809300388F858093013886E08093D6
:1003F000EF378C819D819093FB378093FA378E8104
:100400009F819093FD378093FC3780916D39909157
:100410006E39A0916F39B09170398093F237909313
:10042000F337A093F437B093F53788819981AA8187
:10043000BB818093F6379093F737A093F837B0934A
:10044000F937898D84FF05C0109209381092083859
:1004500005C01092083888EC8093093880E48093B6
:10046000EE378091DE379091DF379093E8378093B5
:10047000E93710920D3810920C3810920B38109208
:100480000A380E94247B8095909590930B38809336
:100490000A3885E48093E6371092E7371092ED37FB
:1004A0001092EC3780912E1C90912F1C0196909306
:1004B0002F1C80932E1C9093EA378093EB37109279
:1004C000F1371092F0370E94137B809590959093AE
:1004D000F1378093F03704C01092DF371092DE3787
:1004E0001092D638DF91CF911F910F91FF90EF902E
:1004F000DF90CF90BF90AF90089582E39CE10C9481
:1005000096719093311C8093301C089582E39CE196
:100510000C949A71EF92FF920F931F93CF93DF93F6
:100520008C01EB017A0182E39CE10E949A710097B1
:10053000D9F0DC0112962D913C9113972C173D07B1
:1005400081F41696ED91FC911797309769F0970119
:10055000AE01B801DF91CF911F910F91FF90EF9005
:1005600019940E94FF71E3CFDF91CF911F910F91FA
:10057000FF90EF90089508950F931F93CF93DF930B
:10058000C3E7DCE1488159816A817B8100E010E0AA
:1005900026EE32E883E59CE10E94CF6D0E9432672F
:1005A000BC0180E090E0288139814A815B810E9412
:1005B000D988AB01BC012BE033E88FE39CE10E94BA
:1005C000CF6DDF91CF911F910F9108958091731C92
:1005D0009091741CA091751CB091761C40916F1C79
:1005E0005091701C6091711C7091721C880F991F42
:1005F000AA1FBB1F481759076A077B0710F4DB01C6
:10060000CA018093731C9093741CA093751CB093C3
:10061000761C0C94BC82CF93DF930E94BB750E9422
:100620002A75EC01198218820E94868228813981FC
:10063000009719F1FC0140854423F9F0FC01428147
:100640005381F901EE0FFF1FEE0FFF1FEC0FFD1F8F
:1006500053834283FC01448155812F5F3F4FF90151
:10066000EE0FFF1FEE0FFF1FEC0FFD1F51834083A6
:10067000398328830E94FF71D9CFC901880F991F40
:10068000880F991F02960E94257588819981892B70
:1006900031F084E39CE1DF91CF910C94E173DF9121
:1006A000CF910895AF92BF92CF92DF92EF92FF92D7
:1006B0000F931F93CF93DF931F921F92CDB7DEB797
:1006C0005B010E942A758C01FC01E080F180FA82B6
:1006D000E9820E9472759701220F331F220F331F88
:1006E0002E5F3F4F8217930798F0C12CD12CCE1468
:1006F000DF0471F0F8014481558162817381C50185
:100700000E948A82FFEFCF1ADF0A0C5F1F4FEFCFE4
:100710000F900F90DF91CF911F910F91FF90EF906D
:10072000DF90CF90BF90AF9008950F93013099F470
:100730008091671C9091681CA091691CB0916A1C03
:100740008093731C9093741CA093751CB093761CBB
:100750000F910C94BC820F9108954F925F926F920B
:100760007F928F929F92AF92BF92CF92DF92EF9241
:10077000FF920F931F932A013B014801590142E365
:100780005AE0BC0184E39CE10E94C473E4E3FCE111
:1007900043AA54AA65AA76AA87AA90AEA1AEB2AE21
:1007A000C3AED4AEE5AEF6AE85E993E81F910F91E6
:1007B000FF90EF90DF90CF90BF90AF909F908F9081
:1007C0007F906F905F904F900C9481820C94EE73A9
:1007D000CF93DF93E091360AF091370A1995EC0137
:1007E000892B29F06A817B8181E00E940F76CE01FE
:1007F000DF91CF9108950F931F93CF93DF93EC0177
:10080000E091380AF091390A19958C016A817B814F
:1008100081E00E940F7681E090E0012B11F480E0EE
:1008200090E0DF91CF911F910F910895E0913A0AE6
:10083000F0913B0A1994CF93DF93FC01DB0185E033
:10084000EB0119928A95E9F78581837011F082E0B6
:100850008C938781837021F082E012968C9312979B
:100860008581837081F08781837069F02389348961
:10087000818592852817390731F481E084831296A7
:100880001C92129701C0148285818370823029F0F6
:10089000833011F488E001C080E011968C931197A9
:1008A00087818370823029F0833011F488E001C0A1
:1008B00080E013968C93DF91CF910895CF93DF93CF
:1008C00000D01F921F92CDB7DEB7BE016F5F7F4F82
:1008D0000E941B84898190E003962A81820F911DDA
:1008E0002B81820F911D2C81820F911D2D81820FF2
:1008F000911D0F900F900F900F900F90DF91CF915F
:1009000008953F924F925F926F927F928F929F9243
:10091000AF92BF92CF92DF92EF92FF920F931F930D
:10092000CF93DF9300D01F921F92CDB7DEB78C011B
:100930007B013A01BE016F5F7F4F0E941B8469817A
:100940007A81472F50E0EB813C80232D30E0862FC9
:1009500090E00396840F951F8E0F911D820F931FB9
:10096000AD818A0F911D681679060CF4A4C0D801D8
:1009700011968C91119780FB882480F8912C83E04C
:10098000880C991C8A95E1F712968C91129780FB3E
:10099000AA24A0F8B12C94E0AA0CBB1C9A95E1F70C
:1009A0008A288C918770882A13968C91139780FBE4
:1009B000CC24C0F8D12CF5E0CC0CDD1CFA95E1F785
:1009C000C82814968C9180FB442440F8512CA6E052
:1009D000440C551CAA95E1F74C28D7014C92D8013C
:1009E00015968C918370B4E08B9F60011124D8011F
:1009F00016969C919370B0E19B9FC00111248C29A5
:100A0000D8011796FC9190E4F99FD00111248A2B0C
:100A1000D70111968C93D80118968C91D701129614
:100A20008C93623071F4D80119968C91D70113968A
:100A30008C93D8011A968C91D70114968C9385E0EB
:100A400001C083E0780F872F972F941B4115510524
:100A500061F041505109D801A40FB51F1B968C912C
:100A6000D701A90FB11D8C93EECFE23071F4D701FD
:100A7000A70FB11DF80193899C9391E0970FD701BF
:100A8000A90FB11D8E5F94899C93F32DF80F8F2FC2
:100A9000821B2115310561F021503109D801A20FC7
:100AA000B31F55969C91D701A80FB11D9C93EFCF12
:100AB0008F2F90E002C080E090E00F900F900F9099
:100AC0000F900F90DF91CF911F910F91FF90EF90BA
:100AD000DF90CF90BF90AF909F908F907F906F905E
:100AE0005F904F903F900895AF92BF92CF92DF9268
:100AF000EF92FF920F931F93CF93DF9363307105B3
:100B00000CF4B3C0EA016B017C01FC01908196FBFF
:100B1000AA24A0F88181282F269526952370B82E27
:100B2000B294B694B69453E0B522392F3770388317
:100B300093FB332730F9398394FB332730F93A8319
:100B400095FB992790F99B83AC822D8382958370C6
:100B50008E83BF8282818887222379F133818481C9
:100B600090E0982F8827830F911D9A8789878701A6
:100B70000B5F1F4F223071F460E07AE0CE010B96DC
:100B80000E94DC74F70186818B8785818C870E5FDC
:100B90001F4F1EC02330E1F4F7013D96DE011B9686
:100BA0009E012D5E3F4F9E2F8F2F42914D93A21796
:100BB000B307D9F7092F182F0BC087010D5F1F4FFF
:100BC00060E07AE0CE010B960E94DC741A861986EA
:100BD000BB20A1F1A1100DC0F8012081818190E01E
:100BE000982F8827820F911D9C8B8B8B0E5F1F4F38
:100BF00004C089859A859C8B8B8BF2E0BF120EC056
:100C000060E07AE0CE0145960E94DC74F8018181B3
:100C10008D8B80818E8B0E5F1F4F18C0F3E0BF124B
:100C200015C0085F1F4FD801FE017596CE014D9685
:100C30002E912193E817F907D9F708C060E07AE010
:100C4000CE0145960E94DC741C8A1B8A98012E19DD
:100C50003F09C601821B930B98AB8FA71EA70DA758
:100C6000C216D30614F0C90102C080E090E0DF9103
:100C7000CF911F910F91FF90EF90DF90CF90BF9099
:100C8000AF90089520E030E00296FC013297408159
:100C9000442331F0FC0131974081240F311DF4CF02
:100CA000C9010895FC01208130E0322F2227818183
:100CB000282B02C0220F331F6A95E2F7232F332718
:100CC000FA01E45CF54F808190E08223932328E0D1
:100CD00030E0241B350B02C0969587952A95E2F7E4
:100CE00008956F927F928F929F92AF92BF92CF9210
:100CF000DF92EF92FF920F931F93CF93DF937C01CC
:100D00008B015A01E9012830310544F4A901B501EC
:100D1000C8010E945286F701808346C0690183E0C2
:100D2000D594C7948A95E1F7452B21F04701612CB2
:100D3000712C06C0FB01D701CB018C0D9D1D1FC07E
:100D400048E050E0B501C801860D971D0E9452860B
:100D5000F40181934F01FFEF6F1A7F0A6C147D0439
:100D600079F7AE014770552741155105E9F0E701C4
:100D7000C60DD71DB501C801860D971D12C0E81715
:100D8000F90719F021912D93FACFAE01477055273D
:100D90004115510549F0E701CC0DDD1D60E070E023
:100DA000CF010E9452868883DF91CF911F910F91CE
:100DB000FF90EF90DF90CF90BF90AF909F908F907B
:100DC0007F906F9008958F929F92AF92BF92CF9233
:100DD000DF92EF92FF920F931F93CF93DF931F92B7
:100DE0001F92CDB7DEB70E942A758C0182E090E099
:100DF0000E940875892B19F480E090E05FC0F8012B
:100E0000218130E0322F22278081A901480F511D16
:100E1000CA010E94FF737C01892B71F30E942A751D
:100E20004C01F7019681292F26952695269530E0CD
:100E3000977041E050E011F440E050E0C901840FA8
:100E4000951F0E940875892BB9F2F701048115815D
:100E5000A12CB12CF8018081882379F1F801C1809F
:100E6000D12CA50147705527B50193E0759567957D
:100E70009A95E1F7680D791D883168F09601CE01E9
:100E800001960E947186BE016F5F7F4FF8018081DD
:100E90000E9423760DC01A8219829601CE01019616
:100EA0000E94718669817A81F80180810E940F76A3
:100EB000AC0CBD1C0E5F1F4FCDCFC7010F900F9024
:100EC000DF91CF911F910F91FF90EF90DF90CF9026
:100ED000BF90AF909F908F900895DC0150E0E0E1CB
:100EE000F0E0CF01861B970B821B930B02C0440FCF
:100EF000551F8A95E2F78C91852B8C9311968C91D6
:100F00001197482B11964C9308956F927F928F9270
:100F10009F92AF92BF92CF92DF92EF92FF920F9388
:100F20001F93CF93DF93283031051CF4FA014081E1
:100F30005AC05901E3E0B594A794EA95E1F7611529
:100F4000710541F03901EA018B017C014A01C12C94
:100F5000D12C05C0EA01FC014A0D5B1D2AC0F40139
:100F600041914F0128E030E0B801C7018C0D9D1D73
:100F70000E946D87FFEFCF1ADF0ACA14DB0479F7EE
:100F800093012770332721153105E9F1CC0DDD1DC3
:100F9000488150E0021B130B085F1F4F02C055959C
:100FA00047950A95E2F760E070E0C7018C0D9D1D42
:100FB0001AC0C417D50719F069916193FACF277049
:100FC000332721153105F9F0488150E068E070E0E1
:100FD000621B730B02C0559547956A95E2F760E076
:100FE00070E08A0D9B1DDF91CF911F910F91FF90B3
:100FF000EF90DF90CF90BF90AF909F908F907F90B9
:101000006F900C946D87DF91CF911F910F91FF909E
:10101000EF90DF90CF90BF90AF909F908F907F9098
:101020006F9008956F927F928F929F92AF92BF922E
:10103000CF92DF92EF92FF920F931F93CF93DF93A4
:101040001F921F92CDB7DEB77C01FC018681082F6D
:10105000069506950695202F30E0877001E010E098
:1010600011F400E010E0020F131FC80102960E9465
:101070008475009709F448C00E943175F7012281F8
:10108000FC012083F7012381FC0121830E9431753B
:1010900002965C01A80160E070E00E946493F70191
:1010A000048115810F5F1F4F812C912CF80131971E
:1010B0008081882339F1F801C080D12C3401F7E018
:1010C0006F227724740193E0F594E7949A95E1F701
:1010D000EA0CFB1C883128F00E942D769601AC01A9
:1010E00008C00E941A769A8389839601AE014F5FE9
:1010F0005F4FB301C7010E9485878C0C9D1C0E5F5A
:101100001F4FD4CF81E090E00F900F90DF91CF91EF
:101110001F910F91FF90EF90DF90CF90BF90AF9015
:101120009F908F907F906F900895DB018F939F9396
:101130000E944089BF91AF91A29F800D911DA39FF6
:10114000900DB29F900D11240895991B79E004C071
:10115000991F961708F0961B881F7A95C9F78095F6
:101160000895AA1BBB1B51E107C0AA1FBB1FA617EE
:10117000B70710F0A61BB70B881F991F5A95A9F740
:1011800080959095BC01CD01089597FB072E16F42C
:10119000009407D077FD09D00E94B18807FC05D0E4
:1011A0003EF4909581959F4F0895709561957F4F7E
:1011B0000895A1E21A2EAA1BBB1BFD010DC0AA1F98
:1011C000BB1FEE1FFF1FA217B307E407F50720F0B0
:1011D000A21BB30BE40BF50B661F771F881F991F2B
:1011E0001A9469F760957095809590959B01AC0174
:1011F000BD01CF010895052E97FB1EF400940E94B7
:10120000128957FD07D00E94D98807FC03D04EF4FD
:101210000C94128950954095309521953F4F4F4F32
:101220005F4F089590958095709561957F4F8F4F92
:101230009F4F0895EE0FFF1F881F8BBF0790F691F9
:10124000E02D19940E942A89332312F48A1B9B0BE8
:101250000C943B89A29FB001B39FC001A39F700D66
:10126000811D1124911DB29F700D811D1124911DAE
:1012700008950E942A89B7FF0895821B930B089551
:101280000E942A89A59F900DB49F900DA49F800D68
:10129000911D11240895B7FF0C9440890E94408944
:1012A000821B930B0895DF93CF931F930F939A9D07
:1012B000F02D219FF00D8B9DF00D8A9DE02DF10DFD
:1012C000039FF00D029FE00DF11D4E9DE00DF11DFD
:1012D0005E9DF00D4F9DF00D7F936F93BF92AF9287
:1012E0005F934F93D5010E942A898B01AC01D701EE
:1012F0000E942A89EB01E80FF91FD6010E94A389F9
:101300002F913F91D6010E942A89C60FD71FE81F4F
:10131000F91FAF91BF910E94A3892F913F910E9425
:101320002A89C60FD71FE81FF91FD6010E942A89F4
:10133000E60FF71F9801BE01CF0111240F911F91F5
:10134000CF91DF9108950E942A89460F571FC81F29
:10135000D91F08F431960895E894DF93CF93FC01E8
:10136000DB010E942A897F936F93E9019A01AC0106
:10137000BF93AF933F932F93DF010E942A8926F4F6
:101380006C1B7D0B820B930B9E01EB01FC010E94F9
:10139000A389AF91BF912F913F910E94A389BE0174
:1013A000CF01F9012F913F91CF91DF91089568947A
:1013B00001C0E894F92FF12B12F00C940B8AA0E0F5
:1013C000B0E0E5EEF9E80C947D8A092E059422F44C
:1013D0000E94678A112392F4F0E80F26FFEFE09451
:1013E000F09400951095B094C094D094A194BF0A45
:1013F000CF0ADF0AEF0AFF0A0F0B1F0B0E94168AA3
:1014000007FC0E94678ACDB7DEB7ECE00C94998A9E
:10141000689401C0E8948F929F92CF93DF930E94CB
:10142000168ADF91CF919F908F90089588249924F8
:10143000F401E401B0E49F93AA279A158B049C045D
:10144000ED05FE05CF05D007A10798F4AD2FDC2FE1
:10145000CF2FFE2FE92D982C892E982F872F762FAE
:10146000652F542F432F322F2227B85031F7BF91C9
:1014700027C01B2EBF91BB27220F331F441F551FB0
:10148000661F771F881F991F881C991CEE1FFF1F5E
:10149000CC1FDD1FAA1FBB1F8A149B04EC05FD0592
:1014A000CE05DF05A007B10748F08A189B08EC09B4
:1014B000FD09CE09DF09A00BB10B21601A94E1F6FA
:1014C0002EF49401AF01BE01CD01000C089560958A
:1014D00070958095909530954095509521953F4F0A
:1014E0004F4F5F4F6F4F7F4F8F4F9F4F08952F92FA
:1014F0003F924F925F926F927F928F929F92AF92A4
:10150000BF92CF92DF92EF92FF920F931F93CF93F0
:10151000DF93CDB7DEB7CA1BDB0B0FB6F894DEBF87
:101520000FBECDBF19942A88398848885F846E849D
:101530007D848C849B84AA84B984C884DF80EE80F7
:10154000FD800C811B81AA81B981CE0FD11D0FB600
:10155000F894DEBF0FBECDBFED0108950F930830A4
:1015600090F0982F872F762F652F542F432F322FEF
:1015700022270850F4CF220F331F441F551F661F28
:10158000771F881F991F0A95B2F70F91089597FB4F
:1015900010F8169400080F93083098F00850232F85
:1015A000342F452F562F672F782F892F902DF4CF6A
:1015B00005949795879577956795579547953795AE
:1015C00027950A95AAF70F9108952A0D3B1D4C1DEA
:1015D0005D1D6E1D7F1D801F911F08950024A7FDB6
:1015E00000942A0F301D401D501D601D701D801D70
:1015F000901D08952A193B094C095D096E097F0960
:10160000800B910B08952A153B054C055D056E0571
:101610007F058007910708950024A7FD00942A17ED
:10162000300540055005600570058005900508955A
:101630005058BB27AA270E94308B0C949B8D0E9488
:101640008D8D38F00E94948D20F039F49F3F19F46D
:1016500026F40C94538D0EF4E095E7FB0C944D8D1D
:10166000E92F0E94AC8D58F3BA17620773078407FD
:10167000950720F079F4A6F50C94CE8D0EF4E09544
:101680000B2EBA2FA02D0B01B90190010C01CA013C
:10169000A0011124FF27591B99F0593F50F4503EE7
:1016A00068F11A16F040A22F232F342F4427585FD9
:1016B000F3CF469537952795A795F0405395C9F7F1
:1016C0007EF41F16BA0B620B730B840BBAF09150A9
:1016D000A1F0FF0FBB1F661F771F881FC2F70EC048
:1016E000BA0F621F731F841F48F48795779567951B
:1016F000B795F7959E3F08F0B0CF9395880F08F007
:101700009927EE0F9795879508950E948D8D60F02B
:1017100080E891E009F49EEF0E94948D28F040E863
:1017200051E071F45EEF0CC00C94538D0C94CE8D8F
:10173000E92FE0780E94AC8D40F3092E052AB1F321
:10174000261737074807590738F00E2E07F8E02507
:1017500069F0E025E0640AC0EF6307F8009407FA37
:10176000DB01B9019D01DC01CA01AD01EF930E94CB
:10177000138C0E949B8D0E94C88B5F91552339F07A
:101780002BED3FE049E450FD49EC0C94198B089592
:10179000DF93DD27B92FBF7740E85FE31616170602
:1017A00048075B0718F4D92F0E94DA8D9F938F9317
:1017B0007F936F930E94658FE4E4F1E00E94668D51
:1017C0000E949B8D2F913F914F915F910E94BB8E04
:1017D000DD2351F09058A2EA2AED3FE049EC5FE3A7
:1017E000D0785D270E94308BDF910C949B8D0E94F6
:1017F000298D08F481E008950E94108C0C949B8D33
:101800000E94948D58F00E948D8D40F029F45F3F26
:1018100029F00C944D8D51110C94CF8D0C94538D57
:101820000E94AC8D68F39923B1F3552391F3951B76
:10183000550BBB27AA2762177307840738F09F5FF1
:101840005F4F220F331F441FAA1FA9F335D00E2E5E
:101850003AF0E0E832D091505040E695001CCAF7CB
:101860002BD0FE2F29D0660F771F881FBB1F26178E
:1018700037074807AB07B0E809F0BB0B802DBF0165
:10188000FF2793585F4F3AF09E3F510578F00C9434
:101890004D8D0C94CF8D5F3FE4F3983ED4F3869545
:1018A00077956795B795F7959F5FC9F7880F911D55
:1018B0009695879597F90895E1E0660F771F881F41
:1018C000BB1F621773078407BA0720F0621B730BF4
:1018D000840BBA0BEE1F88F7E095089529F416F0F3
:1018E0000C944D8D0C94CE8D0C94538D0E94B48D20
:1018F000A8F39638A0F707F80F92E8942BE33AEA9A
:1019000048EB5FE70E94BE8E0F920F920F924DB789
:101910005EB70F920E94748EE1E7F1E00E94668D3F
:101920004F915F91EF91FF91E595EE1FFF1F49F0F9
:10193000FE57E0684427EE0F441FFA95E1F7419502
:10194000550B0E94E68D0F9007FE0C94DA8D0895DA
:1019500097FB16F40E94568D0C94EC8CE89409C009
:1019600097FB3EF490958095709561957F4F8F4FD2
:101970009F4F9923A9F0F92F96E9BB279395F695E8
:10198000879577956795B795F111F8CFFAF4BB0F66
:1019900011F460FF1BC06F5F7F4F8F4F9F4F16C0CA
:1019A000882311F096E911C0772321F09EE8872F54
:1019B000762F05C0662371F096E8862F70E060E010
:1019C0002AF09A95660F771F881FDAF7880F969589
:1019D000879597F90895E894F92F96EBFF2381F006
:1019E000121613061406440B9395F6958795779572
:1019F000679557954040FF23B9F71BC09927089575
:101A0000882351F49850D2F7872B762F652F542FC7
:101A1000432F322F20E0B1F3121613061406440BA5
:101A200088233AF09A95440F551F661F771F881F29
:101A3000CAF755234AF4440F551F11F460FF04C040
:101A40006F5F7F4F8F4F9F4F880F9695879597F9C0
:101A50000895990F0008550FAA0BE0E8FEEF16163F
:101A60001706E807F907C0F012161306E407F50792
:101A700098F0621B730B840B950B39F40A2661F006
:101A8000232B242B252B21F408950A2609F4A140A9
:101A9000A6958FEF811D811D089597F99F6780E8B6
:101AA00070E060E008959FEF80EC08959095809538
:101AB0007095609550954095309521953F4F4F4FCB
:101AC0005F4F6F4F7F4F8F4F9F4F0895DF93CF939F
:101AD0001F930F93FF92EF92DF927B018C0168942A
:101AE00006C0DA2EEF010E94BB8EFE01E894A5919C
:101AF0002591359145915591A6F3EF010E94308BC8
:101B0000FE019701A801DA9469F7DF90EF90FF904A
:101B10000F911F91CF91DF91089500240A9416161A
:101B2000170618060906089500240A9412161306CB
:101B3000140605060895092E0394000C11F4882359
:101B400052F0BB0F40F4BF2B11F460FF04C06F5F75
:101B50007F4F8F4F9F4F089557FD9058440F551F4B
:101B600059F05F3F71F04795880F97FB991F61F01F
:101B70009F3F79F087950895121613061406551F96
:101B8000F2CF4695F1DF08C0161617061806991F02
:101B9000F1CF86957105610508940895E894BB27F7
:101BA00066277727CB0197F908950E94298D08F4BD
:101BB0008FEF08959B01AC0160E070E080E89FE347
:101BC0000C94FC8B0C944D8D0C94698F0E94B48DF9
:101BD000D8F39923C9F3940F511DA3F391505040AA
:101BE00094F059F0882332F0660F771F881F9150C8
:101BF0005040C1F79E3F51052CF7880F911D9695D7
:101C0000879597F908955F3FACF0983E9CF0BB270D
